:020000040800F2
:10000000000400204B010008590100085B010008B2
:100010005D0100085F0100086101000800000000A8
:100020000000000000000000000000006301000864
:10003000650100080000000067010008851C000839
:10004000A52D00087D170008AD2800082519000817
:10005000830D000821190008750D0008790D0008AE
:100060007B0D00087D0D00087F0D00086B01000866
:100070006B0100086B0100086B010008D50B00083C
:100080006B0100086B0100086B0100086B010008A0
:100090006B0100086B0100086B010008810D00086E
:1000A000AF280008B5280008B3280008B1280008C8
:1000B000B7280008B9280008BB2800083515000833
:1000C0003315000839150008371500088B1A000889
:1000D0008D1A00084D2C00084F2C0008512C0008E8
:1000E000770D000823190008412D00086B01000856
:1000F0006B0100086B0100086B0100086B01000830
:100100006B0100086B0100086B0100086B0100081F
:100110006B0100086B0100086B0100086B0100080F
:100120006B0100086B0100086B0100086B010008FF
:10013000DFF810D000F042FA004800471D5B0008CD
:10014000AFF30080C84C002070470848804708493A
:1001500081F3088807480047FEE7FEE7FEE7FEE771
:10016000FEE7FEE7FEE7FEE7FEE7FEE749010008DF
:10017000C84C00203101000840EA01039B0703D06E
:1001800009E008C9121F08C0042AFAD203E011F8D6
:10019000013B00F8013B521EF9D27047421C10F897
:1001A000011B0029FBD1801A7047034611F8012B6F
:1001B00000F8012B002AF9D11846704730B50B46DC
:1001C000014600202022012409E021FA02F59D4287
:1001D00005D303FA02F5491B04FA02F52844151E5B
:1001E000A2F10102F1DC30BD2DE9F05F05460020EF
:1001F00092469B4688460646814640241BE0284698
:1002000041464746224600F0FAF953465A46C01A7C
:10021000914110D311461846224600F0E1F92D1AFB
:1002200067EB01084F4622460120002100F0D8F973
:1002300017EB00094E41201EA4F10104DFDC484603
:1002400031462A464346BDE8F09F2DE9FE4F8046E1
:1002500081EA0300C00F0C46009021F0004123F01A
:100260000045B8EB0200A94105D240462146904620
:100270001C460B46024623F00040104347D0270D92
:10028000C7F30A00C3F30A510290401A01904028B4
:100290006BDAC3F3130040F4801B0098924620B140
:1002A0000023D2EB030A63EB0B0B01985946C0F114
:1002B0004002504600F094F906460D465046594615
:1002C000019A00F0ACF910EB08006141002487EAC4
:1002D000115284EAE7731A4340D0009A62B3019A3C
:1002E000012A4FEA075215DC001B61EB02014FF0B7
:1002F000004202EA0752CDE90042001C41F580119C
:1003000032462B4600F0ACF903B0BDE8F08F404612
:100310002146F9E7001B61EB0201001C41F5801347
:1003200000185B412018A2F5001747EB030140EAD3
:10033000D570B6196D4111E06D084FEA360645EAF1
:10034000C0754FEA0752001B61EB0201001C41F52A
:10035000801149084FEA30000019514132462B46BE
:1003600003B0BDE8F04F00F06CB9009801224000E6
:100370000023D0EB020263EBE073009821464FEAC2
:10038000E074B8EB000061EB0401E9E783F000439F
:100390005BE781F0004158E72DE9FE4F81EA030455
:1003A00004F0004421F0004100944FF0000B23F0D2
:1003B000004350EA01045ED052EA03045BD0C3F369
:1003C0000A54C1F30A552C44A4F2F3340194A0FB5F
:1003D0000254C1F3130141F48011C3F3130343F436
:1003E000801301FB024400FB034E840A970A44EA8F
:1003F000815447EA8357A4FB076802958D0A05FBE1
:1004000007854FEA932C04FB0C542705029D4FEA05
:10041000065847EA1637B5EB08056EEB070C870E52
:10042000920E47EA811742EA8312A7FB0201B6EB5C
:100430000B0164EB00042B0D43EA0C335E1844EB14
:100440001C50DA465146E7FB0201C5F313044FEA9C
:100450000B3343EA14534FEA0432019C43EA060388
:10046000A4F10C040294009CCDE900B400F0F8F86B
:1004700003B0BDE8F08F00200146F9E72DE9F04D0B
:1004800081EA030404F0004B21F0004514464FF0CC
:10049000000A23F0004150EA050220D054EA01028C
:1004A0001DD0C5F30A570246C5F31303C1F3130069
:1004B000C1F30A5640F4801543F48013A7EB0608F5
:1004C000101BD64608F2FD3873EB050002D308F185
:1004D000010801E092185B41B8F1000F03DA002037
:1004E0000146BDE8F08D00204FF480110646844699
:1004F0000EE0171B73EB050705D3121B63EB050317
:1005000006434CEA010C49084FEA300092185B415F
:1005100050EA0107EDD152EA030012D082EA04004A
:1005200083EA0501084305D0101BAB4106D2012226
:10053000002306E000224FF0004302E06FF00102CA
:1005400053101AEB06004CEB085110EB0A0041EB7C
:100550000B01BDE8F04D00F074B8C1F30A52C1F3CD
:10056000130140F2FF3341F480119A4202DA002075
:100570000146704740F233439A42A2F2334202DC12
:10058000524200F03CB800F02BB8000030B5041E19
:1005900071F1000404DB4FF00044404264EB0101C0
:1005A000141E73F1000405DB1C464FF00043524259
:1005B00063EB0403994208BF904230BD064C074DDF
:1005C00006E0E06840F0010394E807009847103423
:1005D000AC42F6D3FFF7B0FD0C6701082C670108A9
:1005E000202A04DB203A00FA02F1002070479140F3
:1005F000C2F1200320FA03F3194390407047202AE8
:1006000004DB203A21FA02F00021704721FA02F3BC
:10061000D040C2F120029140084319467047202A79
:1006200006DBCB17203A41FA02F043EAE07306E01A
:1006300041FA02F3D040C2F120029140084319462A
:10064000704710B5141E73F1000408DA401C41F124
:10065000000192185B411A4301D120F0010010BD46
:100660002DE9F04D92469B4611B1B1FA81F202E0BC
:10067000B0FA80F220329046FFF7B2FF04460F46F0
:1006800040EA0A0041EA0B0153465A46084313D098
:10069000114653EA010019D0C8F140025046FFF755
:1006A000AEFF05460E46504659464246FFF798FFB4
:1006B000084305D0012004E020463946BDE8F08D0E
:1006C0000020054346EAE0762C4337430A98630549
:1006D000E40AA0EB08000022FD0A44EA47540A306D
:1006E00002D500200146E9E7010510196941DDE95D
:1006F000084500196941BDE8F04DA2E770B58C18B6
:1007000010F8015B15F0070301D110F8013B2A1125
:1007100006D110F8012B03E010F8016B01F8016B12
:100720005B1EF9D12B0705D40023521E0DD401F80E
:10073000013BFAE710F8013BCB1A921C03E013F8D7
:10074000015B01F8015B521EF9D5A142D8D300200C
:1007500070BD21B1826842F00102826003E08268CC
:1007600022F001028260704721B1826842F48072F7
:10077000826003E0826822F4807282607047000029
:1007800010B504461548204430B1B0F5806F0DD047
:10079000B0F5C05F1ED113E00121480201F03CF822
:1007A00000214FF4007001F037F814E001218802B5
:1007B00001F032F800214FF4806001F02DF80AE0DA
:1007C0000121C80301F028F800214FF4004001F096
:1007D00023F800E000BF00BF10BD000000DCFEBF3A
:1007E00021B1826842F48012826003E0826822F4C0
:1007F000801282607047014600208A6802F004027D
:100800000AB1012000E000207047014600208A68FC
:1008100002F008020AB1012000E000207047000049
:1008200030B502460020002350680F4C20400D795F
:100830000C6844EA05242043506090680B4C20402B
:10084000D1E902542C434D7944EA45042043906099
:10085000D06A20F470000C7C641E1C43E3B240EAB2
:100860000350D06230BD0000FFFEF0FFFDF7F1FF46
:10087000F0B504460D4600200021092D11DDE06889
:10088000A5F10A0606EB4607072606FA07F1884394
:10089000A5F10A0606EB460603FA06F10843E060F6
:1008A0000CE0206905EB4507072606FA07F18843A7
:1008B00005EB450603FA06F108432061072A0FDA23
:1008C000606B561E06EB86071F2606FA07F1884363
:1008D000561E06EB860605FA06F10843606322E021
:1008E0000D2A0FDA206BD61F06EB86071F2606FAA5
:1008F00007F18843D61F06EB860605FA06F1084382
:10090000206310E0E06AA2F10D0606EB86071F26C1
:1009100006FA07F18843A2F10D0606EB860605FAF2
:1009200006F10843E062F0BD816841F00801816092
:10093000704721B1826842F4A002826003E08268BD
:1009400022F4A00282607047816841F00401816056
:100950007047000010B500EB80034FF6FF7404EA07
:100960008303074C2380074B1A8001EB8103248803
:1009700004EB8303044C23800023044C238010BD2C
:1009800008000020060000200A0000200C000020C3
:10099000F0B53A4EB6F8DC615EB9002004E0384E9E
:1009A00026F81000461CB0B240F25D56B042F6DBAD
:1009B00062E00021314EB6F8DC210024B6F8DE51A9
:1009C00008460EE08A420AD02E1B471A7E43571A69
:1009D00096FBF7F62644B7B2294E26F81070461C4F
:1009E000B0B29042EEDB00232FE0254E3E3E36F8BB
:1009F00023602EB1224E3E3E06EB8306768806B972
:100A000025E01F4E3E3E36F823105F1C36F82720A7
:100A100006EB830674881A4E3E3E06EB8706758801
:100A200008460EE08A420AD02E1B471A7E43571A08
:100A300096FBF7F62644B7B2114E26F81070461C06
:100A4000B0B29042EEDB5E1CB3B20E2BCDDB00BF2A
:100A50000EE08A420AD02E1B471A7E43571A96FB95
:100A6000F7F62644B7B2064E26F81070461CB0B210
:100A700040F25D56B042ECDBF0BD00001C020020ED
:100A80003604002070B500F0D7FE00F07BF900F0CE
:100A90001DFE16480068C822B0FBF2F1B1F1807F5C
:100AA00001D301201DE021F07F40401E4FF0E022E5
:100AB000506150170022002807DA13071D0E0C4B57
:100AC00000F00F04241F1D5503E013071C0E094BF3
:100AD0001C5400BF00204FF0E022906107201061FD
:100AE000002008B100BFFEE770BD0000F8660108F5
:100AF00018ED00E000E400E02DE9FC4106460C465C
:100B0000174600F01BFD32480670002E59D004EB4A
:100B1000840040002E49486007EB87004000C86011
:100B2000A0B2694600F014FDBDF80200642190FBFC
:100B3000F1F094FBF1F188420AD125490198086649
:100B4000BDF80000C1F88C000846C0F884400FE0F2
:100B5000A4F2F2300A2190FBF1F0C0EB001040004B
:100B60001B4908660A20C1F88C000846C0F884407A
:100B700000201749C1F8880040F2F230001B88605D
:100B800008468068322801DA3220886013F08AFC37
:100B900005460DB1FF2D0ED14FF47A700C498866D1
:100BA0000846806E0A2190FBF1F000F0FF084046F5
:100BB00013F089FC09E005EB8500400004498866D4
:100BC00003E00020024948600867BDE8FC8100009E
:100BD000FC3D0020704721B1026842F00102026032
:100BE00003E0026822F0010202607047016821F010
:100BF000010101600021016041608160C160484ADB
:100C0000811A90425BD012DC464AA0EB020190426E
:100C10003AD007DC44490144D9B1142922D028290B
:100C20007AD128E0142938D0282975D13EE0B1F5D1
:100C30006C7F5BD006DCB1F5627F49D0B1F5677F90
:100C40006AD14CE0B1F5717F57D0B1F5767F63D1B1
:100C50005BE034494439496841F00F01314A443A74
:100C600051605AE02F494439496841F0F0012D4A5A
:100C7000443A516051E02B494439496841F470616C
:100C8000284A443A516048E026494439496841F4C9
:100C90007041244A443A51603FE02249443949684E
:100CA00041F470211F4A443A516036E01D494439ED
:100CB000496841F470011B4A443A51602DE01949DA
:100CC0004439496841F07061164A443A516024E061
:100CD0001649096841F00F01144A11601DE01349DB
:100CE000096841F0F001114A116016E00F490968E6
:100CF00041F470610D4A11600FE00C49096841F43C
:100D000070410A4A116008E006E00849096841F4A8
:100D10007021064A116000E000BF00BF704700006C
:100D20008000024044000240F8FFFDBF040402407E
:100D30000146486880B2704710B50022026847F645
:100D4000F0739A430C6A8B6823430C6923434C6904
:100D500023438C692343CC6923434C6A23438C6A25
:100D600023431A430260CB6843600B6883604B687F
:100D7000C36010BD70477047704770477047704739
:100D80007047704700B59FB00121084600F034FD60
:100D90000121042000F030FD0121082000F02CFD8D
:100DA0000121102000F028FD0121202000F024FD69
:100DB0000121880300F020FD0121480200F01CFD04
:100DC0000121080300F018FD0121880400F0F4FC63
:100DD0000121022000F0F0FC0121084600F0DCFCBB
:100DE0000121FE4800F060FB0121042000F05CFBC3
:100DF0000B20ADF8780000208DF87B001EA9F84884
:100E000000F0C6FA0320ADF8780000208DF87B00D2
:100E10001EA9F44800F0BCFA49F60400ADF87800C9
:100E200048208DF87B0003208DF87A001EA9ED483C
:100E300000F0AEFA3F20ADF8780048208DF87B0036
:100E400003208DF87A001EA9E74800F0A1FA47F6C2
:100E50001040ADF8780048208DF87B0003208DF815
:100E60007A001EA9DE4800F093FA0420ADF878005D
:100E700048208DF87B0003208DF87A001EA9DB48FE
:100E800000F086FA4FF4E360ADF8780010208DF89A
:100E90007B0003208DF87A001EA9D24800F078FA72
:100EA0000821D04800F043FB1021CE4800F03FFB62
:100EB0004FF44070ADF8780014208DF87B000320CB
:100EC0008DF87A001EA9C84800F062FA4FF230008F
:100ED000ADF8780010208DF87B0003208DF87A00A3
:100EE0001EA9C14800F054FA1021BF4800F01DFBB4
:100EF0002021BD4800F019FB48F2E430ADF878003D
:100F000010208DF87B0003208DF87A001EA9B448CC
:100F100000F03EFAE020ADF8780003208DF87A006A
:100F200018208DF87B001EA9AE4800F031FA002190
:100F3000AF4800F0ACFD0020ADF84C004FF48270DB
:100F4000ADF84E000020ADF85000ADF85200012081
:100F5000ADF854004002ADF856003820ADF8580006
:100F60000020ADF85A000720ADF85C0013A9A04896
:100F700000F0A7FD01219E4800F089FD4020ADF85A
:100F8000780003208DF87A0018208DF87B001EA9C8
:100F9000954800F0FDF98020ADF8780048208DF8E4
:100FA0007B001EA9904800F0F3F94FF416501A90F8
:100FB0000020ADF86C00ADF86E00ADF87000ADF833
:100FC00074000C20ADF872000020ADF86000ADF8A0
:100FD00062004FF40070ADF864000020ADF86600C8
:100FE00018A9844801F038FE1AA9824801F05AFE77
:100FF0000121804801F041FE40217E4801F029FE98
:101000007D48FFF7F3FD7B48001D08907B48099061
:1010100000200A904FF480700B9000200C908020EC
:101020000D9000200E900F90202010900002119043
:101030000020129008A97048FFF77EFE012240218F
:101040006C4801F026FE01216B48FFF7C4FD00202B
:101050006B498870C8706848FFF76AFE6849487035
:101060006548FFF765FE6649087000208880C880E3
:10107000088161481438FFF7B9FD5E48001D0890EB
:101080006048099010200A9000010B9000200C90FD
:1010900080200D9000200E900F9010904FF4005083
:1010A00011900020129008A953481438FFF744FE0D
:1010B000012280214F4801F0ECFD4FF48060ADF833
:1010C000780003208DF87A0018208DF87B001EA987
:1010D000454800F05DF94FF40060ADF87800042059
:1010E0008DF87B001EA9404800F052F94FF41650CD
:1010F0001A900020ADF86C00ADF86E00ADF87000ED
:10110000ADF874000C20ADF872000020ADF860005E
:10111000ADF862004FF40070ADF864000020ADF847
:10112000660018A9384801F097FD1AA9364801F061
:10113000B9FD0121344801F0A0FD4021324801F001
:1011400088FD2D482838FFF751FD2F48001D0890D5
:101150002E48099000200A904FF480700B900020D8
:101160000C9080200D9000200E900F902020109069
:10117000000211900020129008A91F482838FFF79C
:10118000DBFD01224021204801F083FD01211A48A6
:101190002838FFF720FD00201D498870C8701648C8
:1011A0002838FFF7C5FD1A49487013482838FFF75B
:1011B000BFFD1749087000208880C88008810E484C
:1011C0003C38FFF713FD1048001D089011480990A6
:1011D00010200A9000010B9000201DE0000230005A
:1011E0000010014000080140000C014000140140C3
:1011F000003001400038014058000240D442002035
:10120000C8410020D443002000480040BC3F0020DB
:10121000B03E0020BC4000200C9080200D900020AB
:101220000E900F9010904FF40050119000201290EB
:1012300008A95248FFF780FD01228021504801F0A3
:1012400028FD504801F046FB0020ADF80600ADF83F
:1012500002000520ADF8000045F6BF50ADF80400CF
:101260006946484801F0B0FB2021464801F0A2FB46
:101270004FF4404000F084FA4348FFF781FA002021
:10128000039001208DF810008DF81100C004059026
:101290000020069005208DF81C0003A93A48FFF7AE
:1012A000BFFA072301220A213748FFF7E1FA072393
:1012B00002220B213448FFF7DBFA072303220D211A
:1012C0003148FFF7D5FA0723042200212E48FFF703
:1012D000CFFA0723052201212B48FFF7C9FA012184
:1012E0002948FFF741FA01212748FFF732FA26483B
:1012F000FFF71AFB00BF2448FFF787FA0028FAD14E
:101300002148FFF721FB00BF1F48FFF774FA0028B0
:10131000FAD11A481438FFF769FC1B484C30089082
:101320001A48099000200A9040F6C4100B90002043
:101330000C9080200D9040000E9080000F90202097
:101340001090000211900020129008A90B48143848
:10135000FFF7F2FC012109481438FFF73CFC01219A
:101360000948FFF7E6FA01210748FFF739FA01219A
:10137000044801F0A3FA1FB000BD00001C000240A9
:10138000004800400004004000240140520F0020AB
:101390002DE9F0410246002500260020002300240C
:1013A000002791F803C00CF00F0591F803C00CF072
:1013B000100CBCF1000F03D091F802C04CEA0505F7
:1013C00091F800C0BCF1000F31D0146800202BE070
:1013D0004FF0010C0CFA00F3B1F800C00CEA030660
:1013E0009E4220D183004FF00F0C0CFA03F7BC4350
:1013F00005FA03FC4CEA040491F803C0BCF1280F81
:1014000006D14FF0010C0CFA00FCC2F814C00AE03F
:1014100091F803C0BCF1480F05D14FF0010C0CFA54
:1014200000FCC2F810C0401C0828D1D31460B1F8E9
:1014300000C0BCF1FF0F34DD546800202EE000F145
:10144000080C4FF0010808FA0CF3B1F800C00CEAE0
:1014500003069E4221D183004FF00F0C0CFA03F7D4
:10146000BC4305FA03FC4CEA040491F803C0BCF148
:10147000280F05D100F1080C08FA0CF8C2F8148006
:1014800091F803C0BCF1480F07D100F1080C4FF0F0
:10149000010808FA0CF8C2F81080401C0828CED3C6
:1014A0005460BDE8F0810000F0B50A460023002436
:1014B00000210025174E7168C0F3034583B200F484
:1014C0004016B6F5401F08D121F07061114E7668C4
:1014D00026F070660F4F7E6012E000F48016B6F5BD
:1014E000801F06D1032606FA05F4A14341F070617E
:1014F00006E0460D360103FA06F6B14341F070618D
:1015000022B1460D360103FA06F63143014E7160F1
:10151000F0BD0000000001400246002093680B402F
:101520000BB1012000E0002070474161704701616C
:1015300070477047704770477047000000200349AC
:10154000886781F87C00C86670470000FC3D002079
:10155000F0B589B007460C46642097FBF0F086B2E0
:10156000C72E00DDC72606F1320086B24FF6FF70A7
:1015700000EA461601AA2021304603F093FA00251E
:1015800029466D1C01A8405C208020884FF6FF7121
:1015900001EA00202080228829466D1C01A8405CB9
:1015A0001044208029466D1C01A8405C6080608842
:1015B0004FF6FF7101EA00206080628829466D1CA9
:1015C00001A8405C1044608029466D1C01A8405C65
:1015D000606060680002606029466D1C01A8405C84
:1015E00062681044606060680002606029466D1C9B
:1015F00001A8405C6268104460606068000260603E
:1016000029466D1C01A8405C62681044606009B006
:10161000F0BD00000FB41CB5002416480068002877
:1016200014D101201349086000F0B8F9022000230A
:101630001A4619460090184600F076F90EA10020CF
:1016400000F016FA16A1002000F012FA05A8019089
:101650004FF480711C48019B049A01F053FC04462E
:101660001949002000F004FA0020019020461CBC1B
:101670005DF814FBC80100205345474745522052EE
:1016800065616C2D54696D652D5465726D696E616F
:101690006C2053616D706C650D0A0D0A000000002E
:1016A0002323232323232054657374696E672053F7
:1016B00045474745525F7072696E7466282920233A
:1016C00023232323230D0A000C45002008B54FF4E3
:1016D000C06000F049F809208DF8000001208DF865
:1016E000010003208DF8020001208DF803006846F8
:1016F00000F002F808BD000070B5002100230F22A1
:10170000C47804B3154C246804F4E064C4F5E064C0
:10171000210AC1F10403CA40447804FA03F1847831
:101720001440214309010E4C0678A155047804F0B9
:101730001F050124AC4005786D11AD0005F1E025D1
:10174000C5F8004109E0047804F01F050124AC400D
:10175000044D0678761145F8264070BD0CED00E08A
:1017600000E400E080E100E002490143024A116028
:10177000704700000000FA050CED00E07047000023
:1017800001460020034A506820F44040084350605E
:10179000704700000010024029B1064A5269024316
:1017A000044B5A6104E0034A52698243014B5A6177
:1017B000704700000010024029B1064AD269024376
:1017C000044BDA6104E0034AD2698243014BDA61D7
:1017D000704700000010024029B1064A1269024316
:1017E000044B1A6104E0034A12698243014B1A61F7
:1017F000704700000010024029B1064A9269024376
:10180000044B9A6104E0034A92698243014B9A6156
:10181000704700000010024029B1064AD268024316
:10182000044BDA6004E0034AD2688243014BDA6079
:10183000704700000010024010B501F00FF8024898
:1018400000F004F810BD0000F844002030B500217D
:101850000022002400232D4D6D6805F00C0121B1FC
:10186000042905D0082923D105E0294D056022E08F
:10187000274D05601FE0254D6D6805F470120225A7
:1018800005EB9242214D6D6805F480341CB9214D61
:10189000554305600BE01D4D6D6805F400351DB125
:1018A0001C4D5543056002E0194D5543056002E0AB
:1018B000174D056000BF00BF144D6D6805F0F001C5
:1018C0000909154D6B5C0568DD4045600F4D6D687D
:1018D00005F4E061090A104D6B5C4568DD408560E8
:1018E0000A4D6D6805F46051C90A0B4D6B5C456883
:1018F000DD40C560054D6D6805F44041890B074D1D
:101900006B5CC568B5FBF3F5056130BD00100240A6
:1019100000127A0000093D00B4010020C40100203B
:1019200070477047704700002DE9F05F05460F468D
:1019300090469946DFF860B000BF9BF8000008B9F8
:1019400001F032FA00BFDFF850A0032D1FD2EFF3F1
:1019500011810846202181F3118800BF00BF05EBEB
:1019600045020AF1180101EBC2043DB12760C4F839
:101970000480C4F8089000212161E1600A99616146
:10198000C1B281F3118800BF00BF002601E04FF013
:10199000FF363046BDE8F09F0C46002010B501F040
:1019A00003FA10BD2DE9F04104460D4616460E4FD0
:1019B00000BF387808B901F0F7F900BFEFF31180E4
:1019C0000746202080F3118800BF00BF3246294619
:1019D000204600F00BF88046F8B280F3118800BF73
:1019E00000BF4046BDE8F0810C4600202DE9F047DD
:1019F000074688461646C24607EB47011B4800EBE0
:101A0000C109D9F8140020B1012811D0022826D12B
:101A10001EE0484601F000FA0546B54201D2002416
:101A200005E0344632465146484601F03EFA18E099
:101A3000484601F0F1F90546B54201D2284600E0DA
:101A40003046044622465146484601F02EFA08E048
:101A500032465146484601F0EDF9044601E00024C3
:101A600000BF00BF2046BDE8F087000024460020EC
:101A700070B505460C462046FEF790FB06463246FA
:101A800021462846FFF78EFF70BD7047704721B191
:101A9000028842F04002028004E002884FF6BF73E1
:101AA0001A40028070470246002013890B400BB198
:101AB000012000E00020704701468889704781813D
:101AC000704710B50022028802F441520B884C88FE
:101AD00023438C882343CC8823430C8923434C899C
:101AE00023438C892343CC8923431A430280838B6D
:101AF0004FF2FF74234083830B8A038210BD70B5BD
:101B000088B004466088642190FBF1F086B2C72E4D
:101B100000DDC72606F1320086B24FF6FF7000EAFC
:101B2000461600252088021229466D1C0DF801205A
:101B3000227829466D1C0DF8012060880212294682
:101B40006D1C0DF80120A27829466D1C0DF80120AE
:101B50006068020E29466D1C0DF801206068C0F314
:101B6000074229466D1C0DF80120A088C0F307220A
:101B700029466D1C0DF80120227929466D1C0DF8AF
:101B8000012055208DF81F006A462021304602F0C2
:101B9000CDFF08B070BD10B500F002F810BD000018
:101BA0000CB50020019000903448006840F480306B
:101BB0003249086000BF3148006800F400300090EE
:101BC0000198401C0190009818B90198B0F5A06FD9
:101BD000F1D12A48006800F4003010B101200090D3
:101BE00001E0002000900098012844D124480068BA
:101BF00040F01000224908600846006820F0030009
:101C000008600846006840F0020008601B48406811
:101C10001A4948600846406848600846406840F4F1
:101C2000806048600846406820F47C1048600846A0
:101C3000406840F4E81048600846006840F0807052
:101C4000086000BF0D48006800F000700028F9D05F
:101C50000A48406820F00300084948600846406888
:101C600040F00200486000BF0448406800F00C00EB
:101C70000828F9D101E000BFFEE70CBD00100240CA
:101C8000002002402DE9F047FE48006820B1FD48E1
:101C90000068401EFB490860FB48006820B1FA4814
:101CA0000068401EF8490860F848D0F8D80B30B1F9
:101CB000F648D0F8D80B401EF449C1F8D80BF448C8
:101CC000B0F8F20038B1F248B0F8F200401E81B22C
:101CD000EF48A0F8F21000244FF48061ED48FFF7C0
:101CE0001BFC08B144F080044FF40041EA48FFF7C0
:101CF00013FC08B144F040044FF48051E648FFF76C
:101D00000BFC08B144F020044FF40061E248FFF7F7
:101D100003FC08B144F010044FF48051DD48FFF794
:101D2000FBFB08B144F008044FF40061D948FFF709
:101D3000F3FB08B144F004040821D848FFF7ECFB9A
:101D400008B144F002040421D548FFF7E5FB08B1CF
:101D500044F00104E4B2D3480470D348045DD3488E
:101D60000078844208D1D248007868B10020D04978
:101D70000870D0490C7007E0CC490C70FF20CD49A9
:101D800008700120CA490870CB48008838B3CB4896
:101D90000088CB490988884209DAC8480088401C75
:101DA000C64908808021BB48FFF7C1FB17E0C34844
:101DB0000088C4490988884209DAC0480088401C64
:101DC000BE4908808021B348FFF7AFFB07E0002041
:101DD000BA490880B8480088401EB7490880BA4808
:101DE0000078642805DA4FF48051AC48FFF79FFB78
:101DF00004E04FF48051A948FFF797FBB34890F8EF
:101E00004800C72807DAB14890F84800401CAF499D
:101E100081F848000AE00020AC4981F84800012020
:101E200081F849000846C06C401CC864A848D0F836
:101E3000A000012810D104219648FFF776FB4FF44B
:101E400000419448FFF771FB0120A149C1F8B0009F
:101E50000020C1F8AC00BDE09D48D0F8A0004FF6CE
:101E6000FF7188420FD104218A48FFF760FB4FF4CD
:101E700000418848FFF75BFB01209549C1F8B0009D
:101E8000C1F8AC00A6E09248D0F8A00088BB90480A
:101E9000D0F89000B0F5FF7F07D88D48D0F89000BB
:101EA000401C8B49C1F8900094E000208849C1F89B
:101EB00090000120C1F894000846006F486708466A
:101EC000406FD1F89010B0EB510F13D38048406FA2
:101ED00080B104216F48FFF72AFB4FF400416D48A1
:101EE000FFF725FB01207A49C1F8B000C1F8AC002A
:101EF00070E010E004216748FFF717FB4FF4004142
:101F00006448FFF712FB01207149C1F8B0000020BE
:101F1000C1F8AC005EE06E48D0F8A000012849D9B5
:101F20006B48D0F8A000672844D26948D0F89800E0
:101F3000B0F5C77F07D86648D0F89800401C6449C0
:101F4000C1F8980006E000206149C1F8980001201E
:101F5000C1F89C005E48B0F8A00084B2A01E84B214
:101F60004FF6FF7000EA84045948D0F89800A04268
:101F70000FD204214748FFF7DAFA4FF400414548F1
:101F8000FFF7D5FA01205249C1F8B000C1F8AC0002
:101F900020E004213F48FFF7C8FA4FF400413D48D4
:101FA000FFF7C3FA01204A49C1F8B0000020C1F888
:101FB000AC000FE004213748FFF7B7FA4FF40041B7
:101FC0003448FFF7B2FA01204149C1F8B0000020BF
:101FD000C1F8AC003E48D0F8AC0078B12B48B0F85E
:101FE000FE002B49FE3131F81000401C81B2274819
:101FF000B0F8FE00264AFE3222F81010354800786C
:10200000802876D010212348FFF786FAC0BB012034
:10201000314908703148806C3049C8640846406CCA
:1020200088640846006C48640846C06B086408462B
:10203000806BC8630846406B88630846006B486342
:102040000846C06A08630846806AC8620846406A53
:1020500088620846006A48620846C0690862084605
:102060008069C8610846406988610846006948611E
:102070000846C068086108468068C86008462FE0C6
:1020800037E0000070010020840100201C32002095
:102090001C2200200010014000080140000C0140FB
:1020A0000014014017000020DE6501081500002023
:1020B0001600002014000020060000200C00002064
:1020C000080000200A000020050000201C0200205B
:1020D000FC3D00202C00002024000020CC0100202A
:1020E0004068886008460068486001F03DFCF74998
:1020F0000860F7480078C72805DAF5480078401CE2
:10210000F3490870B4E20020F14908700120F14958
:102110000870F148006D20B1EF48006D401EEE4997
:1021200008650120EC4981F865000021EB48C0F802
:10213000C010C0F8C410C0F8C810C0F8CC10C0F867
:10214000D010894641E0E548D0F8C0204846411CFF
:102150001FFA81F9E24931F810001118DF48C0F880
:10216000C010D0F8C4204846411C1FFA81F9DC4950
:1021700031F810001118D948C0F8C410D0F8C820A0
:102180004846411C1FFA81F9D54931F81000111851
:10219000D248C0F8C810D0F8CC204846411C1FFADD
:1021A00081F9CF4931F810001118CC48C0F8CC1093
:1021B000D0F8D0204846411C1FFA81F9C84931F8AF
:1021C00010001118C548C0F8D01040F6C410814561
:1021D000B9DBC248D0F8C000C249884213D2BF4818
:1021E000D0F8C00040F6C4114843BC49C1F8C00053
:1021F0000846D0F8C010D0F8C800B1FBF0F1B748DD
:10220000C0F8C01018E0B548D0F8C00040F2E24174
:102210004843B249C1F8C0000846D0F8C800410898
:10222000AE48C0F8C810D0F8C010D0F8C800B1FB54
:10223000F0F1AA48C0F8C010A848D0F8C400A949D5
:10224000884213D2A548D0F8C40040F6C4114843D0
:10225000A249C1F8C4000846D0F8C410D0F8C8009C
:10226000B1FBF0F19D48C0F8C41018E09B48D0F8CD
:10227000C40040F2E24148439849C1F8C40008460E
:10228000D0F8C80041089548C0F8C810D0F8C4106C
:10229000D0F8C800B1FBF0F19048C0F8C4108F48E6
:1022A000D0F8CC008F49884213D28C48D0F8CC00AB
:1022B00040F6C41148438949C1F8CC000846D0F81B
:1022C000CC10D0F8C800B1FBF0F18448C0F8CC10B5
:1022D00018E08248D0F8CC0040F2E24148437F4900
:1022E000C1F8CC000846D0F8C80041087B48C0F8C7
:1022F000C810D0F8CC10D0F8C800B1FBF0F1774886
:10230000C0F8CC107548D0F8D0007649884213D276
:102310007248D0F8D00040F6C41148436F49C1F864
:10232000D0000846D0F8D010D0F8C800B1FBF0F1CA
:102330006A48C0F8D01018E06848D0F8D00040F2E1
:10234000E24148436549C1F8D0000846D0F8C800CA
:1023500041086248C0F8C810D0F8D010D0F8C800C2
:10236000B1FBF0F15D48C0F8D0105C48D0F8C480F3
:1023700090F8DC00642805DB584890F8DC006438ED
:10238000804410E0554890F8DC00C0F164004045FE
:1023900007D8524890F8DC00C0F16400A8EB0008B0
:1023A00001E04FF00008B8F5FA7F0BD3A8F5FA78F2
:1023B0000A20B8FBF0F84C4830F818104748C0F82D
:1023C000E81010E0C8F5FA780A20B8FBF0F84648A3
:1023D00030F818104148C0F8E810D0F8E800414241
:1023E0003E48C0F8E8100025A94607E0374850F8F5
:1023F0002900054409F101001FFA80F9B9F1140F11
:10240000F4DB1420B5FBF0F53448C0F8F850374839
:10241000854206D93448B0F8281A3048C0F8E01090
:1024200023E02E48D0F8D800A8420CD82B48D0F88A
:10243000D8002D1A05EB4500C0EBC510810B2748CD
:10244000C0F8E01011E02548D0F8D800451B05EB96
:102450004500C0EBC510810B2048C0F8E010D0F853
:10246000E00041421D48C0F8E0101C48D0F8E010E0
:10247000D0F8E80001441948C0F8EC10D0F8EC009E
:10248000002806DB1548D0F8EC50002180F8DE105B
:1024900007E01248D0F8EC00454201210F4880F8CF
:1024A000DE10002600270C48008E0F4931F810007E
:1024B000A84224D80848068E1CE00B4830F81600C5
:1024C000A84215D30EB1701E87B217E0CC010020D0
:1024D00005000020040000201C0200201C22002017
:1024E000520F0020E2361A00343300200EADE10016
:1024F000701C86B240F25A508642DEDB0FE0CD48B7
:10250000078E09E0CC4830F81700A84202D8781CA2
:1025100086B203E0781E87B2002FF3DC00BFBE4214
:1025200001D1701C86B2C44830F81600C24931F897
:102530001710401AC04931F81710691A01EB8101D0
:102540004900B1FBF0F084B2BA48008EB84204D121
:10255000082C12DBB74806860FE0B648008EB04262
:1025600004D1022C09DCB348078606E0052C02DC06
:10257000B048078601E0AF480686AE48008EAD49F8
:1025800048860846018E00F21A2030F81100A94949
:1025900008860846018D4185C18C0185818CC184E6
:1025A000008EA44988848A8CC98C501800EBD071A5
:1025B000C1F34F019F4AD1831046008E00EB80008B
:1025C00004EB4000114688860846418F8187018FC1
:1025D0004187C18E0187808E1146C886CA8E098FB9
:1025E000501800EBD0714910944AC2F880109448FA
:1025F00090F8DE0088B98F48C08B01B29148B0F8DE
:10260000FE20B0F8FE00401C83B28E48A0F8FE30D9
:10261000A0F2027020F8121011E08648C08B4042F0
:1026200001B28848B0F8FE20B0F8FE00401C83B22A
:102630008448A0F8FE30A0F2027020F81210814801
:10264000B0F8FE00C0F309017E48A0F8FE10D0F8F3
:102650000001401C7B49C1F8000101217948C0F804
:1026600004110021B0F8FE00754AFE3222F8101065
:102670007548FEF75DFB754948700846C07840B95B
:1026800008464078097888425DD001206F49C870BB
:1026900059E06E48C078012809D16C4840786B49F0
:1026A000097888424FD102206849C8704BE06748DA
:1026B000C078022847D16548407864490978884243
:1026C0003ED10120614988700320C8700846C08847
:1026D000888008464078C0F58070C88008468088A9
:1026E000C988884207DA5948C08858498988401AF9
:1026F0005649088108E05548C08800F58070534964
:102700008988401A514908814FF0000A13E04F4967
:10271000898801EB0A00C11700EB11610912A0EBD7
:1027200001224B498A5CA1F5807101F80A200AF167
:10273000010000F0FF0A454800895045E7DC02E04F
:1027400001204249C87041484078404908703E48DD
:102750002838FEF7EDFA3F4948700846C07840B97E
:1027600008464078097888425DD001203949C87010
:1027700059E03848C078012809D1364840783549B1
:10278000097888424FD102203249C8704BE0314865
:10279000C078022847D12F4840782E4909788842CE
:1027A0003ED101202B4988700320C8700846C0889C
:1027B000888008464078C0F58070C88008468088C8
:1027C000C988884207DA2348C08822498988401A84
:1027D0002049088108E01F48C08800F580701D4925
:1027E0008988401A1B4908814FF0000A13E01949F3
:1027F000898801EB0A00C11700EB11610912A0EBF7
:10280000012215498A5CA1F5807101F80A200AF1BC
:10281000010000F0FF0A0F4800895045E7DC02E0A4
:1028200001200C49C8700B4840780A490870BDE87F
:10283000F08700001C02002034330020FC3D002003
:102840001C2200201C32002058000240C8410020F9
:10285000D4420020B03E0020BC3F002010B51048FC
:10286000006840F001000E490860084640680D49C4
:1028700008400B494860084600680B490840084971
:1028800008600846006820F4802008600846406818
:1028900020F4FE00486000208860FFF77CF910BD3E
:1028A000001002400000FFF8FFFFF6FE704770477F
:1028B00070477047704770477047704721B1028872
:1028C00042F00102028004E0028840F2FE331A4026
:1028D0000280704710B504463449601A8C4245D0D6
:1028E0000CDCB4F1804F1DD03148204418B3B0F552
:1028F000806F29D0B0F5006F54D12EE0B0F5806F15
:102900003DD0B0F58E3F03D0B0F5923F4AD13FE0C5
:102910000121C802FEF780FF00214FF40060FEF79E
:102920007BFF40E001210846FEF756FF0021012011
:10293000FEF752FF37E001210220FEF74DFF002194
:102940000220FEF749FF2EE001210420FEF744FF9C
:1029500000210420FEF740FF25E001210820FEF7BA
:102960003BFF00210820FEF737FF1CE0012110206B
:10297000FEF732FF00211020FEF72EFF13E00121A9
:102980002020FEF729FF00212020FEF725FF0AE086
:1029900001214803FEF740FF00214FF40050FEF7ED
:1029A0003BFF00E000BF00BF10BD00000010004072
:1029B00000FCFFBF82884FF68F731A4082808288A6
:1029C0000A43828070470000028802F08F02028072
:1029D000CA884B881A4303881A4302808A888285F2
:1029E0000A880285054A904202D0054A904201D1E8
:1029F0000A7A02860122828270470000002C014080
:102A0000003401403EB58848D0F8800043F2D4013C
:102A1000884204D900208449086748663EBD0824DE
:102A20000AE0601E8049103151F820107E481030B5
:102A300040F82410601EC4B2002CF2DC7A484068D2
:102A40007949D1F88010401A7749086109240AE0D1
:102A5000601E7549343151F820107348343040F805
:102A60002410601EC4B2002CF2DC6F48016940697A
:102A7000081A6D4948630846416B806B01446A48F7
:102A8000C06B01446848006C01446748406C0844CE
:102A90006549C86508460078002863D00846006983
:102AA0008968884248DA604800695F49496B484351
:102AB000002805DC5C48006910BB5B48406BF8B13E
:102AC0005948006E5849096908445749086608463C
:102AD000006E10F5967F01DA544808665248006E81
:102AE00000EB800040000F2190FBF1F0C0EB0010E4
:102AF0004D490969C1EB011108444B49C8661EE004
:102B0000494800694849496B4843002802DB464868
:102B1000406B60B94448006E00EB800040000F211C
:102B200090FBF1F0C0EB00103F49C86607E03E485B
:102B3000406E3D49C86602E0FF203B49C8663A48FE
:102B4000C06E002802DA00203749C8663648C06ED9
:102B5000FF2802DDFF203449C8663348C06E324981
:102B6000486602E000203049C8662F48C06E2E49F2
:102B7000096E2D4AD26DCDE9002102902A48436B9F
:102B8000026981682AA0FEF745FD2748C06E2649E4
:102B900008670846406EC96E88423FD12248C06E21
:102BA000FF283BD02048C06EB8B31F48D0F888102B
:102BB000D0F88800401C1C4AC2F888001046D0F8A3
:102BC0008C0081422ED91046D0F8880040F2FF7167
:102BD000884227D21046B0F888001B49088010466A
:102BE000D0F884006421B0FBF1F000EBC00101EBF0
:102BF00000104FF6FF7101EA80001349488010462B
:102C0000006E48600846FEF77AFF0748D0F8880053
:102C1000401D0549C1F88C0004E0FFE7002002498F
:102C2000C1F8880000BFF9E6FC3D0020D4FEFFFF9C
:102C3000256C642C256C642C256C642C256C642C10
:102C4000256C642C25640A00A80100207047704799
:102C50007047CA430280704710B502460020108AB0
:102C60004FF2FF0318400B884C8823438C88234382
:102C7000CC8823431843108210BD21B1828942F4CD
:102C80000052828104E082894DF6FF731A408281EE
:102C900070471AB1838A0B43838202E0838A8B4395
:102CA000838270472DE9F04786B005460E46002422
:102CB000A24600BF00BF00272F462C8A4CF6FF70AB
:102CC0000440F08804432C82AC894EF6F310044093
:102CD000B08831890843718908430443AC81AC8AC8
:102CE0004FF6FF400440B0890443AC8201A8FEF7D0
:102CF000ADFD1248874202D1DDF810A001E0DDF8F9
:102D00000CA00AEBCA0000EB0A1031688900B0FB86
:102D1000F1F86420B8FBF0F004012009642101FB04
:102D20001089322000EB0910B0FBF1F000F00F0029
:102D300004432C8106B0BDE8F08700000038014054
:102D400070470000002002498870C87008817047F1
:102D5000C841002010B5044600210548FDF73BFF9F
:102D600003484438846401210148FDF734FF10BD55
:102D700044000240002002498870C87008817047F2
:102D8000B03E002010B5044600210548FDF723FFA2
:102D900003481C38046201210148FDF71CFF10BDE7
:102DA0001C0002407047000010B5124C0320206147
:102DB000606111A0A0611349E1614FF4806121625B
:102DC0000021A1626162E1620BA020660E4961668A
:102DD0001021A16600212167E16661670BA1E01D5A
:102DE000FDF7E3F90AA12046FDF7DFF92020A071E5
:102DF00010BD00000C4600205465726D696E616C58
:102E000000000000B4460020B44A00205254540090
:102E1000534547474552000010B501460A69CB6843
:102E20009A4204D88C68641EE41AA01801E0D41AEF
:102E3000601E10BD2DE9F05F0446894617464FF02D
:102E4000000AE56800BFD4F81080A84503D9A8EBB4
:102E50000500461E04E0A5EB0800401CA1680E1A00
:102E6000A068401BB04201D9304601E0A068401B79
:102E70000646BE4201D2304600E03846064660684B
:102E800000EB050B324649465846FDF775F9B2444A
:102E9000B144BF1B3544A068A84200D10025E560BD
:102EA000002FD0D15046BDE8F09F2DE9F0470446F1
:102EB00089461546E668A068871BAF420AD9606854
:102EC00000EB060A2A4649465046FDF755F97019A7
:102ED000E06014E0B846606800EB060A42464946E6
:102EE0005046FDF749F9A5EB0708D4F804A009EB13
:102EF000070142465046FDF73FF9C4F80C80BDE893
:102F0000F08700007CB50C001D461646014601D036
:102F1000601E00E00020CDE90010064B6A462946FD
:102F2000304600F0DBF8002C02D0009A002111702E
:102F30007CBD0000E337000802E008C8121F08C18A
:102F4000002AFAD170477047002001E001C1121F2A
:102F5000002AFBD1704700002DE9FF5F82B00021FD
:102F6000DDE90430020DDDF840B0034318D044F62B
:102F70001050A2F2FF3242431514119801281FD0BD
:102F8000A5EB0B00401C5FEA000A4FF000064E4F15
:102F9000DFF83891B046504615D5CAF1000413E069
:102FA000119801244AA3012801D16FEA0B0102986C
:102FB000119AC0E90031C0E9024206B0BDE8F09FB5
:102FC000CBF10000DFE704460021404A491842EBFC
:102FD0000450CDE9001012E0E00707D032463B462E
:102FE00040464946FDF7D8F98046894632463B4679
:102FF00010461946FDF7D0F906460F466410002C1E
:10300000EAD1DDE90401DDE90023BAF1000F06DAB7
:10301000FDF7C2F942464B46FDF7BEF905E0FDF764
:103020002DFA42464B46FDF729FA04460E46002289
:10303000284BFDF7ABFA03D84FF0FF30014607E00D
:103040000022254B20463146FDF7FFF8FDF785FAB3
:10305000102409E0002C0ADB0A220023FDF7C4F843
:10306000039B30321A55641E50EA0102F2D1641CEF
:10307000039AC4F111031444119A012A03D00122C6
:1030800008430DD10AE0084304D000204FF0110B93
:10309000119072E7A3EB0B056D1E0DE05B4504DD9F
:1030A0004FF0000205F1010504E003DA4FF00002E1
:1030B000A5F10105002AECD002981199C0E902316E
:1030C000C0E9004579E70000000014400000F03F2F
:1030D000300000000000F0430000E03F2DE9FF4F0A
:1030E00095B09A46884606460025EEE1252877D118
:1030F00000242746F94A0121039400E0044316F80E
:10310000013F203B01FA03F01042F7D130782A2822
:1031100011D06FF02F033078A0F13002092A16D8B1
:10312000039A44F0020402EB820203EB42021044D1
:10313000761C0390EFE758F8042B0392002A03DA79
:10314000504244F40054039044F00204761C30785A
:103150002E2816D116F8010F44F004042A280DD0A9
:103160006FF02F023078A0F13003092B09D807EB5C
:10317000870302EB4303C718761CF3E758F8047B78
:10318000761C30786C280FD006DC4C2817D06828C5
:103190000DD06A2814D104E0742810D07A280FD1F9
:1031A0000DE044F400140AE044F4801401E044F417
:1031B00040147278824202D104F58014761C761C89
:1031C000307866280BD013DC582877D009DC00282B
:1031D00075D04528F6D04628F4D047281AD193E177
:1031E00018E0632835D0642879D0652812D18BE1A6
:1031F000702873D008DC6728F1D069286FD06E285A
:103200000DD06F2806D1ACE073282CD0752874D06F
:10321000782853D05246179990476D1C54E1C4F357
:103220000250022809D003280DD0D8F80010042835
:103230000DD00D6008F1040846E1D8F80010EA1737
:10324000C1E90052F6E7D8F800100D80F2E70D70E2
:10325000F0E718F8041B8DF8001000208DF801002D
:10326000EB46012003E058F804BB4FF0FF30610744
:103270004FF0000102D40DE009F101018946B94285
:103280000FDA8145F8DB1BF809100029F4D108E0BA
:1032900009F1010189468142FADB1BF80910002976
:1032A000F6D103985346A0EB090721463846179AF2
:1032B00000F080FA284400EB090507E044E008E14B
:1032C0000DE01BF8010B524617999047B9F101091F
:1032D000F7D2534621463846179AF2E039E00A21E0
:1032E000C4F302524FF0000B0091022A06D058F8A6
:1032F000040BC117032A09D00AE023E008F10700F4
:1033000020F00702F2E80201904605E000B2C11782
:10331000042A01D140B2C117002906DA0A46002169
:10332000404261EB02012D2202E0220504D52B224E
:103330008DF80420012203E0E20701D02022F7E704
:10334000914657E00A2100E010214FF0000B009158
:103350000BE010214FF0000B44F00404082700910B
:1033600003E008204FF0000B0090C4F30252022A41
:1033700005D058F8040B0021032A08D008E008F112
:10338000070020F00702F2E80201904603E080B255
:10339000042A00D1C0B24FF0000922072AD53278A2
:1033A000702A07D0DDF800C08CF0100C5CEA0B0C22
:1033B00005D00EE040228DF80420012208E050EAFA
:1033C000010306D030238DF804308DF80520022249
:1033D0009146009B83F0080353EA0B030AD150EA9D
:1033E000010201D1620705D530228DF804204FF08B
:1033F00001097F1E3278582A04D039A20C920CAAF7
:1034000002920BE03BA2F9E75B46009AFCF7ECFE68
:103410000C9B9B5C029A521E0292137050EA0102AE
:10342000F2D1029804A9081A00F1200B600702D516
:1034300024F4803400E001275F4502DDA7EB0B0098
:1034400000E0002000EB0B01009003984944401A73
:103450000390E00306D453462146179A039800F0E0
:10346000A9F90544002706E001A85246C05D179956
:1034700090476D1C7F1C4F45F6DBE0030CD553468F
:103480002146179A039800F095F9054404E030208E
:103490005246179990476D1C0099481E00900029CC
:1034A000F5DC08E00298029952460078491C029126
:1034B000179990476D1CBBF10001ABF1010BF1DCDA
:1034C0005BE100F065F90544761C307800287FF454
:1034D0000DAE19B02846BDE8F08F000009280100A4
:1034E000303132333435363738396162636465667A
:1034F000000000003031323334353637383941423C
:103500004344454600000000600700D4062708F148
:10351000070020F00700F0E80223804603F0004C8B
:103520005FEA0C0001D097A009E0200501D596A024
:1035300005E0E00701D095A001E0AFF24C00139048
:10354000307823F0004365280CD006DC452809D0EC
:1035500046281DD047287FD13BE0662818D0672831
:103560007AD136E00021112F01DB112000E0781C18
:10357000CDE9000104A90CA8FFF7EEFCDDE90D017F
:103580000C9A4FF0000B07F10109109200914EE0E8
:103590004FF000400097CDE9011004A90CA8FFF7F7
:1035A000DBFCDDE90D020C9B0F994FF0000B9146FF
:1035B0001093009211B9791C00EB0109B7EB0900D7
:1035C00003D4C0F1FF3B07F10109A9EB070001900B
:1035D00042E0012F00DA01270021112F01DD112027
:1035E00000E03846CDE9000104A90CA8FFF7B4FCBF
:1035F000DDE90D010C9A00914FF0000BB9461092D5
:1036000021070FD4009A4A4503DA914601E0A9F157
:103610000109B9F1010F05DD109AA9F10101515C11
:103620003029F4D0B84202DA10F1040F03DA012194
:10363000CDE9011010E0002803DC8344A9EB000170
:1036400002E0411C494500DD8946A0EB0B00401C0F
:1036500001904FF000400290200705D401984845A2
:1036600002DB4FF0FF30019000208DF84B000298F4
:103670000DF14B07B0F1004F25D002200C902B200C
:103680000D90029800280CDA404202902D200D90F7
:1036900007E00A210298FCF791FD3031029007F80B
:1036A000011D0C99481E0C900029F2DC029800289C
:1036B000EFD1791E0D980870307800F0200040F0AE
:1036C000450007F8020D11A8C01BC01D02901398F9
:1036D000007800B1012000EB0901019801EBE071D5
:1036E000029801440398401A401E0390E00306D458
:1036F00053462146179A039800F05CF80544139846
:10370000007818B15246179990476D1CE00323D5F5
:1037100053462146179A039800F04CF805441BE0E5
:10372000BBF1000F07DB0098584504DD109817998E
:1037300010F80B0001E0179930205246904701988D
:103740000BF1010B401E05F10105019004D12E2063
:103750005246179990476D1CB9F10001A9F1010972
:10376000DEDC05E017F8010B5246179990476D1CF7
:103770000299481E02900029F4DC53462146179A0C
:1037800003989EE62D0000002B00000020000000A2
:103790002DE9F041044600251E461746880404D44E
:1037A00005E039462020B0476D1C641EF9D5284637
:1037B000BDE8F0812DE9F041044600251E46904603
:1037C000C80301D5302700E02027880404D505E090
:1037D00041463846B0476D1C641EF9D52846BDE801
:1037E000F0814A68002A06D00A68531C0B601070EA
:1037F0004868401E4860704710B5002400E0641C13
:1038000048488442FBD310214748FDF790FE102121
:103810004548FDF78AFE10214348FDF786FE10213A
:103820004148FDF782FE062000F082F8002400E007
:10383000641C3C488442FBD310213B48FDF775FED5
:1038400010213948FDF771FE10213748FDF76DFE54
:1038500010213548FDF76BFE002400E0641C33485E
:103860008442FBD310213048FDF761FE10212E4821
:10387000FDF75BFE10212C48FDF757FE10212A486A
:10388000FDF753FE432000F053F85A2000F050F8A3
:10389000002000F04DF8202000F04AF8002000F051
:1038A00047F810212048FDF740FE10211E48FDF783
:1038B0003CFE10211C48FDF738FE10211A48FDF788
:1038C00036FE002400E0641C18488442FBD310211B
:1038D0001548FDF72CFE10211348FDF726FE102198
:1038E0001148FDF722FE10210F48FDF71EFE44206F
:1038F00000F01EF8042000F01BF8082000F018F873
:1039000010210948FDF711FE10210748FDF70DFEB3
:1039100010210548FDF709FE10210348FDF707FEB9
:1039200010BD000080EE360000080140407E05001A
:1039300010B5044600BF02210A48FEF7B4F800287B
:10394000F9D021460748FEF7BAF800BF0121054823
:10395000FEF7A9F80028F9D00248FEF7ADF8C0B28A
:1039600010BD00000030014010B500241021204897
:10397000FDF7DDFD10211E48FDF7D7FD10211C4885
:10398000FDF7D3FD10211A48FDF7CFFD1020FFF7FA
:10399000CFFFFF20FFF7CCFF04442402FF20FFF7F6
:1039A000C7FF04442402FF20FFF7C2FF044424F0B1
:1039B0007F44B4F5000F02D204F5000405E0641E54
:1039C000E44324F07F44C4F5000410210848FDF7C7
:1039D000ACFD10210648FDF7A8FD10210448FDF7B5
:1039E000A4FD10210248FDF7A2FD204610BD0000F5
:1039F0000008014070B598B000244FF6FF7000EA4F
:103A0000441410AA2021204601F04CF8002405E0BF
:103A100010A8005D0DF80400601C84B2202CF7DBB8
:103A20000024641C4FF6FF7000EA441410AA202101
:103A3000204601F037F8002407E010A8015D04F1EA
:103A400020000DF80010601C84B2202CF5DB9DF8DE
:103A50003F0055287DD100250024A2E02846691C9E
:103A60008DB21DF8001004EB4402FE4820F822102D
:103A700004EB440130F821004FF6FF7101EA002108
:103A800004EB4402F74820F8221004EB440130F81C
:103A900021202846691C8DB21DF80000104481B217
:103AA00004EB4402EF4820F822102846691C8DB22E
:103AB0001DF8001004EB4402EA4800EB820041804C
:103AC00004EB4401E74800EB810040884FF6FF71AA
:103AD00001EA002104EB4402E24800EB820041804D
:103AE00004EB4401DF4800EB810042882846691C52
:103AF0008DB21DF80000104481B204EB4402D94895
:103B000000EB820041802846691C8DB21DF80060E0
:103B10004FF6FF7000EA06262846691C8DB21DF894
:103B20000000304486B24FF47A7096FBF0F081B218
:103B300004EB4402CB4800EB820081804FF47A70A2
:103B400096FBF0F100FB116081B204EB4402C54822
:103B500000E02AE000EB8200C18004EB4401C14890
:103B600000EB8100C088642190FBF1F081B204EB8E
:103B70004402BC4800EB8200018104EB4401B948D7
:103B800000EB8100C088642190FBF1F201FB120080
:103B900081B204EB4402B34800EB82004181601C17
:103BA00084B20A2CFFF65AAF34E0002430E0002043
:103BB00000EB8400AC4931F8101004EB4402A94832
:103BC00020F82210012000EB8400A74931F81010E2
:103BD00004EB4402A34800EB82004180022000EB8A
:103BE0008400A14931F8101004EB44029D4800EB19
:103BF00082008180032000EB84009B4931F8101083
:103C000004EB4402974800EB8200C180601C84B240
:103C10000A2CCCDB02244FF6FF7000EA441410AAF1
:103C20002021204600F03EFF002405E010A8005DA2
:103C30000DF80400601C84B2202CF7DB0224641C05
:103C40004FF6FF7000EA441410AA2021204600F02D
:103C500029FF002407E010A8015D04F120000DF801
:103C60000010601C84B2202CF5DB9DF83F00552825
:103C70007ED100250024B0E02846691C8DB21DF8D5
:103C8000001004EB44027748783020F8221004EB4F
:103C9000440130F821004FF6FF7101EA002104EBE6
:103CA00044027048783020F8221004EB440130F8C8
:103CB00021202846691C8DB21DF80000104481B2F5
:103CC00004EB44026748783020F822102846691C2B
:103CD0008DB21DF8001004EB44026248783000EB0E
:103CE0008200418004EB44015E48783000EB8100A3
:103CF00040884FF6FF7101EA002104EB4402594865
:103D0000783000EB8200418004EB44015548783064
:103D100000EB810042882846691C8DB21DF8000026
:103D2000104481B204EB44024E48783000EB82002C
:103D300041802846691C8DB21DF800604FF6FF7067
:103D400000EA06262846691C8DB21DF800003044A2
:103D500086B24FF47A7096FBF0F081B204EB440225
:103D60004048783000EB820081804FF47A7000E0A8
:103D700037E096FBF0F100FB116081B204EB4402E6
:103D80003848783000EB8200C18004EB44013548AC
:103D9000783000EB8100C088642190FBF1F081B2A3
:103DA00004EB44022F48783000EB8200018104EBE1
:103DB00044012C48783000EB8100C088642190FBDE
:103DC000F1F201FB120081B204EB44022548783085
:103DD00000EB82004181601C84B20A2CFFF64CAFDC
:103DE00038E0002434E0002000EB84001E4931F864
:103DF000101004EB44021B48783020F822100120F8
:103E000000EB8400184931F8101004EB4402154807
:103E1000783000EB82004180022000EB84001249E0
:103E200031F8101004EB44020E48783000EB8200A9
:103E30008180032000EB84000B4931F8101004EB63
:103E400044020848783000EB8200C180601C84B2D4
:103E50000A2CC8DB04244FF6FF7000EA441410AAB1
:103E6000202103E0FA02002076640108204600F0D9
:103E700019FE002405E010A8005D0DF80400601C88
:103E800084B2202CF7DB0424641C4FF6FF7000EA98
:103E9000441410AA2021204600F004FE002407E06C
:103EA00010A8015D04F120000DF80010601C84B220
:103EB000202CF5DB9DF83F00552848D10025002433
:103EC00042E02846691C8DB21DF80010FE4820F81B
:103ED000241030F824004FF6FF7101EA0021FA485F
:103EE00020F8241030F824202846691C8DB21DF8D3
:103EF0000000104481B2F44820F824102846691CC0
:103F00008DB21DF80010F04800EB84004180EE48AF
:103F100000EB840040884FF6FF7101EA0021EA4877
:103F200000EB84004180E84800EB8400428828468A
:103F3000691C8DB21DF80000104481B2E24800EB0C
:103F400084004180601C84B20F2CBADB18E000248E
:103F500014E0002000EB4400DC4931F81010DA488E
:103F600020F82410012000EB4400D84931F810104B
:103F7000D54800EB84004180601C84B20F2CE8DB44
:103F800006244FF6FF7000EA441410AA20212046B0
:103F900000F088FD002405E010A8005D0DF8040085
:103FA000601C84B2202CF7DB0624641C4FF6FF70E3
:103FB00000EA441410AA2021204600F073FD0024DA
:103FC00007E010A8015D04F120000DF80010601C4E
:103FD00084B2202CF5DB9DF83F0055287ED10025CA
:103FE000002486E02846691C8DB21DF8001004EB01
:103FF0004402B74820F8121004EB440130F81100D5
:104000004FF6FF7101EA002104EB4402B04820F8AA
:10401000121004EB440130F811202846691C8DB2BF
:104020001DF80000104481B204EB4402A84820F8B7
:1040300012102846691C8DB21DF8001004EB4402D2
:10404000A34800EB4200418004EB4401A04800EB90
:10405000410040884FF6FF7101EA002104EB440261
:104060009B4800EB4200418004EB4401984800EB80
:10407000410042882846691C8DB21DF8000010449A
:1040800081B204EB4402924800EB42004180284692
:10409000691C8DB21DF8001004EB44028C4800EB43
:1040A0004200818004EB4401894800EB4100808894
:1040B0004FF6FF7101EA002104EB4402844800EB53
:1040C0004200818004EB4401814800EB410082887A
:1040D0002846691C8DB21DF8000000E00DE0104478
:1040E00081B204EB44027A4800EB42008180601CFC
:1040F00084B20A2CFFF676AF27E0002423E004EB1D
:104100004400744931F8101004EB4402704820F860
:10411000121004EB4400401C6E4931F8101004EBFF
:1041200044026B4800EB4200418004EB4400801CD9
:10413000684931F8101004EB4402654800EB420076
:104140008180601C84B20A2CD9DB0A244FF6FF70F0
:1041500000EA441410AA2021204600F0A3FC002409
:1041600005E010A8005D0DF80400601C84B2202C4E
:10417000F7DB0A24641C4FF6FF7000EA441410AA0F
:104180002021204600F08EFC002407E010A8015DED
:1041900004F120000DF80010601C84B2202CF5DB27
:1041A0009DF83F00552824D1002500241EE0284614
:1041B000691C8DB21DF80010474820F8141030F823
:1041C00014004FF6FF7101EA0021434820F8141053
:1041D00030F814202846691C8DB21DF800001044E8
:1041E00081B23D4820F81410601C84B2042CDEDB40
:1041F0000BE0002407E0394830F81410364820F866
:104200001410601C84B2042CF5DB08244FF6FF70F8
:1042100000EA441410AA2021204600F043FC0024A8
:1042200005E010A8005D0DF80400601C84B2202C8D
:10423000F7DB0824641C4FF6FF7000EA441410AA50
:104240002021204600F02EFC002407E010A8015D8C
:1042500004F120000DF80010601C84B2202CF5DB66
:104260009DF83F0055287DD10025002496E0284682
:10427000691C8DB21DF8001004EB440214483C3058
:1042800020F8121004EB440130F811004FF6FF71D2
:1042900001EA002104EB44020D483C3020F81210E2
:1042A00004EB440130F811202846691C8DB21DF83A
:1042B0000000104481B204EB440205483C3020F871
:1042C00012102846691C0BE0F8030020C6640108A0
:1042D0008202002002650108220F0020CE6501083D
:1042E0008DB21DF8001004EB4402F14800EB4200CF
:1042F000418004EB4401EE4800EB410040884FF65A
:10430000FF7101EA002104EB4402E94800EB42009E
:10431000418004EB4401E64800EB41004288284616
:10432000691C8DB21DF80000104481B204EB4402F8
:10433000DF4800EB420041802846691C8DB21DF821
:10434000001004EB4402DA4800EB4200818004EBE9
:104350004401D74800EB410080884FF6FF7101EA25
:10436000002100E01EE004EB4402D14800EB4200D3
:10437000818004EB4401CE4800EB4100828828464E
:10438000691C8DB21DF80000104481B204EB440298
:10439000C74800EB42008180601C84B20A2CFFF603
:1043A00066AF27E0002423E004EB4400C14931F864
:1043B000101004EB4402BE4820F8121004EB440035
:1043C000401CBC4931F8101004EB4402B84800EB23
:1043D0004200418004EB4400801CB64931F81010C3
:1043E00004EB4402B24800EB42008180601C84B2BE
:1043F0000A2CD9DB0C244FF6FF7000EA441410AAF3
:104400002021204600F04EFB00259DF85F00552836
:104410004BD12846691C8DB210A9095CA648C0F88A
:10442000D810D0F8D8000102A348C0F8D810D0F8AE
:10443000D8202846691C8DB210A9085C11189E4826
:10444000C0F8D810D0F8D80001029B48C0F8D810A6
:10445000D0F8D8202846691C8DB210A9085C111824
:104460009548C0F8D810D0F8D80001029248C0F89A
:10447000D810D0F8D8202846691C8DB210A9085C45
:1044800011188D48C0F8D8102846691C8DB210A9A3
:10449000095C894880F8DC1090F8DC00C7280CDD46
:1044A000C721854880F8DC1007E04FF400018248FE
:1044B000C0F8D810642180F8DC100E244FF6FF708D
:1044C00000EA441410AA2021204600F0EBFA00254F
:1044D0009DF85F00552848D12846691C8DB210A967
:1044E000085C7349A239C8820846C08A4FF6FF713A
:1044F00001EA00206E49A239C8820846C28A2846CD
:10450000691C8DB210A9085C10446949A239C8829F
:104510000846C08AB0F5105F02DB4FF40060C88225
:104520002846691C8DB210A9085C6149A2398882AD
:104530000846808A4FF6FF7101EA00205C49A239E3
:1045400088820846828A2846691C8DB210A9085CB8
:1045500010445749A23988820846808AB0F57A7F8C
:104560000BDB4FF46670888207E04FF4006050491F
:10457000A239C8824FF4667088824FF4007000F050
:10458000BAFA4D4981F8F00020244FF6FF7000EA96
:10459000441410AA2021204600F084FA9DF85F0000
:1045A000552812D19DF847004449088008460088E4
:1045B0004FF6FF7101EA0020404908809DF848004D
:1045C000098808443D49088002E000203B490880F2
:1045D00021244FF6FF7000EA441410AA202120463F
:1045E00000F060FA9DF85F00552812D19DF8470051
:1045F00033490880084600884FF6FF7101EA002021
:104600002F4908809DF84800098808442C490880F3
:1046100003E04FF6FF702A49088022244FF6FF700E
:1046200000EA441410AA2021204600F03BFA9DF82D
:104630005F00552812D19DF849002249088008469C
:1046400000884FF6FF7101EA00201E4908809DF89E
:104650004A00098808441B49088002E000201949E3
:10466000088023244FF6FF7000EA441410AA20218A
:10467000204600F017FA9DF85F00552812D19DF8EA
:10468000490011490880084600884FF6FF7101EA89
:1046900000200D4908809DF84A00098808440A490D
:1046A000088003E04FF6FF700549088018B070BD20
:1046B000BE0200203E6501081C2200209E01002051
:1046C0009C0100209A010020980100202DE9F84F5C
:1046D0008046894692460921012001F03BF9454672
:1046E000B5F5FA7F02D3A5F5FA7500E00025642040
:1046F000B5FBF0F087B207EBC70000EB0710A5EBA6
:1047000080050A20B5FBF0F01FFA80FB0BEB8B0055
:10471000A5EB4005A8B200902FB107F1300188B297
:1047200000F0ACFD02E0202000F0A8FD0BF130010C
:1047300088B200F0A3FD2E2000F0A0FD00993031DA
:1047400088B200F09BFD0921022001F003F94D46DB
:1047500025F07F452C0D00BF0A2C05DA04F130014D
:1047600088B200F08BFD04E004F1370188B200F05C
:1047700085FD2C0C04F00F040A2C05DA04F130013D
:1047800088B200F07BFD04E004F1370188B200F04C
:1047900075FDC5F30F3404F00F040A2C05DA04F19B
:1047A000300188B200F06AFD04E004F1370188B2FC
:1047B00000F064FDC5F30F2404F00F040A2C05DAA1
:1047C00004F1300188B200F059FD04E004F1370132
:1047D00088B200F053FDC5F30F1404F00F040A2C47
:1047E00005DA04F1300188B200F048FD04E004F17C
:1047F000370188B200F042FDACB204F00F040A2C7D
:1048000005DA04F1300188B200F038FD04E004F16B
:10481000370188B200F032FD0921032001F09AF837
:10482000554640F6C410854200D305464FF47A70D1
:10483000B5FBF0F606EB4600C0EBC610A5EBC005D5
:1048400006F1300188B200F019FD6420B5FBF0F6E6
:1048500006EBC60000EB0610A5EB800506F1300163
:1048600088B200F00BFD0A20B5FBF0F606EB8600DF
:10487000A5EB400506F1300188B200F0FFFC2E46A2
:1048800006F1300188B200F0F9FCBDE8F88FF0B510
:1048900089B007460E46354625F07F4500242A0E8E
:1048A0002146641C01A842542A0C2146641C42542F
:1048B000C5F307222146641C42542146641C45541A
:1048C0002146641C475455208DF823000C244FF6D4
:1048D000FF7000EA441401AA2021204600F026F9C6
:1048E00009B0F0BD2DE9F84F804689469246052172
:1048F000012001F02FF84746642F06DBA7F1640082
:10490000C7B22B2000F0BAFC05E0C7F16400C7B2C3
:104910002D2000F0B3FC0A2097FBF0F000F0FF0B15
:104920000BEB8B00A7EB4000C0B200900BF1300006
:1049300000F0A4FC2E2000F0A1FC0098303000F024
:104940009DFC0521022001F005F84D4625F07F452C
:104950002C0D00BF0A2C05DA04F1300188B200F0FA
:104960008DFC04E004F1370188B200F087FC2C0CC8
:1049700004F00F040A2C05DA04F1300188B200F0CB
:104980007DFC04E004F1370188B200F077FCC5F348
:104990000F3404F00F040A2C05DA04F1300188B258
:1049A00000F06CFC04E004F1370188B200F066FC12
:1049B000C5F30F2404F00F040A2C05DA04F13001CA
:1049C00088B200F05BFC04E004F1370188B200F02B
:1049D00055FCC5F30F1404F00F040A2C05DA04F19A
:1049E000300188B200F04AFC04E004F1370188B2DB
:1049F00000F044FCACB204F00F040A2C05DA04F118
:104A0000300188B200F03AFC04E004F1370188B2CA
:104A100000F034FC0521032000F09CFF554640F6D1
:104A2000C410854200D305464FF47A70B5FBF0F60A
:104A300006EB4600C0EBC610A5EBC00506F1300141
:104A400088B200F01BFC6420B5FBF0F606EBC60054
:104A500000EB0610A5EB800506F1300188B200F0EE
:104A60000DFC0A20B5FBF0F606EB8600A5EB400531
:104A700006F1300188B200F001FC2E4606F130014B
:104A800088B200F0FBFBBDE8F88F08E0421E90B250
:104A9000002101E04A1C91B2B1F57A7FFADB0028CF
:104AA000F4D170472DE9F04105460F46164600F057
:104AB00025F9A02000F09EFA281200F09BFAE8B237
:104AC00000F098FA00F01AF9A12000F093FA0024FF
:104AD00005E0002000F068F83055601CC4B2781E74
:104AE000A042F6DC012000F05FF8305500F0D8F964
:104AF0000120BDE8F08170B5044600F0FFF8A02069
:104B000000F078FA201200F075FAE0B200F072FAC4
:104B100000F0F4F8A12000F06DFA012000F044F854
:104B2000054600F0BDF9284670BD00002DE9F041B2
:104B300004460F46904600F0E1F8A02000F05AFA33
:104B4000201200F057FAE0B200F054FA002505E018
:104B500018F8050000F04EFA681CC5B2BD42F7DB3C
:104B600000F09EF9002600E0761C03488642FBD345
:104B70000120BDE8F08100006C3F090070B50446DB
:104B80000D4600F0BBF8A02000F034FA201200F02F
:104B900031FAE0B200F02EFA284600F02BFA064671
:104BA00000F07EF9304670BD70B505460024002641
:104BB00042E04FF480715048FCF7B7FC4FF480712D
:104BC0004D48FCF7B2FC4FF480714B48FCF7ADFC4C
:104BD0004FF480714848FCF7A8FC4FF480714648B8
:104BE000FCF7A3FC4FF400714348FCF7A0FC4FF422
:104BF00080714148FCF79BFC4FF480713E48FCF704
:104C000096FC4FF480713C48FCF791FC4FF48071A6
:104C10003948FCF78CFC4FF480713748FCF787FC6F
:104C20006006040E4FF400713348FCF775FC08B1C0
:104C3000601CC4B2701CC6B2082EBADB4FF480717F
:104C40002D48FCF772FC2DB14FF400712A48FCF797
:104C50006EFC04E04FF400712748FCF766FC4FF44B
:104C600080712548FCF761FC4FF480712248FCF705
:104C70005CFC4FF480712048FCF757FC4FF48071C6
:104C80001D48FCF752FC4FF480711B48FCF74DFCAB
:104C90004FF480711848FCF74AFC4FF480711648B5
:104CA000FCF745FC4FF480711348FCF740FC4FF4CF
:104CB00080711148FCF73BFC4FF480710E48FCF703
:104CC00036FC4FF480710C48FCF72FFC4FF48071D8
:104CD0000948FCF72AFC4FF480710748FCF725FCD3
:104CE0004FF480710448FCF720FC4FF480710248B7
:104CF000FCF71BFC204670BD000C014010B54FF4C2
:104D000080716648FCF711FC4FF400716348FCF7B2
:104D10000EFC4FF400716148FCF709FC4FF4007180
:104D20005E48FCF704FC4FF400715C48FCF7FFFBA5
:104D30004FF400715948FCF7FAFB4FF400715748E3
:104D4000FCF7F5FB4FF400715448FCF7F0FB4FF40F
:104D500000715248FCF7EBFB4FF400714F48FCF731
:104D6000E6FB4FF400714D48FCF7E1FB4FF4807116
:104D70004A48FCF7DCFB4FF480714848FCF7D7FB4E
:104D80004FF480714548FCF7D2FB4FF480714348E3
:104D9000FCF7CDFB4FF480714048FCF7C8FB4FF4A3
:104DA00080713E48FCF7C3FB4FF480713B48FCF731
:104DB000BEFB4FF480713948FCF7B9FB4FF48071AA
:104DC0003648FCF7B4FB4FF480713448FCF7AFFB76
:104DD0004FF400713148FCF7A8FB4FF400712F48E5
:104DE000FCF7A3FB4FF400712C48FCF79EFB4FF43B
:104DF00000712A48FCF799FB4FF400712748FCF733
:104E000094FB4FF400712548FCF78FFB4FF40071C1
:104E10002248FCF78AFB4FF400712048FCF785FB21
:104E20004FF400711D48FCF780FB4FF400711B48E4
:104E3000FCF77BFB4FF480711848FCF776FB4FF4CE
:104E400080711648FCF771FB4FF480711348FCF732
:104E50006CFB4FF480711148FCF767FB4FF48071D5
:104E60000E48FCF762FB4FF480710C48FCF75DFBC9
:104E70004FF480710948FCF758FB4FF480710748E4
:104E8000FCF753FB4FF480710448FCF74EFB4FF4E2
:104E900080710248FCF749FB10BD0000000C014086
:104EA00010B54FF480715248FCF73FFB4FF400718E
:104EB0004F48FCF73AFB4FF480714D48FCF737FB45
:104EC0004FF480714A48FCF732FB4FF48071484838
:104ED000FCF72DFB4FF480714548FCF728FB4FF49D
:104EE00080714348FCF723FB4FF480714048FCF786
:104EF0001EFB4FF480713E48FCF719FB4FF48071A4
:104F00003B48FCF714FB4FF480713948FCF70FFB6A
:104F10004FF480713648FCF70AFB4FF400713448B7
:104F2000FCF705FB4FF400713148FCF700FB4FF430
:104F300000712F48FCF7FBFA4FF400712C48FCF786
:104F4000F6FA4FF400712A48FCF7F1FA4FF40071B9
:104F50002748FCF7ECFA4FF400712548FCF7E7FA14
:104F60004FF400712248FCF7E2FA4FF40071204838
:104F7000FCF7DDFA4FF400711D48FCF7D8FA4FF446
:104F800000711B48FCF7D3FA4FF400711848FCF786
:104F9000CEFA4FF400711648FCF7C9FA4FF40071CD
:104FA0001348FCF7C4FA4FF400711148FCF7BFFA3C
:104FB0004FF400710E48FCF7BAFA4FF400710C4838
:104FC000FCF7B5FA4FF400710948FCF7B0FA4FF45A
:104FD00000710748FCF7ABFA4FF400710448FCF786
:104FE000A6FA4FF480710248FCF79FFA10BD00004A
:104FF000000C014070B505462E460024A7E04FF492
:1050000080719D48FCF791FA4FF480719A48FCF743
:105010008CFA4FF480719848FCF787FA4FF480714E
:105020009548FCF782FA4FF480719348FCF77DFABB
:105030004FF480719048FCF778FA4FF480718E48F5
:10504000FCF773FA4FF480718B48FCF76EFA4FF45B
:1050500080718948FCF769FA4FF480718648FCF743
:1050600064FA06F0800028B14FF400718248FCF722
:105070005EFA04E04FF400717F48FCF756FA4FF4F3
:1050800080717D48FCF751FA4FF480717A48FCF743
:105090004CFA4FF480717848FCF747FA4FF480716E
:1050A0007548FCF742FA4FF480717348FCF73DFAFB
:1050B0004FF480717048FCF738FA4FF480716E48F5
:1050C000FCF733FA4FF480716B48FCF72EFA4FF47B
:1050D00080716948FCF729FA4FF480716648FCF743
:1050E00024FA4FF480716448FCF721FA4FF4807180
:1050F0006148FCF71CFA4FF480715F48FCF717FA1F
:105100004FF480715C48FCF712FA4FF480715A48F2
:10511000FCF70DFA4FF480715748FCF708FA4FF48A
:1051200080715548FCF703FA4FF480715248FCF740
:10513000FEF94FF480715048FCF7F9F94FF4807193
:105140004D48FCF7F4F97006060E601CC4B2082C3A
:10515000FFF655AF4FF480714748FCF7E6F94FF47E
:1051600000714548FCF7E3F94FF480714248FCF7C1
:10517000DCF94FF480714048FCF7D7F94FF48071A7
:105180003D48FCF7D2F94FF480713B48FCF7CDF96C
:105190004FF480713848FCF7C8F94FF480713648F5
:1051A000FCF7C3F94FF480713348FCF7BEF94FF4B4
:1051B00080713148FCF7B9F94FF480712E48FCF743
:1051C000B4F94FF480712C48FCF7AFF94FF48071BB
:1051D0002948FCF7ACF94FF480712748FCF7A7F990
:1051E0004FF480712448FCF7A2F94FF480712248F3
:1051F000FCF79DF94FF480711F48FCF798F94FF4C4
:1052000080711D48FCF793F94FF480711A48FCF740
:105210008EF94FF480711848FCF789F94FF48071CA
:105220001548FCF784F94FF480711348FCF77FF9B7
:105230004FF400711048FCF76FF908B1FF2400E04B
:1052400000244FF480710C48FCF76FF94FF4807123
:105250000948FCF76AF94FF480710748FCF765F9D3
:105260004FF480710448FCF760F94FF480710248F4
:10527000FCF75BF9204670BD000C014070B5044698
:10528000802C05DAE5B22946FA2000F09DFB09E002
:1052900025122946FA2000F097FBE5B22946FA20AC
:1052A00000F092FB70BD00002DE9FF5F04460F4641
:1052B0009046039808B1FF2600E00026022C03DA8E
:1052C00000201E49087004E001201C490870A01E3F
:1052D000C4B220074FEA106A102000EB041000F05F
:1052E000FF0B3421F82000F06FFB55461AE005F162
:1052F0008000C1B2F82000F067FB07F18000C1B266
:10530000F82000F061FB4FF0000907E03146FA2079
:1053100000F05AFB09F1010000F0FF09C145F5DB7F
:10532000681CC5B25D45E2DB3621F82000F04CFB7D
:105330003021F82000F048FBBDE8FF9F000000206E
:105340002DE9F05F05460E469246BAF1000F01D0F6
:10535000FF2700E00027022D03DA00202A49087009
:1053600004E0012028490870A81EC5B228074FEAAA
:105370001068102000EB051000F0FF0906F0010B8B
:1053800076103421F82000F01FFBBBF1000F16D17E
:10539000444611E004F18000C1B2F82000F014FB93
:1053A00006F18000C1B2F82000F00EFB3946FA2069
:1053B00000F00AFB601CC4B24C45EBDB19E044462C
:1053C00015E004F18000C1B2F82000F0FDFA06F10A
:1053D0008000C1B2F82000F0F7FA0021FA2000F0B6
:1053E000F3FA3946FA2000F0EFFA601CC4B24C45DB
:1053F000E7DB3621F82000F0E7FA3021F82000F052
:10540000E3FABDE8F09F00000000002070B50546FB
:105410000E4614461DB901200849C1F8B0003146B6
:10542000284600F097FA04E014F8011BFA2000F077
:10543000CBFA20780028F7D170BD0000FC3D002099
:105440002DE9F0479E48D0F8F400F0B92020FFF78E
:1054500015FF2020FFF712FF2020FFF70FFF20206D
:10546000FFF70CFF2020FFF709FF2020FFF706FFC2
:105470002020FFF703FF2020FFF700FF2020FFF789
:10548000FDFE2020FFF7FAFE18E18D48D0F8F40069
:10549000012878D12020FFF7F1FE2020FFF7EEFE53
:1054A0002020FFF7EBFE874804884FF47A70B4FBA6
:1054B000F0F505EB4500C0EBC510A4EBC00464207B
:1054C000B4FBF0F606EBC60000EB0610A4EB80047C
:1054D0000A20B4FBF0F800BF00BF1DB92020FFF781
:1054E000CDFE04E005F1300188B2FFF7C7FE25B913
:1054F0001EB92020FFF7C2FE04E006F1300188B299
:10550000FFF7BCFE08F1300188B2FFF7B7FE562066
:10551000FFF7B4FE6C4804884FF47A70B4FBF0F5E2
:1055200005EB4500C0EBC510A4EBC0046420B4FB40
:10553000F0F606EBC60000EB0610A4EB80040A2090
:10554000B4FBF0F808EB8800A4EB4004A1461DB9B9
:105550002020FFF793FE04E005F1300188B2FFF749
:105560008DFE25B91EB92020FFF788FE04E006F164
:10557000300188B2FFF782FE08F1300188B2FFF7F0
:105580007DFE9BE0FFE74E48D0F8F4000228F8D1FA
:105590004B48D0F8C45000272020FFF76FFE4FF48F
:1055A0007A70B5FBF0F424B91FB92020FFF766FE2E
:1055B00005E004F1300188B2FFF760FE012704EB3B
:1055C0004400C0EBC410A5EBC0056420B5FBF0F4AB
:1055D00024B91FB92020FFF751FE05E004F1300186
:1055E00088B2FFF74BFE012704EBC40000EB041068
:1055F000A5EB80050A20B5FBF0F424B91FB92020E3
:10560000FFF73CFE05E004F1300188B2FFF736FEFB
:10561000012704EB8400A5EB40052C4604F1300182
:1056200088B2FFF72BFE2648D0F8CC500027202068
:10563000FFF724FE4FF47A70B5FBF0F424B91FB9DC
:105640002020FFF71BFE05E004F1300188B2FFF7D0
:1056500015FE012704EB4400C0EBC410A5EBC00508
:105660006420B5FBF0F424B91FB92020FFF706FE33
:1056700005E004F1300188B2FFF700FE012704EBDA
:10568000C40000EB0410A5EB80050A20B5FBF0F484
:1056900024B91FB92020FFF7F1FD05E004F1300126
:1056A00088B2FFF7EBFD012704EB8400A5EB400572
:1056B0002C4604F1300188B2FFF7E0FDBDE8F08729
:1056C0001C220020A0010020A201002070B5334858
:1056D000D0F8F400552812D02020FFF7CFFD20206D
:1056E000FFF7CCFD2020FFF7C9FD2020FFF7C6FD06
:1056F0002020FFF7C3FD2020FFF7C0FD4CE0202055
:10570000FFF7BCFD2020FFF7B9FD2548058E0026D8
:105710004FF47A70B5FBF0F424B91EB92020FFF7DE
:10572000ADFD05E004F1300188B2FFF7A7FD0126C9
:1057300004EB4400C0EBC410A5EBC0056420B5FB2E
:10574000F0F424B91EB92020FFF798FD05E004F11C
:10575000300188B2FFF792FD012604EBC40000EB94
:105760000410A5EB80050A20B5FBF0F424B91EB99E
:105770002020FFF783FD05E004F1300188B2FFF738
:105780007DFD012604EB8400A5EB40052C4604F1C9
:10579000300188B2FFF772FD70BD00001C220020AE
:1057A0001C02002010B54FF480713A48FBF7BDFE93
:1057B0004FF400713848FBF7B8FE4FF400713548DC
:1057C000FBF7B3FE4FF480613248FBF7AEFE4FF4B7
:1057D00080713148FBF7A9FEC820FFF756F94FF456
:1057E00080712D48FBF7A3FE4FF480612948FBF739
:1057F0009EFE0020294908703021F82000F0E4F8CE
:105800003220FFF742F93021F82000F0DDF8322095
:10581000FFF73BF90C21F82000F0D6F83220FFF713
:1058200034F90121F82000F0CFF8C820FFF72DF956
:105830000621F82000F0C8F8C820FFF726F901205B
:10584000164908703021F82000F0BEF83220FFF72A
:105850001CF93021F82000F0B7F83220FFF715F9D5
:105860000C21F82000F0B0F83220FFF70EF90121EA
:10587000F82000F0A9F8C820FFF707F90621F82062
:1058800000F0A2F8C820FFF700F900F009F800F0D6
:105890007DF810BD0008014000100140000000200C
:1058A00070B500202A4908703421F82000F08CF8E7
:1058B0000120274908703421F82000F085F80020E5
:1058C00023490870002415E004F18000C1B2F820DB
:1058D00000F07AF88021F82000F076F8002505E045
:1058E0000021FA2000F070F8681CC5B2182DF7DB13
:1058F000601CC4B2202CE7DB01201549087000248D
:1059000015E004F18000C1B2F82000F05DF88021BC
:10591000F82000F059F8002505E00021FA2000F0F9
:1059200053F8681CC5B2182DF7DB601CC4B2202CDC
:10593000E7DB0020064908703621F82000F044F823
:105940000120034908703621F82000F03DF870BDB1
:105950000000002070B504460D46022C03DA00203A
:105960000949087002E0012007490870012C01D0A4
:10597000032C02D105F11000C5B205F18000C1B2BF
:10598000F82000F021F870BD0000002010B50020C4
:105990000C4908703021F82000F016F80121F82099
:1059A00000F012F80120074908703021F82000F0BB
:1059B0000BF80121F82000F007F8C820FFF765F880
:1059C00010BD0000000000202DE9F04107460E4602
:1059D0003D4600242DE04E48007828B94FF48071F0
:1059E0004C48FBF7A2FD04E04FF400714A48FBF776
:1059F0009CFD05F0800028B14FF400714548FBF78D
:105A000096FD04E04FF400714248FBF78EFD4048DC
:105A1000007828B94FF480713E48FBF788FD04E018
:105A20004FF400713C48FBF782FD6806050E601CD0
:105A3000C4B2082CCFDB06F0F00500242DE034487A
:105A4000007828B94FF480713248FBF76EFD04E00E
:105A50004FF400713048FBF768FD05F0800028B175
:105A60004FF400712B48FBF762FD04E04FF4007126
:105A70002848FBF75AFD2648007828B94FF4807172
:105A80002448FBF754FD04E04FF400712248FBF773
:105A90004EFD6806050E601CC4B2082CCFDB300733
:105AA000060E06F0F00500242DE01948007828B90C
:105AB0004FF480711748FBF738FD04E04FF4007194
:105AC0001548FBF732FD05F0800028B14FF4007156
:105AD0001048FBF72CFD04E04FF400710D48FBF774
:105AE00024FD0B48007828B94FF480710948FBF772
:105AF0001EFD04E04FF400710748FBF718FD68062F
:105B0000050E601CC4B2082CCFDBBDE8F08100009C
:105B1000000000200008014000100140ACB000BFB0
:105B200000BF0EF0E5FCFE48B0F89E1000F50050F6
:105B3000A0F8F210B0F8F20000EB80004FF6FF7111
:105B400001EA8001F748A0F8F21000202B9008E04D
:105B50000021F54A2B9842F820102B98401C81B266
:105B60002B912B981428F3DB0021F048A0F8FE10AD
:105B7000C0F80811EA48B0F8DC0040F2E73188428A
:105B800004D10121E948C0F8DC1B03E00021E7480B
:105B9000C0F8DC1BE248B0F8D810E448C0F8D41BC9
:105BA00000202B9017E0E148D0F8D40B012807D152
:105BB000DF492B9831F81010DE4A22F8101006E069
:105BC000DD492B9831F81010DA4A22F810102B9882
:105BD000401C81B22B9140F25D512B988842E2DB50
:105BE0002021D648FBF7A3FC4FF47A71CF48C0F8C8
:105BF000D81B00202B900EE00021CA4AFE322B98C1
:105C000022F8101002F500622B9822F810102B9841
:105C1000401C81B22B912B98B0F5806FECDBC04813
:105C2000B0F89C00642190FBF1F1C048C0F80C1161
:105C3000BB48B0F89C10BD48D0F80C0100EBC00286
:105C400002EB0010A1EB80000A21B0FBF1F1B74894
:105C5000C0F81011B248B0F89C10B448D0F80C014C
:105C600000EBC00202EB0010A1EB8001AF48D0F8BE
:105C7000100100EB8000A1EB4001AC48C0F814110A
:105C8000D0F80C0164214843A849C1F80C0108462A
:105C9000D0F81001C0EB00108100A448C0F810112A
:105CA0000021C0F80411C0F80811C0F800119D4887
:105CB000C0F8F410A2480078F6280BD101220A217E
:105CC0000846FAF747FE90209E49087001209E4939
:105CD00008702CE09A4800787B280BD101220A2119
:105CE0000846FAF737FE8020964908700120964949
:105CF00008701CE092480078F32809D1022211466E
:105D00000320FAF727FE02218648C0F8F4100EE0BF
:105D10008B4800787E280AD1032202211046FAF728
:105D200019FEA020874908700120874908701020BB
:105D30008649087001218648017000208549086065
:105D4000854908804FF6FE70844908800020844908
:105D500008800420834908700020834908701920B6
:105D60008249087040208249087041F250408149C0
:105D700008801020804908700120804908700020A8
:105D80007F4908607F4908804FF6FE707E49088091
:105D900000207E49088004207D49087000207D494C
:105DA000087019207C49087040207C49087041F235
:105DB00050407B4908805A48B0F86A00642190FB43
:105DC000F1F201FB12025648B0F86800029000EBB5
:105DD000D070C2EB6000734908805148B0F86A0087
:105DE000642190FBF1F201FB12024D48B0F86810FB
:105DF00001EBD17002EB600002916B4908800DF05D
:105E0000BDB95D48007810282BD15C48007858B1A6
:105E100000205A490870FCF7ADFF00206349088054
:105E20004FF4C870564908605548006848B92020AA
:105E30005149087001205149087064205049086098
:105E400014E25B4880780128FAD1FCF793FF202008
:105E50004949087001204949087064204849086090
:105E600004E245480078202858D1454800680028B9
:105E7000E6D1444908804F480178424802880088AA
:105E8000401C404B18804C4881544A484178184681
:105E900002880088401C1880474881544548827811
:105EA000184601880088401C1880434842544148E5
:105EB000C278184601880088401C18803E48425429
:105EC0003C480279184601880088401C18803A48EE
:105ED000425438484279184601880088401C18808E
:105EE0003548425433488279184601880088401C5E
:105EF0001880314842542F48C279184601880088DA
:105F0000401C18802C484254184600780290FCF738
:105F100039FF4FF4C8711A4801604FE055E00000A6
:105F20001C0200201C220020CC0100201C3200207A
:105F3000C44E0108343300207E590108001001408E
:105F4000170000202C0000202E0000202F00002031
:105F50006F010020700100207401002076010020F4
:105F6000780100207A0100207B0100207C010020C4
:105F70007D0100207E0100208001002081010020A1
:105F800084010020880100208A0100208C0100206B
:105F90008E0100208F01002090010020910100203F
:105FA000920100209401002096010020A40100200D
:105FB000B03E0020D6650108BC4000203020FA49E0
:105FC00008700120F949087050E1F748007830283E
:105FD000FAD1F748006830B92020F3490870012051
:105FE000F249087042E1F34880780128ECD1F14889
:105FF000007B01287ED1EF48407B0328FAD1ED4891
:10600000807B0628F6D1EB48C07BEB490880084628
:1060100000884FF6FF7101EA0020E7490880E54853
:10602000007C09880844E4490880E248C07CE349D0
:106030000880084600884FF6FF7101EA0020DF491A
:106040000880DC48007D09880844DC490880DA487B
:106050000088DB490988884210DDD7480088D84984
:106060000880D84A072102200EF07CF8D54BD3488F
:106070000288D148018820200EF0CAF9CE48008855
:10608000D1490988884210DACB480088CE49088077
:10609000CC4A072102200EF065F8CA4BC748028897
:1060A000C548018821200EF0B3F9C4480088C749CB
:1060B0000988884210DDC1480088C4490880C14A67
:1060C000072102200EF04EF8BE4BBC480288BA48A9
:1060D000018822200EF09CF9BD48008800EB80006A
:1060E000B6490988B1EB400F24DDBA48008800EBBF
:1060F000800000E0A6E0B1490988B1EB400F19DA51
:10610000B548008828B1B44800884FF6FF7188422E
:1061100010D1AA480088B0490880AA4A0721022065
:106120000EF020F8A74BA5480288A3480188232039
:106130000EF06EF90120A9490880A948007800F006
:106140000F0000287ED0A748B0F8660000EB800062
:1061500099490988B1EB400F1FDDA3A20021084631
:10616000FFF754F9A0A200210120FFF74FF9A5A2E3
:1061700000210220FFF74AF99BA200210320FFF72C
:1061800045F94CF2503201210846FAF7E3FB0120B1
:10619000A349C1F8A00000BFFEE79248B0F868002C
:1061A00000EB800085490988B1EB400F1FDD8EA20E
:1061B00000210846FFF72AF98BA200210120FFF7F2
:1061C00025F998A200210220FFF720F986A20021DC
:1061D0000320FFF71BF94CF2503201210846FAF771
:1061E000B9FB01208E49C1F8A00000BFFEE7784846
:1061F000008800EB800071490988B1EB400F2ADD6F
:106200007448008800EB80006C490988B1EB400FAE
:1062100021DA75A200210846FFF7F8F872A20021E2
:106220000120FFF7F3F886A200210220FFF7EEF825
:106230006DA200210320FFF7E9F84CF25032012152
:10624000084600E007E0FAF785FB01207449C1F831
:10625000A00000BFFEE7FCF78DFD2020524908702A
:106260000120524908706420514908607B48007839
:1062700010281BD17A48007868B10020784908704E
:1062800020217848FBF753F910217648FBF74FF9A6
:106290000A207549086074480068002805D120204C
:1062A0006E49087001206E490870EEE16B48007875
:1062B000202878D100206D490880C2220846018834
:1062C0000088401C694B18806948425400221846D7
:1062D00001880088401C18806548425408211846EF
:1062E00002880088401C18806148815461480088F9
:1062F0000212184601880088401C18805C484254ED
:106300005C480278184601880088401C188058486C
:106310004254594800786030C2B21846018800885B
:10632000401C18805248425454480178184602884C
:106330000088401C18804E48815451480278184605
:1063400001880088401C1880494842544D48017813
:10635000184602880088401C1880454881544A48E5
:1063600000880212184601880088401C18804048A6
:10637000425445480178184602880088401C18801D
:106380003B488154184600780290FCF7E3FCFCF788
:10639000D9FC64203449086030203049087001205D
:1063A0002F49087071E171E0800100208101002017
:1063B00084010020B03E0020A0010020A2010020A6
:1063C0009E010020460000209C0100209A01002030
:1063D000940100209601002098010020A4010020D3
:1063E0002C0000201C020020202020202020202023
:1063F000202020202020202020202020202020209D
:10640000000000002020B9A9B5E7B5E7D1B9C6ABB7
:10641000B8DFA3ACC7EBBCECB2E9A3A1000000005D
:10642000FC3D00202020BCD3C8C8B5E7C1F7C6ABEF
:10643000B4F3A3ACC7EBBCECB2E9A3A1000000002D
:106440002020BCD3C8C8B5E7C1F7C6ABD0A1A3AC68
:10645000C7EBBCECB2E9A3A1000000002F000020B4
:106460006F010020000C0140700100207401002029
:10647000D4430020780100207A0100207B01002015
:106480007C0100207D0100207E010020FE48007874
:10649000302842D1FD48006828B92020FA49087008
:1064A0000120FB490870FB488078012834D1FA4963
:1064B000088012E0F948F8490988415CA0F50070AD
:1064C000F54A1288805C814202D0FE20F2490880A1
:1064D000F1480088401CF0490880EF4800880B28EC
:1064E000E8DBED480088FE280EDA2021EC48FBF7B7
:1064F0001CF81021EA48FBF718F84020E249087020
:106500000120E349087005E02020DF4908700120E0
:10651000DF490870FCF716FCB7E0DB48007840283C
:10652000FAD1DC4880780128F6D1DA48007BA5282A
:106530007ED10020D8490880DA4800880212084637
:1065400001880088401CD44B1880D4484254D54858
:106550000278184601880088401C1880CF484254B1
:10656000D1480278184601880088401C1880CB4822
:106570004254A521184602880088401C1880C7484C
:1065800081540022184601880088401C1880C348A6
:106590004254C64890F86400411CC44A029082F8F4
:1065A000641019460A880988491C1980BB49885417
:1065B000BF480278184601880088401C1880B748F8
:1065C0004254BA4890F8D011184602880088401CFE
:1065D0001880B2488154B548C08B2B902B9802127A
:1065E000184601880088401C1880AC4842542B98FB
:1065F000C1B2184602880088401C1880A748815400
:10660000AA48C06C80B22B902B98021218460188C1
:106610000088401C1880A14842542B98C2B21846EA
:1066200001880088401C18809C484254184600E0AD
:1066300029E00078C01EC1B2964880F810120020F0
:10664000289003202A900AE094482A99415C2898CF
:106650000844C1B228912A98401C81B22A918E49DF
:1066600009882A988842EFDB8B490A880988491CE7
:10667000894B28981980894988541846017808461A
:106680000291FCF767FBFCF75DFB8A48D0F8D80B5A
:10669000002879D186480078A02875D084480078F1
:1066A0008028FAD0824800789028F6D08148D0F827
:1066B0000801002869D07D48B0F89C006F2864DB91
:1066C0007C48D0F804010028F4D07B48B0F8F200F0
:1066D00000285AD100217748C0F804117348C18BB3
:1066E0007448D0F80C0181424FD27248D0F80011A2
:1066F000D0F81001814248D900BF002125914FF404
:10670000FA612291494221916A48B0F8FE10D0F80E
:10671000100181423AD36748B0F8FE10B0F810017A
:10672000081A81B224916348B0F8FE10239124988E
:106730002B9024E061492B9831F910102198814267
:1067400005DD5E492B9831F9101021910BE05B4972
:106750002B9831F910102298814204DA57492B986E
:1067600031F9101022915449FE312B9831F8101054
:106770002598014425912B98401C81B22B91239997
:106780002B988842D6DB6BE076E1CCE04948B0F844
:10679000FE0000F5806081B224914648B0F81011E7
:1067A0002498401A81B224914248B0F8FE102391F7
:1067B00024982B9024E041492B9831F9101021980E
:1067C000814205DD3D492B9831F9101021910BE0F4
:1067D0003A492B9831F910102298814204DA37494E
:1067E0002B9831F9101022913349FE312B9831F852
:1067F00010102598014425912B98401C81B22B91B3
:106800002B98B0F5806FD6DB00202B9024E02B492D
:106810002B9831F910102198814205DD27492B98DA
:1068200031F9101021910BE024492B9831F9101007
:106830002298814204DA21492B9831F910102291D3
:106840001D49FE312B9831F81010259801442591EF
:106850002B98401C81B22B9123992B988842D6DB30
:106860001448D0F814012599414325911148D0F8D6
:1068700010112598B0FBF1F12591C8212598B0FBA6
:10688000F1F125911CE000002F0000207001002094
:106890006F010020C841002074010020D443002073
:1068A000000C0140760100207C0100201C02002029
:1068B0002C0000201C3200201C2200201A2B00205B
:1068C000DDE92110081A01B2219125992198884209
:1068D00029D2AFF2EC4200210846FEF797FDAFF255
:1068E000F84200210120FEF791FDFEA200210220C6
:1068F000FEF78CFDAFF2105200210320FEF786FD5B
:106900004CF2503201210846FAF724F80120FC49E4
:10691000C1F8A0000020FB4908802021FA48FAF7BE
:1069200004FE00BFFEE7F948B0F8A000002838DDFB
:10693000F748B0F8F20098BBF54890F8DE0078B35D
:10694000F248C18BB0F8A00081422ADBAFF2685256
:1069500000210846FEF75AFDAFF2745200210120D3
:10696000FEF754FDEBA200210220FEF74FFDAFF22F
:10697000885200210320FEF749FD4CF250320121DC
:106980000846F9F7E7FF0120DD49C1F8A000002023
:10699000DC4908802021DC48FAF7C7FD00BFFEE78C
:1069A000FFE7DB4890F8DE0078BBD848C08B40F2A8
:1069B000145188422ADBAFF2D05200210846FEF77C
:1069C00025FDAFF2DC5200210120FEF71FFDD8A209
:1069D00000210220FEF71AFDAFF2F452002103203D
:1069E000FEF714FD4CF2503201210846F9F7B2FFD0
:1069F0000120C349C1F8A0000020C249088020211D
:106A0000C148FAF792FD00BFFEE7FFE7C04890F8E3
:106A1000DE0088BBBD48C18BB0F8DA0000F57A70A3
:106A200081422ADBAFF2406200210846FEF7EEFC0D
:106A3000AFF24C6200210120FEF7E8FCC3A2002166
:106A40000220FEF7E3FCAFF2606200210320FEF7B4
:106A5000DDFC4CF2503201210846F9F77BFF0120A2
:106A6000A749C1F8A0000020A64908802021A64817
:106A7000FAF75BFD00BFFEE7FFE7A148D0F89400FE
:106A800028B100209E49C1F89400FBF7BBFFB6482F
:106A9000007821281BDBB4480078272817DC9848A9
:106AA000D0F8B00098B100209549C1F8B0000B2192
:106AB000FEF750FF9248D0F8AC0020B14AF2F11036
:106AC000FEF7DCFB03E04AF2A110FEF7D7FBA64875
:106AD0000078902837D1A548007838B10020A34924
:106AE00008700DF0EFF9FF20A1490870A048007868
:106AF000042817D101220A210846F9F72BFF9DA28D
:106B000000210320FEF782FC0DF01CFD01220A216A
:106B10000846F9F71FFF9EA200210320FEF776FC2E
:106B200000BFFEE79248007805284CF02783012239
:106B30000A210846F9F70EFF9CA200210320FEF768
:106B400065FC00BFFEE788480078A0285DD19EA2C2
:106B500000210846FEF75AFCA2A200210120FEF700
:106B600055FCA7A200210220FEF750FCABA2002199
:106B70000320FEF74BFC2022012100200DF034FB06
:106B80002122012108460DF02FFB222201210220A3
:106B90000DF02AFB2322012103200DF025FB01200B
:106BA0005749C1F8A0002CE071480078042828D18A
:106BB000012211460A20F9F7CDFE20200DF010FC2D
:106BC00021200DF00DFC22200DF00AFC23200DF0F9
:106BD00007FCAFF2EC7200210846FEF717FCAFF29B
:106BE000F87200210120FEF711FC93A2002102207F
:106BF000FEF70CFCAFF6100200210320FEF706FCA6
:106C000000E0D1E700BF00BFFEE7574800788028CA
:106C100066D15648007818B30020544908700CF02B
:106C200009FB8C48D0F8D40B012803D140F21F2176
:106C3000299102E040F6E20129913548D0F8D800C8
:106C40000290334890F8DC100191299ADDE90101A6
:106C5000FDF748FE002080490870FF204449087075
:106C600010212948FAF758FC10B9FCF77DFE269050
:106C70007A48007878B10020784908702448D0F824
:106C8000D00002902248D0F8C4100191DDE9010241
:106C90002699FDF71BFD36480078032821D10122F3
:106CA00011461046F9F756FEFF2031490870184882
:106CB00090F8DC00C7288CF26182154890F8DC005F
:106CC000401CC1B2124880F8DC10D0F8D800029005
:106CD0000F4890F8DC100191299ADDE90101BFE02D
:106CE0002CE1C1E0C8C8B5E7C5BCBCD3C8C8D2EC6C
:106CF000B3A3A3ACC7EBBCECB2E9A3A100000000B6
:106D0000FC3D002012000020001001401C02002069
:106D10001C2200202020C8C8B5E7C5BCB7B4BDD32D
:106D2000A3ACC7EBBCECB2E9A3A12020000000009B
:106D30002020C8C8B5E7C5BCB6CFC2B7A3ACC7EB67
:106D4000BCECB2E9A3A12020000000002020BCD3AD
:106D5000C8C8BBD8C2B7D2ECB3A3A3ACC7EBBCECDA
:106D6000B2E92020000000002C0000202E000020AE
:106D70001400002020202020D5FDD4DABBD6B8B4E2
:106D8000D6D0A3ACC7EBC9D4BAF3202000000000D2
:106D90002020D2D1BBD6B8B4B3F6B3A7C9E8D6C3C6
:106DA000A3ACC7EBD6D8C6F40000000020202020FA
:106DB0002020D2D1C8A1CFFBBBD6B8B4A3ACC7EBBF
:106DC000D6D8C6F40000000056483A2020202020E3
:106DD00020202020202020202020202020202020B3
:106DE00000000000564C3A202020202020202020A7
:106DF0002020202020202020202020200000000013
:106E000041483A202020202020202020202020201F
:106E1000202020202020202000000000414C3A208B
:106E20002020202020202020202020202020202062
:106E300020202020000000002020C7E5B3FDCDEA7F
:106E4000B3C9A3ACC7EBD6D8C6F4C9E8B1B8202003
:106E5000000000001C320020380000200400002048
:106E6000FDF740FD0CF08AB9FE48007808BB01220E
:106E700011461046F9F76EFDFF20FA490870FA48EE
:106E800090F8DC000128EDDDF74890F8DC00401EAA
:106E9000C1B2F54880F8DC10D0F8D8000290F24872
:106EA00090F8DC100191299ADDE90101FDF71AFD46
:106EB000D8E7EC480078062818D101221146104680
:106EC000F9F748FDFF20E7490870E7492698C1F81F
:106ED000D8000846D0F8D810029190F8DC10019143
:106EE000299ADDE90101FDF7FDFCBBE7DD480078EB
:106EF0000428B7D101220A210846F9F72BFDDA4808
:106F0000D0F8D8000290D84890F8DC100191DDE963
:106F10000101FDF7BCFCAFF6303200210120FEF785
:106F200075FAAFF63C3200210220FEF76FFACFA2CD
:106F300000210320FEF76AFA00BFFEE7D24800787E
:106F4000102830D1D148007830B10020CF490870E6
:106F50000CF0F8FFF9F71CFDC2480078FF28A7D015
:106F60000020CB490870CB490870CB490870CB4949
:106F70000870CB49087001220A210846F9F7EAFC9B
:106F8000FF20B84908702020BF4908700120BF4980
:106F90000870B54890F8F000BD49087008460078C0
:106FA000BD4908705EE7B8480078202876D1B74818
:106FB000007818B30020B54908700CF089F9B6487C
:106FC0000078B34908700846007800EB4000801C48
:106FD000B449085C0290AE48007800EB4000401CC9
:106FE000095CAB480191007800EB4000AD49095CB9
:106FF000012300919DE80700FEF756F999480078B3
:1070000003284CD1012211461046F9F7A3FCFF20BA
:10701000944908709E48007800EB4000801CA1490C
:10702000085C02909A48007800EB4000401C095C24
:1070300097480191007800EB40009A49095C0023D1
:1070400000919DE80700FEF72FF99148007800288D
:1070500005DD8F480078401E8D49087002E007204A
:107060008B4908708A48007800EB4000801C8D49ED
:10707000085C02908648007800EB4000401C095CE8
:1070800083480191007800EB40008649095C0123A8
:1070900000919DE80700FEF707F9E3E6CBE07148B1
:1070A0000078E8BB012211461046F9F753FCFF2196
:1070B0006C4801707648007800EB4000801C7949EC
:1070C000085C02907248007800EB4000401C095CAC
:1070D0006F480191007800EB40007249095C002381
:1070E00000919DE80700FEF7DFF86948007807285F
:1070F00005DA67480078401C6549087002E0002006
:10710000634908706248007800EB4000801C6549C4
:10711000085C02905E48007800EB4000401C00E0F4
:107120000EE0095C5A480191007800EB40005D498F
:10713000095C012300919DE80700FEF7B5F891E690
:1071400048480078072839D152480078022835DAB3
:10715000012211461046F9F7FDFBFF204149087056
:107160004B48007800EB4000801C4E49085C0290C0
:107170004748007800EB4000401C095C44480191FE
:10718000007800EB40004749095C002300919DE82E
:107190000700FEF789F830203B49087001203B4981
:1071A00008703B4800783C49087000203849087056
:1071B00038480078401C3749087053E62948007861
:1071C0000428BCD1012211460520F9F7C3FBFF209A
:1071D000244908702E4800782F4908702C480178FF
:1071E0004FF40070FDF7CAFC2948007800EB40001E
:1071F000801C2C49085C02902548007800EB400078
:10720000401C095C22480191007800EB40002549B0
:10721000095C002300919DE80700FEF745F81A4835
:1072200000781B4909780844401C17490870012060
:107230001649087016E61448007830287DD11348A6
:10724000007898B30020114908700CF059FB1348DE
:1072500000780F4908700846007800EB4000801C59
:10726000114924E0140000201C2200202020D2D14B
:10727000B1A3B4E6B5F7CAD4B2CECAFDA3ACC7EB8E
:10728000D6D8C6F4000000002C0000202E000020FC
:107290003400002038000020350000203600002097
:1072A000370000204B6401086364010814E0085CA7
:1072B0000290FB48007800EB4000401C095CF84855
:1072C0000191007800EB4000F649095C0123009130
:1072D0009DE80700FDF7E8FFF348007803284CD14C
:1072E000012211461046F9F735FBFF20EE490870E0
:1072F000EB48007800EB4000801CEA49085C0290F3
:10730000E748007800EB4000401C095CE44801912C
:10731000007800EB4000E349095C002300919DE800
:107320000700FDF7C1FFDE480078002806DDDC48D5
:107330000078401EDA49087003E02EE10520D849A4
:107340000870D748007800EB4000801CD549085CE5
:107350000290D348007800EB4000401C095CD04804
:107360000191007800EB4000CE49095C01230091B7
:107370009DE80700FDF798FF74E5CB480078E8BB6F
:10738000012211461046F9F7E5FAFF20C6490870B8
:10739000C348007800EB4000801CC249085C0290A2
:1073A000BF48007800EB4000401C095CBC480191DC
:1073B000007800EB4000BB49095C002300919DE888
:1073C0000700FDF771FFB6480078052805DAB448D4
:1073D0000078401CB249087002E00020B0490870F3
:1073E000AF48007800EB4000801CAE49085C02907A
:1073F000AB48007800EB4000401C00E00EE0095C68
:10740000A7480191007800EB4000A649095C0123E0
:1074100000919DE80700FDF747FF23E5A2480078AB
:10742000072839D1A1480078022835DA012211460F
:107430001046F9F78FFAFF209B49087098480078AA
:1074400000EB4000801C9749085C0290944800784B
:1074500000EB4000401C095C91480191007800EB72
:1074600040009049095C002300919DE80700FDF76A
:107470001BFF40208E49087001208E490870884803
:1074800000788D4908700020854908708748007889
:10749000401C86490870E5E483480078022839D109
:1074A00082480078002835DD012211461046F9F7A0
:1074B00051FAFF207C4908707948007800EB4000C1
:1074C000801C7849085C02907548007800EB400009
:1074D000401C095C72480191007800EB4000714942
:1074E000095C002300919DE80700FDF7DDFE2020E8
:1074F0006F49087001206F490870694800786E492B
:10750000087000206649087068480078401E674986
:107510000870A7E4644800780428BCD10122114611
:107520000520F9F717FAFF205F4908705C480078DA
:10753000614908705A48007800EB4000801C5949A6
:10754000085C02905648007800EB4000401C095C43
:1075500053480191007800EB40005249095C002338
:1075600000919DE80700FDF79FFE514800784C49C7
:1075700009780844401C51490870084600783328AF
:1075800003DD41204A49087003E04C48007848492F
:10759000087001204749087064E445480078402895
:1075A00026D14448007820B10020424908700CF0F0
:1075B00015F83D4800780228ABD13C4800780028F7
:1075C000A7DD012211461046F9F7C4F9FF2036491C
:1075D00008703020364908700120364908700020B4
:1075E0002F49087031480078401E3049087039E44E
:1075F0002F480078212852D12E48007890B10020E1
:107600002C4908700BF09CFF01212D48C0F808118F
:107610000021C0F8001100202A4981F8D001012082
:1076200081F8D1012048007805281CD10020254987
:1076300081F8480001220F210846F9F78BF9FF2055
:1076400019490870282200210846F9F755FA002147
:107650001B48C0F80811C0F8001120201449087018
:10766000012014490870174890F8D0010C287DD2E9
:10767000DFE800F00656F1EFEEEDECEBEAE97CA076
:107680001048008E642821DC01200E4981F8D001C9
:1076900081F8D10100200C49C1F8A0002DE0F9E3E8
:1076A000340000206364010814000020380000202A
:1076B0002C0000202E000020360000202D0000208D
:1076C0001C3200201C020020FC3D0020FE4890F8E7
:1076D000D10168B1012211460520F9F73BF9FBA25F
:1076E00000210320FDF792FE0020F74981F8D10127
:1076F000282200210846F9F7FFF9F34890F84900DD
:1077000068B10020F04981F849000846C08B024664
:107710000521029001200DF075F9FDF791FEE1E3DE
:10772000E94890F8490068B10020E74981F849002C
:107730000846C08B02460521029001200DF062F937
:10774000FDF77EFEE04890F8D10140B101221146DC
:107750001046F9F7FFF80020DB4981F8D10101223A
:1077600011461046F9F7F6F8FF2000E0B9E3DE49CC
:1077700008700B20D44981F8D001012081F8D10193
:1077800028224FF4FA71F9F7B7F9D8A20021084678
:10779000FDF73CFEDCA200210320FDF737FE0020B0
:1077A000C94981F8490081F84800C8640846008E3C
:1077B000086497E3C448008EB0F5FA7F1BDAC2482C
:1077C000C06CC149096CC1F5FA7148434FF4E161DD
:1077D000B0FBF1F0BC49096C0844BB49098E8842F2
:1077E00004D20120CF49C1F8A0000FE00021CD480C
:1077F000C0F8A0100AE00220B34981F8D0010120AE
:1078000081F8D1010020C749C1F8A000AE4890F826
:107810004900B8B10020AC4981F849000846C08B46
:1078200002460521029001200DF0ECF8FDF708FE5C
:10783000A548C16C0A460291052102200DF0F2F91B
:10784000FDF744FF4EE3E1E29DE261E2FEE1B3E1D8
:10785000C4E03FE0FFE79C48008EB0F5FA7F1CDBF8
:1078600002220A210846F9F775F8A0A2002108466D
:10787000FDF7CCFDACA200210220FDF7C7FD0320DF
:10788000914981F8D001012081F8D101002081F8CF
:10789000490081F84800C8641BE08B4890F8490013
:1078A000B8B10020884981F849000846C08B0246DB
:1078B0000521029001200DF0A5F8FDF7C1FD8248D9
:1078C000C16C0A460291052102200DF0ABF9FDF7CB
:1078D000FDFE07E37C4890F84900C8B300207A49D0
:1078E00081F849000846C08BB0F5FA7F13DB0846E3
:1078F000C08BA0F5FA70C117029000EB9170801058
:1079000000F5FA7002460521019001200DF07AF889
:10791000FDF796FD12E06C48C08BC0F5FA70C117F8
:10792000029000EB91708010C0F5FA710A46019147
:10793000052101200DF066F8FDF782FD6248C06C5C
:1079400002460521029002200DF06CF9FDF7BEFE03
:107950005D48C16C40F2EA60814204D101220A21F3
:107960000846F8F7F7FF5848C06CB0F5E16F34D31C
:107970005EA200210846FDF749FD6BA2002102200E
:10798000FDF744FD0420504981F8D001012081F821
:10799000D1010846C18B0184B0F87A104184B0F857
:1079A00078004949C8650846C06DC0EB00108000EA
:1079B000C8650846C06D1E380866002081F8490079
:1079C0000021414880F8481000203F49C86428221F
:1079D00040F22F310120F9F78FF883E23A48018E07
:1079E00040F22F3081421FDB40A200210846FDF704
:1079F0000DFD4DA200210220FDF708FD05203249B2
:107A000081F8D001012081F8D101002081F84900DE
:107A100081F84800C8644349C1F8A00002220A2145
:107A20000846F8F797FFC6E02748008E40F22A3153
:107A3000884226DB2C480078042822D1FF202A49DE
:107A400008702AA200210846FDF7E0FC36A20021BA
:107A50000220FDF7DBFC05201B4981F8D001012045
:107A600081F8D101002081F8490081F84800C864FC
:107A70002C49C1F8A00003220A210846F8F76AFF42
:107A800099E0114890F84900B8B100200E4981F8FA
:107A900049000846C08B02460521029001200CF0E7
:107AA000B1FFFDF7CDFC0848C16C0A4602910521E3
:107AB00002200DF0B7F8FDF709FE0348008E0249D9
:107AC000498C88426DDA3DE01C020020CCE1CABE40
:107AD000A3BAB5C8B4FDC2AFCEC2CFC2BDB52E2EBB
:107AE0002E2020200000000014000020C2FDBBD288
:107AF000D7B4CCACA3BAB2E2CAD4D6D02E2E2E20A4
:107B00002020202000000000CCE1CABEA3BAC7EBB1
:107B1000B4F2BFAAD1CCB4D1B2A2C1F4C3C5B7EC00
:107B200000000000FC3D0020BDF8B3CCCAB1BCE4AD
:107B3000A3BA30302D30302D3030202020202020AE
:107B400000000000FE48008EFD49098C884222DDBD
:107B5000FB48C16C2791B0F87C10279841432791CE
:107B60003C212798B0FBF1F12791F548018C27982B
:107B700001442791F248018E279880B2814204DDAA
:107B80000120F049C1F8A00015E04FF6FF70ED4963
:107B9000C1F8A0000FE04FF6FF70EA49C1F8A0005D
:107BA00009E0E748008E40F22F31884203DA0020D6
:107BB000E449C1F8A00095E1E14890F84900B8B166
:107BC0000020DF4981F849000846C08B02460521A4
:107BD000029001200CF016FFFDF732FCD848C16C72
:107BE0000A460291052102200DF01CF8FDF76EFDFA
:107BF000D348C06CD249096E884204D10F220A21B1
:107C00000846F8F7A7FECE48C06CCD49C96D88423A
:107C10001BD3CDA200210846FDF7F8FBD1A200211D
:107C20000320FDF7F3FB0620C54981F8D0010120B0
:107C300081F8D101002081F8490081F84800C8642A
:107C4000282200210846F8F757FF4BE1BC4890F87E
:107C5000490068B10020BA4981F849000846C08B44
:107C600002460521029001200CF0CCFEFDF7E8FB56
:107C7000C348007804282DD1012211461046F8F798
:107C800069FEFF20BE4908700720AD4981F8D00188
:107C9000012081F8D101BBA200210846FDF7B6FB07
:107CA000AFF27C1200210220FDF7B0FBAFF2A81268
:107CB00000210320FDF7AAFB0020A14981F849001B
:107CC00081F84800C864282240F22F310120F8F7DB
:107CD00013FF1CE0AA480078052818D1012211469C
:107CE0001046F8F737FEFF20A5490870282200212A
:107CF0000846F8F701FF0021A948C0F80811C0F8AC
:107D000000112020A74908700120A7490870E9E068
:107D10008B4890F84900B8B10020894981F84900A2
:107D20000846C08B02460521029001200CF06AFE35
:107D3000FDF786FB8248C16C0A46029105210220AC
:107D40000CF070FFFDF7C2FC7D48008E40F22F3131
:107D5000884217DB8BA200210846FDF757FBAFF2E4
:107D6000382200210220FDF751FB0820744981F8D8
:107D7000D001012081F8D101002081F8490081F86B
:107D80004800C864AEE06E4890F84900B8B10020E1
:107D90006B4981F849000846C08B024605210290D4
:107DA00001200CF02FFEFDF74BFB6548C16C0A4625
:107DB0000291052102200CF035FFFDF787FC604899
:107DC000C06C40F29241884204D10F220A21084639
:107DD000F8F7C0FD5A48C06CB0F5966F15D373A282
:107DE00000210846FDF712FB5EA200210320FDF7EB
:107DF0000DFB0920524981F8D001012081F8D10101
:107E0000282264210020F8F777FE6BE04C4890F8B8
:107E1000490068B100204A4981F849000846C08BF2
:107E200002460521029001200CF0ECFDFDF708FB55
:107E30005348007804282ED1012211461046F8F745
:107E400089FDFF204E49087007203D4981F8D00187
:107E5000012081F8D1014BA200210846FDF7D6FA96
:107E6000AFF23C3200210220FDF7D0FAAFF26832C7
:107E700000210320FDF7CAFA0020314981F84900AA
:107E800081F84800C864282240F22F310120F8F719
:107E900033FE25E028E03A480078052820D1012269
:107EA00011461046F8F756FDFF2035490870282284
:107EB00000210846F8F720FE00213948C0F80811D3
:107EC000C0F8001120203749087001203649087099
:107ED00000203D49087000BF3B480078BE28FBDB0E
:107EE00000E000BF0BF04AB92E48007822286DD17F
:107EF0002D480078E0B100202B4908700BF084FA7F
:107F000000201049C1F8A0000D4981F8490081F80E
:107F10004800C86401212248C0F808110021C0F8B7
:107F200000110020064981F8D001012081F8D1011B
:107F3000034890F8D0010C2873D053DC022846E0A7
:107F40001C020020FC3D0020C2FDBBD2D7B4CCAC4B
:107F5000A3BACAD4D1E9CDEAB3C920202020202079
:107F600000000000CCE1CABEA3BAB0B4C8B7C8CF05
:107F7000BCFCBCECB2E9D7C6C9D52020000000008B
:107F800014000020C2FDBBD2D7B4CCACA3BAD7C674
:107F9000C9D5D6D02E2E2E20202020200000000073
:107FA0001C3200202C0000202E000020C2FDBBD27D
:107FB000D7B4CCACA3BAD7C6C9D5CDEAB3C92020B3
:107FC000202020200000000005000020FEE37DD0DE
:107FD00003DCA0B101287AD149E00A2878D00B2827
:107FE000F9D178E3112874D004DC0E2872D00F2860
:107FF000F1D1ECE328286ED07128ECD128E32822B7
:1080000040F252310120F8F777FDFAA2002108462C
:10801000FDF7FCF9AFF2F04200210220FDF7F6F97E
:1080200000E0FDE3FAA200210320FDF7EFF90120B3
:10803000FE4981F8D0010846C08B08840846B0F894
:10804000800048840846B0F87E0048650846406DC8
:10805000C0EB0010800048650846406D1E388865FA
:10806000002081F8490081F84800C864B8E2EF4870
:1080700090F84900B8B10020EC4981F84900084661
:10808000C08B02460521029001200CF0BBFCFDF7DD
:10809000D7F9E648C16C0A460291052102200CF08E
:1080A000C1FDFDF713FBE148008EE049498C884291
:1080B00035DADE48008EDD49098C884229DDDB484F
:1080C000C16C2791B0F88210279805E071E0EDE3CC
:1080D000B6E086E250E312E1414327913C21279824
:1080E000B0FBF1F12791D148018C279801442791E9
:1080F000CE48018E279880B2814204DD0120CC4910
:10810000C1F8A00014E04FF6FF70C949C1F8A00003
:108110000EE04FF6FF70C649C1F8A00008E0C34862
:10812000008EB0F5547F03DA0020C149C1F8A000E9
:10813000BE48008EB0F5547F17DBBEA20021084672
:10814000FDF764F9C2A200210320FDF75FF90020CA
:10815000B749C1F8A0000220B44981F8D0019622A5
:108160000A210846F8F7F6FB22E0B048008EB0F589
:10817000537F1DDDBD480078042819D1FF20BB497D
:108180000870ACA200210846FDF740F9B0A200211A
:108190000320FDF73BF90020A549C1F8A00002200B
:1081A000A24981F8D00196220A210846F8F7D2FBAD
:1081B000E8E39E4890F84900B8B100209B4981F857
:1081C00049000846C08B02460521029001200CF0B0
:1081D00019FCFDF735F99548C16C0A460291052155
:1081E00002200CF01FFDFDF771FAA0480078FF286F
:1081F00004D000220A210846F8F7ACFB9B4800781F
:1082000004281CD1012211461046F8F7A3FBFF20D9
:1082100096490870AFF2F06200210220FDF7F6F8EF
:1082200093A200210320FDF7F1F80A207F4981F88D
:10823000D001002081F8490081F84800C864A1E31A
:108240007A4890F84900B8B10020784981F849008F
:108250000846C08B02460521029001200CF0D2FB9B
:10826000FDF7EEF87148C16C0A4602910521022023
:108270000CF0D8FCFDF72AFA7C48007804283DD1A0
:10828000012211461046F8F765FBFF207749087078
:108290007EA200210846FDF7B9F8AFF27472002102
:1082A0000220FDF7B3F85AA200210320FDF7AEF833
:1082B00011205E4981F8D001002081F8490081F841
:1082C0004800C864282081F8D001002081F84800C7
:1082D00081F84900C86440F2A230A1F8280D282294
:1082E00040F22F310120F8F707FC002050490866C2
:1082F0000120C1F8A4000020C1F8A80042E34B48C7
:1083000090F84900F0B30020484981F84900084638
:10831000B0F8280D098E884208DD4448008E434994
:10832000A1F8280D0846C06CA1F82A0D3F48B0F806
:10833000280D3E49098E88425ADA3C48008E40F2A8
:108340001B3188423EDA3948008E3849B1F8281D81
:10835000401A00EB800040003449B1F8281D40F27B
:108360001B32511A90FBF1F03048008E2F48018EDD
:10837000B0F8280D081A00EB800040002B49B1F836
:10838000281D00E02CE1511A90FBF1F02749098EDD
:1083900008442649A1F844000846B0F844000246C3
:1083A0000521029001200CF02DFBFDF749F81F4834
:1083B000C16C0A460291052102200CF033FCFDF746
:1083C00085F99BE01948008E00F22F301748008E87
:1083D00000F22F30029000EBD070C0F34F00134931
:1083E000A1F844000846B0F84400024605215BE0CD
:1083F0006BE00000BEADB5E4BFECBBD2A3BAC9FDD3
:10840000CEC22E2E2E202020202020200000000072
:10841000CCE1CABEA3BAC7EBB4F2BFAAD1CCB4D1E7
:108420002020202020202020000000001C0200200E
:10843000FC3D0020BEADB5E4BFECBBD2A3BABAE3AD
:10844000CEC22E2E2E202020202020200000000032
:10845000CCE1CABEA3BAB0B4C8B7C8CFBCFCBFAAEF
:10846000CABCCBCDD1F920200000000014000020B0
:10847000CCE1CABEA3BACBCDD1F9CDEAB3C9BAF328
:10848000B0B4C8B7C8CFBCFC00000000BEADB5E4B6
:10849000BFECBBD2A3BAB2E2CAD4D6D02E2E2E20C5
:1084A0002020202000000000029001200CF0AAFAF9
:1084B000FCF7C6FFFE48C06C024605210290022070
:1084C0000CF0B0FBFDF702F918E0F948C08BF84951
:1084D000A1F844000846C08B024605210290012005
:1084E0000CF090FAFCF7ACFFF148C16C0A4602911F
:1084F000052102200CF096FBFDF7E8F8ED48D0F8D6
:10850000A40008B3EA48C16CB0F8720081420AD2F4
:108510000120E849C1F8A0000020C1F8980001201E
:10852000C1F8A80049E0E248B0F8280DE049098EFA
:1085300088420ADBDE48B0F86C00801CDD49C1F8D7
:10854000A0000220C1F8A80037E0D948B0F84410D4
:10855000B0F8740081420ADAD548B0F86C00801C8B
:10856000D449C1F8A0000320C1F8A80025E0D048F4
:10857000B0F84410B0F8760081420ADA0120CD4903
:10858000C1F8A0000020C1F898000420C1F8A8009C
:1085900013E00020C749C1F8A400C1F8A000C1F849
:1085A0009000282240F22F310120F8F7A5FA002090
:1085B000C04908660520C1F8A800BD48008EB0F586
:1085C0004B7F0DDD282240F22F310120F8F794FA7D
:1085D0001120B74981F8D0010020B649C1F8A000A8
:1085E000D0E1B348008EB0F54B7F14DD7120B04967
:1085F00081F8D001AFF26C1200210846FCF706FFAB
:108600000020AB4981F8490081F84800C864012086
:1086100081F8D1011BE0A64890F84900B8B10020CC
:10862000A34981F849000846C08B02460521029003
:1086300001200CF0E7F9FCF703FF9D48C16C0A46E6
:108640000291052102200CF0EDFAFDF73FF899E1C7
:10865000974890F84900B8B10020954981F8490041
:108660000846C08B02460521029001200CF0CAF991
:10867000FCF7E6FE8E48C16C0A46029105210220F5
:108680000CF0D0FAFDF722F88948C06C8849896D52
:10869000884204D10F220A210846F8F75BF9844882
:1086A000C06C8349496D884214D383A20021022003
:1086B000FCF7ACFEAFF2547200210320FCF7A6FEDB
:1086C0000B207B4981F8D001002081F8490081F816
:1086D0004800C86456E1764890F8490068B1002027
:1086E000734981F849000846C08B02460521029073
:1086F00001200CF087F9FCF7A3FE764800780428E7
:1087000027D1012211461046F8F724F9FF207149BC
:1087100008700E20664981F8D001012081F8D1014E
:10872000AFF2982200210846FCF770FEAFF608422F
:1087300000210220FCF76AFE67A200210320FCF75B
:1087400065FE00205A4981F8490081F84800C86454
:1087500011E06048007805280DD1012211460F2054
:10876000F8F7F8F8FF205B4908702220614908708B
:1087700001206149087005E14D4890F84900B8B101
:1087800000204B4981F849000846C08B024605216C
:10879000029001200CF036F9FCF752FE4448C16CFF
:1087A0000A460291052102200CF03CFAFCF78EFFEC
:1087B0003F48008E40F22F3188421CDB0F203C499D
:1087C00081F8D001012081F8D10101E0DCE013E063
:1087D000AFF2483200210846FCF718FEAFF6B84267
:1087E00000210220FCF712FE0020314981F84900E7
:1087F00081F84800C864C5E02D4890F84900C0B130
:1088000000212B4880F84910C08B024605210290B8
:1088100001200CF0F7F8FCF713FE2548C16C00E0CE
:108820002DE00A460291052102200CF0FBF9FCF72D
:108830004DFF1F48C06C40F29241884204D10F2284
:108840000A210846F8F786F81948C06CB0F5966F0B
:1088500014D319A200210220FCF7D8FDAFF6FC02C8
:1088600000210320FCF7D2FD0C20114981F8D00132
:10887000002081F8490081F84800C86482E00C4873
:1088800090F8490068B10020094981F8490008467C
:10889000C08B02460521029001200CF0B3F8FCF7D2
:1088A000CFFD0C480078042850D127E069E0000093
:1088B0001C020020FC3D0020CCE1CABEA3BAB0B42B
:1088C000CDCBB3F6BCFCBCCCD0F8CAD4D1E92020C7
:1088D0000000000014000020CCE1CABEA3BA202092
:1088E0002020202020202020202020202020202088
:1088F000000000002C0000202E0000200122114664
:108900001046F8F727F8FF20FE4908700E20FE49B0
:1089100081F8D001012081F8D101FCA20021084694
:10892000FCF774FDAFF6006200210220FCF76EFD3B
:10893000AFF25C0200210320FCF768FD0020F24941
:1089400081F8490081F84800C86419E0ED480078D2
:10895000052815D1012211461046F7F7FBFFFF202D
:10896000E84908702220F04908700120EF4908709A
:108970000020EF49087000BFED480078BE28FBDBFF
:1089800000E000BF0AF0FABBE748007827287CD156
:10899000E6480078E0B10020E44908700AF082FD62
:1089A0000020E449C1F8A000D74981F8490081F8C6
:1089B0004800C8640121E048C0F808110021C0F84F
:1089C00000110020D04981F8D001012081F8D101A7
:1089D000CD4890F8D00113287ED005DC58B102288C
:1089E0007BD010287AD151E0142878D0152877D080
:1089F0007128F7D1A8E2C448008EB0F5FA7F1FDBDA
:108A0000282200210846F8F777F8CCA20021084672
:108A1000FCF7FCFCAFF6F06200210220FCF7F6FC4C
:108A2000CDA200210320FCF7F1FC1020B64981F80B
:108A3000D001002081F8490081F84800C86423E093
:108A4000282240F22F310120F8F756F8C9A2002160
:108A50000846FCF7DBFCAFF6307200210220FCF781
:108A6000D5FCCBA200210320FCF7D0FC1320A649A3
:108A700081F8D001FF20A34908700020A24981F8A5
:108A8000490081F84800C864A5E2A5E29E48008E2E
:108A9000B0F5FA7F28DA032205210846F7F75AFFD6
:108AA000B4A200210846FCF7B1FCAFF684720021A5
:108AB0000220FCF7ABFCB6A200210320FCF7A6FCC9
:108AC0001320914981F8D001FF208E4908700020C1
:108AD0008D4981F8490004E067E0B0E17AE2DEE028
:108AE0001FE081F84800C864874890F84900B8B191
:108AF0000020854981F849000846C08B02460521BF
:108B0000029001200BF07EFFFCF79AFC7E48C16CBE
:108B10000A460291052102200CF084F8FCF7D6FDEC
:108B200059E27948008EB0F5FA7F21DA0322052157
:108B30000846F7F70FFF8FA200210846FCF766FCF6
:108B40009A4A00210220FCF761FC91A20021032037
:108B5000FCF75CFC13206C4981F8D001FF206949C7
:108B600008700020684981F8490081F84800C8640D
:108B7000654890F84900B8B10020634981F8490080
:108B80000846C08B02460521029001200BF03AFFF7
:108B9000FCF756FC5C48C16C0A4602910521022094
:108BA0000CF040F8FCF792FD15E25748008EB0F546
:108BB000FA7F1ADB032205210846F7F7CBFE2822AD
:108BC0004FF4FA710120F7F797FF00204E4981F822
:108BD000490081F84800C8644FF4E160086514203A
:108BE00081F8D001FF2047490870464800780428E2
:108BF00038D1012211461046F7F7ACFEFF2041495B
:108C00000870282240F22F310120F7F775FF68A283
:108C100000210846FCF7FAFB644A00210220FCF719
:108C2000F5FB624A203A00210320FCF7EFFB02200B
:108C3000354981F8D0010846C08B08840846B0F851
:108C4000980048840846B0F8960048650846406D8C
:108C5000C0EB001080004865002081F8490081F8D1
:108C60004800C864284890F84900B8B10020264957
:108C700081F849000846C08B024605210290012078
:108C80000BF0C0FEFCF7DCFB1F48C16C0A460291EA
:108C9000052102200BF0C6FFFCF718FD9BE11A48E6
:108CA00090F84900B8B10020174981F849000846FA
:108CB000C08B02460521029001200BF0A3FEFCF7B9
:108CC000BFFB1148C16C0A460291052102200BF03E
:108CD000A9FFFCF7FBFC0C48006D48B94FF0FF30D2
:108CE0000949086528224FF4FA710020F7F704FFBC
:108CF00004480078042869D1012211461046F7F78C
:108D000029FE64E0140000201C020020BEADB5E482
:108D1000BFECBBD2A3BAD7C6C9D5D6D02E2E2E2033
:108D200020202020000000002C0000202E00002029
:108D300005000020FC3D00201C320020BFECCBD9F8
:108D4000BFECBBD2A3BABDB5CEC2D6D02E2E2E203C
:108D50002020202000000000CCE1CABEA3BAC7EB4F
:108D6000B4F2BFAAC2AFC3C52020202020202020FB
:108D700000000000BFECCBD9BFECBBD2A3BAC7EB5D
:108D8000B7C5D1F92E2E2E20202020200000000073
:108D9000CCE1CABEA3BAB7C5D1F9BAF3C7EBB0B438
:108DA000C8B7C8CFBCFC202000000000287B00080A
:108DB000BFECCBD9BFECBBD2A3BAC9FDCEC2D6D0D3
:108DC0002E2E2E20202020200000000036E0FF2044
:108DD000FE490870282240F22F310120F7F78CFE5F
:108DE000AFF2340200210846FCF710FBF84A0021DC
:108DF0000220FCF70BFBF64A203A00210320FCF787
:108E000005FB0220F34981F8D0010846C08B088495
:108E10000846B0F8980048840846B0F896004865BF
:108E20000846406DC0EB001080004865002081F8C6
:108E3000490081F848000021E648C164CBE0E548DC
:108E400090F84900B8B10020E24981F8490008468D
:108E5000C08B02460521029001200BF0D3FDFCF7E8
:108E6000EFFADC48C16C0A460291052102200BF0A2
:108E7000D9FEFCF72BFCD748008ED649498C884296
:108E80002EDAD448008ED349098C884222DDD1489D
:108E9000C16C2791B0F89A102798414327913C2143
:108EA0002798B0FBF1F12791CA48018C279801441B
:108EB0002791C848018E279880B2814204DD0120A5
:108EC000C549C1F8A00015E04FF6FF70C249C1F8CE
:108ED000A0000FE04FF6FF70BF49C1F8A00009E005
:108EE000BC48008E40F22E31884203DA0020BA4995
:108EF000C1F8A000B748008E40F22D31884222DD33
:108F00007120B44981F8D001012205210846F7F704
:108F100021FDB2A200210846FCF778FAAC4A0021F4
:108F20000220FCF773FAAA4A203A00210320FCF73A
:108F30006DFA0020A74981F8490081F84800C8640B
:108F4000A549C1F8A00046E0A24890F84900B8B190
:108F50000020A04981F849000846C08B024605213F
:108F6000029001200BF04EFDFCF76AFA9948C16CA3
:108F70000A460291052102200BF054FEFCF7A6FBE5
:108F80009448C06C9349496D884222D3062205213A
:108F90000846F7F7DFFC98A200210846FCF736FAEE
:108FA0008B4A00210220FCF731FA9AA2002103200B
:108FB000FCF72CFA282200210846F7F79DFD152022
:108FC000844981F8D001002081F8490081F84800E7
:108FD000C86400E000BFD5E49548007823287DD11F
:108FE00094480078C8B10020924908700AF0BEF990
:108FF0000020784981F8480081F84900C8640121BF
:109000008D48C0F808110021C0F8001100207149F6
:1090100081F8D001012081F8D1016E4890F8D0018B
:1090200009287DD005DC58B102287AD0072879D1EB
:1090300018E30A2863D0102875D01328F7D128E048
:109040006448B0F884002822014602900120F7F716
:1090500053FD00206049086678A200210846FCF70D
:10906000D5F95B4A00210220FCF7D0F97AA2002151
:109070000320FCF7CBF91320564981F8D0010020DA
:1090800081F84900C8644FF6FF705349C1F8A00049
:109090005EE3504890F84900B8B100204D4981F88E
:1090A00049000846C08B02460521029001200BF0C2
:1090B000A9FCFCF7C5F94748C16C0A460291052195
:1090C00002200BF0AFFDFCF701FB4248018EB0F827
:1090D0008600814212DB00203F4900E039E3C1F8FD
:1090E000A000FF20394908700A203A4981F8D001D0
:1090F000002081F8480081F84900C86428E3354819
:1091000090F84900E0B10020324981F84900084652
:10911000C08B02460521029001200BF073FC03E096
:1091200003E339E013E307E1FCF78AF92948C16C4E
:109130000A460291052102200BF074FDFCF7C6FAE5
:109140002448018EB0F88800814224DB00202249A7
:10915000C1F8A00047A200210846FCF757F90A22EF
:1091600005210846F7F7F6FBFF201849087048A2CA
:1091700000210320FCF74AF9154A00210220FCF7E0
:1091800045F90220134981F8D001002081F84800F8
:1091900081F84900C864DBE20E4890F8490068B1E4
:1091A00000200C4981F849000846C08B0246052181
:1091B000029001200BF026FCFCF742F903480078EE
:1091C000042873D101221146104670E014000020DB
:1091D000287B00081C020020FC3D0020BFECCBD9FE
:1091E000BFECBBD2A3BABAE3CEC2D6D02E2E2E206D
:1091F0002020202000000000BFECCBD9BFECBBD268
:10920000A3BACAD4D1E9CDEAB3C9202020202020B6
:1092100000000000CCE1CABEA3BACAD4D1E9BDE1C6
:10922000CAF8A3ACC7EBC8A1D1F920200000000008
:109230002C0000202E0000201C320020BBD3B7A23F
:10924000D7B4CCACA3BAC9FDCEC2202020202020A8
:109250002020202000000000CCE1CABEA3BAC7EB4A
:10926000B9D8B1D5D1CCB4D12020202020202020C5
:1092700000000000BBD3B7A2D7B4CCACA3BABAE30A
:10928000CEC220202020202020202020000000000E
:10929000CCE1CABEA3BAB7C5D1F9BAF3B0B4C8B766
:1092A000C8CFBCFC202020200000000043E0F7F7DE
:1092B00051FBFF20F8490870F8A200210846FCF78E
:1092C000A5F8FD4A00210220FCF7A0F8AFF27802D1
:1092D00000210320FCF79AF81020F84981F8D0010A
:1092E000002081F8480081F84900C86440F2A230AB
:1092F000A1F8280D28224FF461710120F7F7FCFB3B
:109300000020EF4908660120C1F8A4000020C1F840
:10931000A8000846D0F8A8000246082102900020C4
:109320000BF070FBE648D0F8A0100A4602910A2123
:1093300000200BF067FB0BE2E04890F84900E8B32F
:109340000020DE4981F849000846B0F8280D098E52
:10935000884208DDD948008ED849A1F8280D084672
:10936000C06CA1F82A0DD548B0F8280DD349098E54
:1093700088426ADAD148008EB0F55C7F3FDACF4888
:10938000008ECE49B1F8281D401A00EB8000400045
:10939000CA49B1F8281DC1F55C7190FBF1F0C748CE
:1093A000008EC648008EC549B1F8281D401A00EB52
:1093B00080004000C149B1F8281D00E051E1C1F52D
:1093C0005C7190FBF1F0BD49098E0844BB49A1F8DE
:1093D00044000846B0F844000246052102900120EE
:1093E0000BF010FBFCF72CF8B448C16C0A46029154
:1093F000052102200BF016FCFCF768F93EE0AF48AF
:10940000008E00F56170AD48008E00F5617002902D
:1094100000EBD070C0F34F00A849A1F84400084603
:10942000B0F8440002460521029001200BF0EAFA50
:10943000FCF706F8A148C06C024605210290022004
:109440000BF0F0FBFCF742F918E09C48C08B9B49FD
:10945000A1F844000846C08B024605210290012075
:109460000BF0D0FAFBF7ECFF9448C16C0A4602916E
:10947000052102200BF0D6FBFCF728F99048D0F824
:10948000A40008B38D48C16CB0F8900081421CD292
:1094900001208B49C1F8A0000020C1F898000120EC
:1094A000C1F8A8000846D0F8A8000246072102909B
:1094B00000200BF0A7FA8248D0F8A0100A460291CB
:1094C000092100200BF09EFA94E07C48B0F8280DAA
:1094D0007A49098E88421CDB7848B0F86C00801C01
:1094E0007749C1F8A0000220C1F8A8000846D0F8CA
:1094F000A80002460721029000200BF083FA704872
:10950000D0F8A0100A460291092100200BF07AFA47
:1095100070E06A48B0F84410B0F8920081421CDA5A
:109520006648B0F86C00801C6549C1F8A0000320B3
:10953000C1F8A8000846D0F8A8000246072102900A
:1095400000200BF05FFA5E48D0F8A0100A460291A6
:10955000092100200BF056FA4CE05848B0F84410AE
:10956000B0F8940081421CDA01205549C1F8A000EE
:109570000020C1F898000420C1F8A8000846D0F8DF
:10958000A80002460721029000200BF03BFA4C484D
:10959000D0F8A0100A460291092100200BF032FAFF
:1095A00028E000204649C1F8A400C1F8A000C1F895
:1095B00090004248B0F86E00282201460290012037
:1095C000F7F79AFA00203E4908660520C1F8A8007E
:1095D0000846D0F8A8100A460291072100200BF097
:1095E00011FA3748D0F8A0100A460291092100204C
:1095F0000BF008FA3148C06CB42805D1012211469D
:109600001046F7F7A7F92CE02C48C06CB0F5C37FE3
:1096100005D10F220A210846F7F79CF921E02748D7
:10962000C06CB0F5D27F1CD396220A210846F7F70A
:1096300091F924A200210846FBF7E8FE28A20021A8
:109640000320FBF7E3FE00201D49C1F8A0002822FB
:109650004FF461710120F7F74FFA0720174981F89D
:10966000D00175E0154890F84900A0B100201349D9
:1096700081F849000846C08B02460521029001206E
:109680000BF0C0F9FBF7DCFE0C48C16C0A460291F6
:109690000521022032E035E014000020BBD3B7A240
:1096A000D7B4CCACA3BAB2E2CAD4D6D02E2E2E20D8
:1096B0002020202000000000287B00081C02002041
:1096C000FC3D0020BBD3B7A2D7B4CCACA3BACAD45C
:1096D000D1E9CDEAB3C920202020202000000000DD
:1096E000CCE1CABEA3BAB0B4C8B7C8CFBCFCBCCC2E
:1096F000D0F8BBD3B7A2B7D6000000000BF092FAA7
:10970000FBF7E4FFFE48007804280DD101220A216E
:109710001420F7F71FF9FF20F94908702320F949B1
:1097200008700120F849087012E02822002108463C
:10973000F7F7E2F90021F548C0F80811C0F8001168
:109740002020F04908700120EF49087000E000BFB8
:1097500041E4EC48007824287ED1EB480078D0B171
:109760000020E94908700AF061FC0020E849C1F8CE
:10977000A000E84981F8480081F84900C86408461B
:10978000C08B8883002081F8D001012081F8D101AD
:10979000002081F8D801DA48007805281CD1012280
:1097A0000A210846F7F7D6F8FF20D5490870282285
:1097B00000210846F7F7A0F90020D549C1F8A0001C
:1097C0000021D248C0F80811C0F800112020CD496E
:1097D00008700120CC490870CE4890F8D0010728C5
:1097E00072D2DFE800F004F8F7F6F5F4F300042095
:1097F000C84981F8D001012081F8D101084690F8CC
:10980000D80100EB4001C348DE3030F821002822A7
:10981000014602900120F7F76FF90020BC49C1F81A
:10982000A0000621FCF796F8BA4890F8D8014AF251
:10983000D921084481B208460291FBF71FFDB548C3
:10984000C18B90F8D80100EB4002B248DE3030F80E
:109850002200814239DA00E0FAE3AFA200210320BE
:10986000FBF7D4FDAB48C18B018490F8D80100EB25
:109870004001A848DE3030F82110DE3890F8D801D9
:1098800000EB4002A348DE3000EB82004089081A5A
:10989000A0494884084690F8D80100EB40019D4853
:1098A000DE3000EB810040889A4948650846406DEB
:1098B000C0EB0010810097484165406D1E38954906
:1098C00088650020488338E0FDE39AA20021032048
:1098D000FBF79CFD8F48C08B8E490884084690F8A2
:1098E000D80100EB40018B48DE3030F82110DE3823
:1098F00090F8D80100EB40028648DE3000EB820091
:109900004089084483494884084690F8D80100EB10
:1099100040018048DE3000EB810040887D49486589
:109920000846406DC0EB001081007A484165406DEB
:109930001E387849886501204883764890F8D80118
:1099400000EB40017348DE3030F821000246092167
:10995000029001200BF056F82020FBF78FFC20200E
:10996000FBF78CFC6B4890F8D80100EB400169488C
:10997000DE3000EB81004088C0EB001081006548BC
:10998000C0F8D411D0F8D4110A460291082102205F
:109990000BF048F900215F4880F8491080F8481022
:1099A00000205C49C8640846408BD0B9084690F84E
:1099B000D80100EB40015748DE3000EB8100808881
:1099C00050B90120534981F8D0010EE063E1D5E19F
:1099D0000CE03EE35BE2D5E004214E4880F8D01174
:1099E00003E006204B4981F8D00177E3494890F81D
:1099F0004900E8B30020474981F849004348D0F8BE
:109A0000DC0B38B10846C08B0246082102900020CA
:109A10000AF0F8FF0BF0EAF8024603210290012059
:109A20000AF0F0FF2020FBF729FC2020FBF726FCA2
:109A30002020FBF723FC2020FBF720FC4AF2AF306C
:109A4000FBF71CFC2020FBF719FC2020FBF716FC81
:109A5000304890F8D80100EB40012E48DE3030F855
:109A600021100A460291092101200AF0CBFF00E0F3
:109A70001AE02020FBF702FC2020FBF7FFFB254823
:109A8000C16C0A460291032102200BF0CBF84AF286
:109A9000AF30FBF7F3FB1F48D0F8D4110A46029110
:109AA000082102200BF0BEF81A48C08B1949498CD6
:109AB00088425EDA1748C08B1649098C884252DD0D
:109AC0001448C16C279190F8D80100EB400111486F
:109AD000DE3000EB810081882798414327913C21AB
:109AE0002798B0FBF1F127910A48018C279801448F
:109AF00027910848C18B279880B281422DDD27E04D
:109B0000140000202C0000202E0000201C32002019
:109B1000FC3D00201C020020CCE1CABEA3BAD5FD4A
:109B2000D4DAC9FDCEC22E2E2E20202020202020C7
:109B300000000000CCE1CABEA3BAD5FDD4DABDB5A1
:109B4000CEC22E2E2E20202020202020000000001B
:109B50000120FE49C1F8A00013E04FF6FF70FB4959
:109B6000C1F8A0000DE04FF6FF70F849C1F8A00061
:109B700007E00020F549C1F8A0000120F44981F870
:109B8000D001ABE2F24890F84900E0B30020F04980
:109B900081F8490001F54050D0F8DC0B38B1084697
:109BA000C08B02460821029000200AF02BFF0BF028
:109BB0001DF802460321029001200AF023FF202015
:109BC000FBF75CFB2020FBF759FB2020FBF756FB43
:109BD0002020FBF753FB4AF2AF30FBF74FFB20206E
:109BE000FBF74CFB2020FBF749FBD94890F8D80144
:109BF00000EB4001D648DE3030F821100A460291D1
:109C00000921012000E01CE00AF0FCFE2020FBF707
:109C100035FB2020FBF732FBCD48C16C0A46029190
:109C2000032102200AF0FEFF4AF2AF30FBF726FBC9
:109C3000C748D0F8D4110A460291082102200AF040
:109C4000F1FFC348C18B90F8D80100EB4002C04837
:109C5000DE3030F8220081421CDB0220BC4981F852
:109C6000D001012081F8D101BAA200210320FBF725
:109C7000CDFB0022032102200AF0D4FF012211466D
:109C80001046F6F767FE0020B14981F8480081F8D8
:109C90004900C86422E2AE4890F84900F0B30020C1
:109CA000AB4981F8490001F54050D0F8DC0B38B1E0
:109CB0000846C08B02460821029000200AF0A2FE4E
:109CC0000AF094FF02460321029001200AF09AFE56
:109CD0002020FBF7D3FA2020FBF7D0FA2020FBF757
:109CE000CDFA2020FBF7CAFA4AF2AF30FBF7C6FAEA
:109CF0002020FBF7C3FA2020FBF7C0FA944890F825
:109D0000D80100EB40019248DE3030F821100A46BD
:109D10000291092101200AF075FE00E01AE02020DE
:109D2000FBF7ACFA2020FBF7A9FA8948C16C0A4678
:109D30000291032102200AF075FF4AF2AF30FBF7CF
:109D40009DFA8348D0F8D4110A46029108210220D6
:109D50000AF068FF7E48C08B7D49498C884204DD4B
:109D600001207A49C1F8A00007E000207749C1F836
:109D7000A0000520764981F8D001AFE1744890F841
:109D80004900E0B30020724981F8490001F54050D4
:109D9000D0F8DC0B38B10846C08B0246082102908F
:109DA00000200AF02FFE0AF021FF02460321029054
:109DB00001200AF027FE2020FBF760FA2020FBF7A5
:109DC0005DFA2020FBF75AFA2020FBF757FA4AF2F7
:109DD000AF30FBF753FA2020FBF750FA2020FBF7B7
:109DE0004DFA5B4890F8D80100EB40015848DE304E
:109DF00030F821100A4602910921012000E01CE000
:109E00000AF000FE2020FBF739FA2020FBF736FA93
:109E10004F48C16C0A460291032102200AF002FF5A
:109E20004AF2AF30FBF72AFA4948D0F8D4110A4673
:109E30000291082102200AF0F5FE4548C18B90F8F6
:109E4000D80100EB40024248DE3030F82200814267
:109E50001CDC02203E4981F8D001012081F8D101AB
:109E60003CA200210320FBF7D1FA002203210220AB
:109E70000AF0D8FE012211461046F6F76BFD0020CD
:109E8000334981F8480081F84900C86426E1304828
:109E900090F84900F0B300202D4981F8490001F500
:109EA0004050D0F8DC0B38B10846C08B0246082180
:109EB000029000200AF0A6FD254890F8D80100EB9A
:109EC00040012348DE3000EB8100008902902048E9
:109ED00090F8D80100EB40011D48DE3030F8211029
:109EE000DE380191C18B00919DE807000AF078FDF2
:109EF000174988830846818B0A4602910321012075
:109F00000AF080FD2020FBF7B9F92020FBF7B6F915
:109F1000202000E04BE0FBF7B1F92020FBF7AEF981
:109F20004AF2AF30FBF7AAF92020FBF7A7F920206F
:109F3000FBF7A4F9064890F8D80100EB400104486B
:109F4000DE3030F821100A46029111E0FC3D00207D
:109F50001C020020CCE1CABEA3BAD5FDD4DABAE314
:109F6000CEC22E2E2E2020202020202000000000F7
:109F7000092101200AF046FD2020FBF77FF920206F
:109F8000FBF77CF9F348C16C0A46029103210220D9
:109F90000AF048FE4AF2AF30FBF770F9ED48D0F80E
:109FA000D4110A460291082102200AF03BFEE9483A
:109FB000C06CE849D1F8D411884248D3E54890F8FC
:109FC000D801092828DAE34890F8D801401CE14973
:109FD00081F8D801084690F8D80100EB4001DD482F
:109FE000DE3030F8210088B1DA4890F8D80100EB73
:109FF0004001D848DE3000EB8100408830B10020BD
:10A00000D44981F8D001012081F8D10101220A212F
:10A010000846F6F79FFC1AE00320CE4981F8D001EC
:10A02000012081F8D101CCA200210846FBF7EEF90E
:10A03000D0A200210320FBF7E9F9282200210846DD
:10A04000F6F75AFD02220A210846F6F783FC45E09E
:10A0500046E0C04890F8490020B30020BD4981F88F
:10A06000490001F54050D0F8DC0B38B10846C08BF0
:10A0700002460821029000200AF0C4FC0AF0B6FD56
:10A0800002460321029001200AF0BCFC2020FBF7CD
:10A09000F5F82020FBF7F2F82020FBF7EFF820205E
:10A0A000FBF7ECF8BA480078052815D101221146D3
:10A0B0001046F6F74FFCFF20B54908700021B5485F
:10A0C000C0F8081100E008E0C0F800112020B249F3
:10A0D00008700120B149087000E000BF09F04EB8D7
:10A0E000AD48007825287CD1AC480078D0B100205C
:10A0F000AA49087009F0E8FF0020A949C1F8A000AA
:10A10000944981F8480081F84900C8640846C08B2A
:10A110008883002081F8D001012081F8D10100203E
:10A1200081F8D8019A48007805281CD101220A211B
:10A130000846F6F70FFCFF209549087028220021F9
:10A140000846F6F7D9FC00209549C1F8A000002187
:10A150009048C0F80811C0F8001120218E48017005
:10A1600001208E4908707B4890F8D00107286FD2F3
:10A17000DFE800F004EEEDECEBEAE90004207549BD
:10A1800081F8D001012081F8D101084690F8D8016A
:10A1900000EB4001834830F821002822014602905C
:10A1A0000120F6F7A9FC00207D49C1F8A000062196
:10A1B000FBF7D0FB674890F8D8014AF2D921084450
:10A1C00081B208460291FBF759F86248C18B90F8BA
:10A1D000D80100EB4002734830F82200814238DA9F
:10A1E00000E0FDE3AFF2D06200210320FBF70EF99F
:10A1F0005848C08B57490884084690F8D80100EBAE
:10A200004001684830F82110524890F8D80100EB1E
:10A210004002644800EB82004089081A4D49488496
:10A22000084690F8D80100EB40015E4800EB810041
:10A230004088484948650846406DC0EB00108000E2
:10A2400048650846406D1E3888650020488335E023
:10A25000EEE3AFF2207200210320FBF7D7F83D4870
:10A26000C08B3C490884084690F8D80100EB4001B7
:10A270004C4830F82110374890F8D80100EB4002E4
:10A28000484800EB82004089084432494884084627
:10A2900090F8D80100EB4001424800EB8100408873
:10A2A0002C4948650846406DC0EB001080004865A9
:10A2B0000846406D1E38886501204883254890F87F
:10A2C000D80100EB4001374830F82100024609214F
:10A2D000029001200AF096FB2020FAF7CFFF202001
:10A2E000FAF7CCFF1B4890F8D80100EB40012D484D
:10A2F00000EB81004088C0EB001080001549C1F8D8
:10A30000D4010846D0F8D4110A460291082102204F
:10A310000AF088FC00200F4981F8490081F84800C4
:10A32000C8640846408BA0B9084690F8D80100EBF5
:10A3300040011C4800EB81008088A8BB0120054932
:10A3400081F8D0013AE064E1D5E138E02CE361E244
:10A35000D7E02FE01C020020D7D4D1A1A3C1D7E9B8
:10A36000A3BAC8ABB2BFBDE1CAF82020202020208C
:10A3700000000000CCE1CABEA3BAB0B4C8A1CFFBB4
:10A38000BCFCCDCBB3F62020202020200000000014
:10A39000140000201C3200202C0000202E00002081
:10A3A000FC3D002072030020FFE70420FE4981F8F5
:10A3B000D00103E00620FC4981F8D00139E3FA48D6
:10A3C00090F84900F0B30020F74981F8490001F501
:10A3D0004050D0F8DC0B38B10846C08B024608214B
:10A3E000029000200AF00EFB0AF000FC0246032156
:10A3F000029001200AF006FB2020FAF73FFF202000
:10A40000FAF73CFF2020FAF739FF2020FAF736FF51
:10A410004AF2AF30FAF732FF2020FAF72FFF202060
:10A42000FAF72CFFE04890F8D80100EB4001DF4834
:10A4300030F821100A460291092101200AF0E2FABF
:10A44000202000E019E0FAF719FF2020FAF716FFA4
:10A45000D548C16C0A460291032102200AF0E2FBB2
:10A460004AF2AF30FAF70AFFCF48D0F8D4110A46C3
:10A470000291082102200AF0D5FBCB48C08BCA49C3
:10A48000498C884234DAC848C08BC749098C884255
:10A4900028DDC548C16C279190F8D80100EB400138
:10A4A000C24800EB810081882798414327913C21D5
:10A4B0002798B0FBF1F12791BB48018C2798014404
:10A4C0002791B948C18B279880B2814204DD0120D1
:10A4D000B749C1F8A00013E04FF6FF70B449C1F8C6
:10A4E000A0000DE04FF6FF70B149C1F8A00007E0F1
:10A4F0000020AF49C1F8A0000120AB4981F8D0018C
:10A5000097E2A94890F84900F0B30020A64981F8E5
:10A51000490001F54050D0F8DC0B38B10846C08B3B
:10A5200002460821029000200AF06CFA0AF05EFB55
:10A5300002460321029001200AF064FA2020FAF773
:10A540009DFE2020FAF79AFE2020FAF797FE2020A1
:10A55000FAF794FE4AF2AF30FAF790FE2020FAF7AD
:10A560008DFE2020FAF78AFE8F4890F8D80100EB84
:10A5700040018E4830F821100A460291092101203D
:10A580000AF040FA202000E019E0FAF777FE2020D8
:10A59000FAF774FE8448C16C0A4602910321022036
:10A5A0000AF040FB4AF2AF30FAF768FE7E48D0F876
:10A5B000D4110A460291082102200AF033FB7A489E
:10A5C000C18B90F8D80100EB4002784830F82200A7
:10A5D00081421DDB0220744981F8D001012081F8FD
:10A5E000D101AFF2906200210320FAF70FFF0022A1
:10A5F000032102200AF016FB012211461046F6F74D
:10A60000A9F90020684981F8480081F84900C86428
:10A610000FE2654890F84900F0B30020624981F8E4
:10A62000490001F54050D0F8DC0B38B10846C08B2A
:10A6300002460821029000200AF0E4F90AF0D6FA56
:10A6400002460321029001200AF0DCF92020FAF7EB
:10A6500015FE2020FAF712FE2020FAF70FFE202028
:10A66000FAF70CFE4AF2AF30FAF708FE2020FAF7AC
:10A6700005FE2020FAF702FE4B4890F8D80100EBC7
:10A6800040014A4830F821100A4602910921012070
:10A690000AF0B8F9202000E019E0FAF7EFFD2020D9
:10A6A000FAF7ECFD4048C16C0A46029103210220F2
:10A6B0000AF0B8FA4AF2AF30FAF7E0FD3A48D0F8BB
:10A6C000D4110A460291082102200AF0ABFA36485A
:10A6D000C08B3549498C884204DD01203449C1F8DA
:10A6E000A00007E000203249C1F8A00005202E4953
:10A6F00081F8D0019DE12C4890F84900F0B300208A
:10A70000294981F8490001F54050D0F8DC0B38B1F7
:10A710000846C08B02460821029000200AF072F918
:10A720000AF064FA02460321029001200AF06AF955
:10A730002020FAF7A3FD2020FAF7A0FD2020FAF749
:10A740009DFD2020FAF79AFD4AF2AF30FAF796FD08
:10A750002020FAF793FD2020FAF790FD124890F898
:10A76000D80100EB4001114830F821100A4602914F
:10A77000092101200AF046F9202000E020E0FAF744
:10A780007DFD2020FAF77AFD0748C16C0A46029148
:10A79000032102200AF046FA4AF2AF30FAF76EFDC2
:10A7A0000148D0F8D41105E01C02002072030020FB
:10A7B000FC3D00200A460291082102200AF032FAEC
:10A7C000FE48C18B90F8D80100EB4002FC4830F8FD
:10A7D000220081421DDC0220F84981F8D0010120CD
:10A7E00081F8D101AFF6940200210320FAF70EFEA2
:10A7F0000022032102200AF015FA01221146104618
:10A80000F6F7A8F80020ED4981F8480081F84900E2
:10A81000C8640EE1E94890F84900E0B30020E74938
:10A8200081F8490001F54050D0F8DC0B38B10846FA
:10A83000C08B02460821029000200AF0E3F8DF48AE
:10A8400090F8D80100EB4001DD4800EB8100008961
:10A850000290DA4890F8D80100EB4001D84830F86F
:10A860002110D6480191C18B00919DE807000AF0A4
:10A87000B7F8D24988830846818B0A4602910321A2
:10A8800001200AF0BFF82020FAF7F8FC2020FAF7A0
:10A89000F5FC202000E037E0FAF7F0FC2020FAF782
:10A8A000EDFC4AF2AF30FAF7E9FC2020FAF7E6FCBB
:10A8B0002020FAF7E3FCC14890F8D80100EB4001F2
:10A8C000BF4830F821100A460291092101200AF000
:10A8D00099F82020FAF7D2FC2020FAF7CFFCB748ED
:10A8E000C16C0A460291032102200AF09BF94AF248
:10A8F000AF30FAF7C3FCB148D0F8D4110A46029140
:10A90000082102200AF08EF9AC48C06CAB49D1F89E
:10A91000D411884247D3A94890F8D801092826DAEB
:10A92000A64890F8D801401CA44981F8D8010846EF
:10A9300090F8D80100EB4001A14830F8210080B127
:10A940009E4890F8D80100EB40019D4800EB810043
:10A95000408830B10020994981F8D001012081F868
:10A96000D10101220A210846F5F7F4FF1BE003207C
:10A97000924981F8D001012081F8D10191A20021F2
:10A980000846FAF743FDAFF2146200210320FAF7FC
:10A990003DFD282200210846F6F7AEF802220A21E2
:10A9A0000846F5F7D7FF44E0844890F8490030B3F3
:10A9B0000020824981F8490001F54050D0F8DC0BB5
:10A9C00038B10846C08B02460821029000200AF0E8
:10A9D00019F80AF00BF9024603210290012000E069
:10A9E00029E00AF00FF82020FAF748FC2020FAF7B7
:10A9F00045FC2020FAF742FC2020FAF73FFC78487B
:10AA00000078052813D1012211461046F5F7A2FF60
:10AA1000FF207349087000217248C0F80811C0F87F
:10AA2000001120207049087001207049087000E072
:10AA300000BF08F0A3BB6C48007828287ED16B4883
:10AA40000078E8B300206949087009F0EDF90121A8
:10AA50006448C0F808110021C0F80011644A0721B9
:10AA6000022009F07FFB5548C08A000B614908703D
:10AA70005248C08AC0F3032048705048C08AC0F3CF
:10AA8000031088704D48C08A00F00F00C8704B4812
:10AA9000808A642190FBF1F0564908714748818A09
:10AAA0005448007900EBC00202EB0010A1EB8000DB
:10AAB0000A2190FBF1F04F4948714048808A00E03C
:10AAC00032E0097901EBC10202EB0111A0EB810038
:10AAD0004849497901EB8101A0EB41004549887162
:10AAE0000020364981F8D001012081F8D1010020F1
:10AAF00081F8D8010846C08B03463D4A05210290E3
:10AB000001200AF03EF93B4A052102200AF0A2F991
:10AB10002A4890F8D8013849085C0A30C1B20122AD
:10AB200002200291FAF70CFC244890F8D00140B1C1
:10AB3000012879D0062878D0072800E0E7E275D10F
:10AB4000A4E22748007820BB012211461046F5F701
:10AB500001FFFF2022490870184890F8D8012549C4
:10AB6000085C50B1154890F8D801085C401E1349A4
:10AB700091F8D8111F4A505405E009200F4991F867
:10AB8000D8111C4A50541B4A052102200AF062F9D0
:10AB9000A6E113480078032849D101221146104646
:10ABA000F5F7D8FEFF200E490870044890F8D80148
:10ABB0001049085C09282BDA00481FE01C0200201D
:10ABC00072030020D7D4D1A1A3C2D7E9A3BAC8ABDE
:10ABD000B2BFBDE1CAF820202020202000000000E4
:10ABE000140000201C3200202C0000202E00002029
:10ABF00046000020E04400204464010890F8D80199
:10AC0000085C401CFB4991F8D811FB4A505405E000
:10AC10000020F84991F8D811F74A5054F64A052116
:10AC200002200AF017F95BE1B3E15AE16DE2F34863
:10AC30000078022832D1012211461046F5F78AFE2B
:10AC4000FF20EE490870EB4890F8D801EC49085C09
:10AC50000A30C0B20022014602900220FAF770FBCF
:10AC6000E44890F8D80138B1E24890F8D801401E85
:10AC7000E04981F8D80103E00620DE4981F8D801D7
:10AC8000DC4890F8D801DE49085C0A30C0B20122E5
:10AC9000014602900220FAF753FB21E1D7480078E1
:10ACA000072833D1012211461046F5F753FEFF2045
:10ACB000D2490870CF4890F8D801D149085C0A30D1
:10ACC000C0B20022014602900220FAF739FBC948BF
:10ACD00090F8D801062807DAC64890F8D801401C39
:10ACE000C44981F8D80103E00020C24981F8D801A5
:10ACF000C04890F8D801C249085C0A30C0B20122AD
:10AD0000014602900220FAF71BFBE9E0BB480078FD
:10AD1000052821D1012211461046F5F71BFEFF2020
:10AD2000B6490870B34890F8D801B549085C0A30B4
:10AD3000C0B20022014602900220FAF701FB002176
:10AD4000B048C0F80811C0F800112020AE490870C2
:10AD50000120AE490870C3E0A848007804287DD1DE
:10AD6000012211461046F5F7F5FDFF20A3490870B2
:10AD7000A1484078A049097801EB810100EB41002E
:10AD800018286BDA9C48C0789B49897801EB8101CF
:10AD900000EB41003C2861DA974800789549C88269
:10ADA0000846C08A4FF6FF7101EA00109149C88237
:10ADB0000846C08A9049497808448E49C8820846A6
:10ADC000C08A4FF6FF7101EA00108A49C88208461E
:10ADD000C08A8949897808448649C8820846C08A59
:10ADE0004FF6FF7101EA00108249C8820846C08A06
:10ADF0008149C97808447F49C8827F4800798882A0
:10AE00000846808A00EB80004FF6FF7101EA40009F
:10AE1000784988820846808A774949790844754983
:10AE200088820846808A00EB80004FF6FF7101EAB5
:10AE30004000704988820846808A6F4989790844B1
:10AE40006C498882002120916A48C08A03122099A7
:10AE50004A1C08A820924354664800E040E0C08A9B
:10AE6000C3B220994A1C08A8209243546148808AA2
:10AE7000031220994A1C08A8209243545D48808AF6
:10AE8000C3B220994A1C08A82092435455218DF83A
:10AE90003F100E212A914FF6FF712A9801EA4011C6
:10AEA0002A9108AA20212A98F9F740FE514890F8E3
:10AEB000D8015349085C0A30C1B200220220029135
:10AEC000FAF73EFA52A200210846FAF79FFA574ACB
:10AED00000210320FAF79AFA0620464981F8D001AA
:10AEE00014E1444890F84900F0B30020414981F84A
:10AEF00049004F4A0721022009F034F93D48C08B30
:10AF000003464B4A05210290012009F03AFF4848C8
:10AF1000807800F03F012B914FF6FF712B9801EAEA
:10AF200000212B914248407800F07F012B9801448A
:10AF30002B913048C18A2B98814229D103220521C7
:10AF40000846F5F707FD2B48C08B2A49898A8842B5
:10AF500010DB38A200210846FAF758FA3CA200217B
:10AF60000320FAF753FA00E012E00720214981F8A4
:10AF7000D0010DE03DA200210846FAF747FA012072
:10AF80001C4981F8D0014FF6FF703F49C1F8A0007D
:10AF9000BCE01848C08B1749898A884212DB25A279
:10AFA00000210846FAF732FA29A200210320FAF715
:10AFB0002DFA032205210846F5F7CCFC07200D49A0
:10AFC00081F8D0010B4890F8490088B10020094968
:10AFD00081F84900164A0721022009F0C3F8054804
:10AFE000C08B0346124A05210290012009F0C9FED8
:10AFF0008CE000001C020020E0440020140000202F
:10B00000446401081C3200202C0000202E00002087
:10B01000D4A4D4BCD7B4CCACA3BAB5C8B4FDCAB11F
:10B02000BCE420202020202000000000D888000858
:10B0300046000020D4A4D4BCD7B4CCACA3BAD4A4CA
:10B04000D4BCBDE1CAF82020202020200000000050
:10B05000CCE1CABEA3BAD4A4D4BCBDE1CAF8C7EB44
:10B06000B0B4C8B7C8CFBCFC00000000D4A4D4BCA6
:10B07000D7B4CCACA3BAC9FDCEC2D6D02E2E2E20CA
:10B080002020202000000000FC3D0020FD4800782A
:10B09000042813D1012211461046F5F75BFCFF206E
:10B0A000F84908700021F848C0F80811C0F80011EC
:10B0B0002020F64908700120F5490870F54890F8FD
:10B0C000490088B10020F34981F84900F24A07217C
:10B0D000022009F047F8EF48C08B0346EE4A0521ED
:10B0E0000290012009F04DFEEA48C08BE949898AA7
:10B0F000884204DB0120E949C1F8A00004E04FF6D2
:10B10000FF70E649C1F8A00000E000BF91E4DF480D
:10B11000007826287ED1DE480078C8B10020DC49BE
:10B12000087008F039F80020DA4981F8480081F801
:10B130004900C8640121D448C0F808110021C0F8B2
:10B1400000110020D34981F8D001012081F8D101FC
:10B15000CC480078052818D101220A210846F5F7C5
:10B16000F9FBFF20C7490870282200210846F5F79F
:10B17000C3FC0021C448C0F80811C0F80011202009
:10B18000C24908700120C2490870C24890F8D00135
:10B1900007287CD2DFE800F004256C7BFEFDBA00B6
:10B1A000282240F252310120F5F7A6FC0020BB49CD
:10B1B0000866BBA200210846FAF728F9BF4A002119
:10B1C0000220FAF723F9BE4A00210320FAF71EF9FC
:10B1D0000120B04981F8D001002081F84900C864FD
:10B1E0003DE2AC4890F84900C8B10020A94981F877
:10B1F00049000846C08B024605210290012009F053
:10B2000001FCFAF71DF9A348C16C0A460291052119
:10B21000022000E024E209F005FDFAF757FA9D4804
:10B22000008E40F25231884221DBA6A2002108465E
:10B23000FAF7ECF8012205210846F5F78BFBFF2011
:10B24000904908709E4A383200210320FAF7DEF850
:10B250009A4A00210220FAF7D9F802208D4981F894
:10B26000D001002081F8480081F84900C864F6E167
:10B27000884890F8490078B10020864981F8490053
:10B280000846C08B024605210290012000E0E5E15E
:10B2900009F0B8FBFAF7D4F87A480078042834D1DA
:10B2A000012211461046F5F755FBFF20754908703D
:10B2B0008BA200210846FAF7A9F8804A0021022053
:10B2C000FAF7A4F87E4A00210320FAF79FF8062037
:10B2D000704981F8D001002081F8480081F84900C8
:10B2E000C86440F2A230A1F8280D00BF282240F225
:10B2F00052310120F5F700FC002068490866012062
:10B30000C1F8A4000020C1F8A800A8E1614890F8A5
:10B310004900E8B300205F4981F849000846B0F8C9
:10B32000280D098E884208DD5A48008E5949A1F837
:10B33000280D0846C06CA1F82A0D5648B0F8280D13
:10B340005449098E88426DDA5248008E40F23E31EF
:10B35000884241DA4F48008E4E49B1F8281D401A04
:10B3600000EB800040004B49B1F8281D40F23E320E
:10B37000511A90FBF1F04748008E4648008E45492F
:10B38000B1F8281D401A00EB80004000414902E05E
:10B3900037E15CE136E1B1F8281D511A90FBF1F07C
:10B3A0003C49098E08443B49A1F844000846B0F8DE
:10B3B0004400024605210290012009F023FBFAF720
:10B3C0003FF83448C16C0A4602910521022009F079
:10B3D00029FCFAF77BF93EE02E48008E00F252304D
:10B3E0002C48008E00F25230029000EBD070C0F377
:10B3F0004F002849A1F844000846B0F8440002462E
:10B4000005210290012009F0FDFAFAF719F8214808
:10B41000C06C024605210290022009F003FCFAF7F5
:10B4200055F918E01B48C08B1A49A1F8440008469A
:10B43000C08B024605210290012009F0E3FAF9F7DA
:10B44000FFFF1448C16C0A4602910521022009F051
:10B45000E9FBFAF73BF91148D0F8A40080B10D4898
:10B46000C16CB0F88A00814248D201200B49C1F872
:10B47000A0000020C1F898000120C1F8A80087E0D2
:10B4800086E00000140000201C3200202C00002068
:10B490002E0000201C02002046000020FC3D002061
:10B4A000C2DEBCD3D7B4CCACA3BAC9FDCEC2202077
:10B4B000202020202020202000000000287B0008E1
:10B4C00058920008C2DEBCD3D7B4CCACA3BABAE35E
:10B4D000CEC220202020202020202020000000009C
:10B4E000C2DEBCD3D7B4CCACA3BAB2E2CAD4D6D0F5
:10B4F0002E2E2E202020202000000000FD48B0F835
:10B50000280DFC49098E88420ADBFA48B0F86C0025
:10B51000801CF949C1F8A0000220C1F8A80037E05A
:10B52000F448B0F84410B0F88C0081420ADAF148CF
:10B53000B0F86C00801CF049C1F8A0000320C1F8ED
:10B54000A80025E0EB48B0F84410B0F88E00814226
:10B550000ADA0120E849C1F8A0000020C1F89800EB
:10B560000420C1F8A80013E00020E349C1F8A400BA
:10B57000C1F8A000C1F89000282240F25231012009
:10B58000F5F7BAFA0020DC4908660520C1F8A800E2
:10B59000D848C06CB0F5B47F05D101220A21084615
:10B5A000F5F7D8F92DE0D348C06C40F266318842F7
:10B5B00005D11E2205210846F5F7CCF921E0CD483A
:10B5C000C06CB0F5617F1CD301220A210846F5F753
:10B5D000C1F9CAA200210846F9F718FFCEA200213E
:10B5E0000320F9F713FF0020C349C1F8A000282267
:10B5F00040F252310120F5F77FFA0421BD4880F86E
:10B60000D0112CE0CB48007804280DD101220A216A
:10B610001420F5F79FF9FF20C64908702620C64977
:10B6200008700120C5490870B24890F8490068B117
:10B630000020B04981F849000846C08B0246052128
:10B640000290012009F0DEF9F9F7FAFE07E0262062
:10B65000B94908700120B949087000E000BF55E5FC
:10B66000B5480078312841F0FB85B4480078E8B34C
:10B670000020B249087008F091F900209D4981F836
:10B68000D001012081F8D101002081F8D80181F892
:10B69000D90C084690F8D80100EB40019548DE30FF
:10B6A00030F82100024604210290012009F045FAF9
:10B6B000904890F8D80100EB40018E48DE3000EB56
:10B6C000810041880A4602910621012009F035FADD
:10B6D000884890F8D80100EB40018648DE3000EB46
:10B6E000810081880A460291082100E09EE0012045
:10B6F00009F023FA7F4890F8D80100EB40017D481B
:10B70000DE3000EB8100C1880A4602910A21012047
:10B7100009F013FA774890F8D801401C00EB40017B
:10B720007448DE3030F821100A46029104210220CC
:10B7300009F003FA6F4890F8D801401C00EB400173
:10B740006C48DE3000EB810041880A4602910621F8
:10B75000022009F0F2F9674890F8D801401C00EB8C
:10B7600040016448DE3000EB810081880A46029186
:10B770000821022009F0E1F95E4890F8D801401C48
:10B7800000EB40015B48DE3000EB8100C1880A46D7
:10B7900002910A21022009F0D0F9564890F8D80108
:10B7A000801C00EB40015348DE3030F821100A467F
:10B7B00002910421032009F0C0F94E4890F8D80105
:10B7C000801C00EB40014B48DE3000EB81004188DB
:10B7D0000A4602910621032009F0AFF9454890F886
:10B7E000D801801C00EB40014248DE3000EB8100B4
:10B7F00081880A4602910821032009F09EF93D48FC
:10B8000090F8D801801C00EB40013A48DE3000EB94
:10B810008100C1880A4602910A21032009F08DF9AE
:10B820000123062200211846F9F73EFD314890F821
:10B83000D00128B101285CD0022841F00E85FCE33C
:10B840002C4890F8D801092840DA3A480078E8BB3B
:10B85000012211461046F5F77DF8FF2035490870A2
:10B86000244890F8D801401C224981F8D8010846A4
:10B8700090F8D90C02281DDA084690F8D90C401C23
:10B88000C0B20023062219460290F9F70DFD1948AF
:10B8900090F8D90C401C174981F8D90C084690F84B
:10B8A000D90C401CC1B2012306220291002102984A
:10B8B000F9F7FAFC0F4890F8D8010E4991F8D91C15
:10B8C000401AC0EBC0001E49084400E049E10246AE
:10B8D000002102900120F9F799FD064890F8D8015F
:10B8E000044991F8D91C401A00EB40010148DE30B0
:10B8F00028E0FDE31C020020FC3D0020C2DEBCD39A
:10B90000D7B4CCACA3BACAD4D1E9CDEAB3C920200C
:10B910002020202000000000CCE1CABEA3BAB0B4B1
:10B92000C8B7C8CFBCFCBCCCD0F8C2DEBCD320208A
:10B9300000000000140000202C0000202E00002039
:10B940002901002030F821100A460291042101202B
:10B9500009F0F3F8FE4890F8D801FD4991F8D91C98
:10B96000401A00EB4001FA48DE3000EB81004188CC
:10B970000A4602910621012009F0DFF8F44890F808
:10B98000D801F34991F8D91C401A00EB4001F04866
:10B99000DE3000EB810081880A46029108210120F7
:10B9A00009F0CBF8EA4890F8D801E94991F8D91C98
:10B9B000401A00EB4001E648DE3000EB8100C18810
:10B9C0000A4602910A21012009F0B7F8E04890F8F0
:10B9D000D801DF4991F8D91C401A401CC0EBC000C7
:10B9E000DC4901440A46029100210220F9F70EFDCC
:10B9F000D74890F8D801D64991F8D91C401A401C74
:10BA000000EB4001D248DE3030F821100A460291A6
:10BA10000421022009F091F8CD4890F8D801CC49D2
:10BA200091F8D91C401A401C00EB4001C848DE3098
:10BA300000EB810041880A4602910621022009F0AC
:10BA40007CF8C34890F8D801C14991F8D91C401A34
:10BA5000401C00EB4001BE48DE3000EB81008188D5
:10BA60000A4602910821022009F067F8B84890F8C8
:10BA7000D801B74991F8D91C401A401C00EB40018D
:10BA8000B348DE3000EB8100C1880A4602910A21EA
:10BA9000022009F052F8AE4890F8D801AC4991F86C
:10BAA000D91C401A801CC0EBC000AA4901440A46B8
:10BAB000029100210320F9F7A9FCA54890F8D801CC
:10BAC000A34991F8D91C401A801C00EB4001A04802
:10BAD000DE3030F821100A4602910421032009F0DB
:10BAE0002CF89B4890F8D801994991F8D91C401A34
:10BAF000801C00EB40019648DE3000EB810041885D
:10BB00000A4602910621032009F017F8904890F8A0
:10BB1000D8018F4991F8D91C401A801C00EB4001D4
:10BB20008B48DE3000EB810081880A4602910821B3
:10BB3000032009F002F8864890F8D801844991F86A
:10BB4000D91C401A801C00EB40018148DE3000EB1C
:10BB50008100C1880A4602910A21032008F0EDFF06
:10BB6000FDE37B4890F8D80100287DDD7A48007815
:10BB7000032879D1012211461046F4F7EBFEFF208D
:10BB800075490870724890F8D801401E704981F8D4
:10BB9000D801084690F8D90C00281DDD084690F819
:10BBA000D90C401CC0B20023062219460290F9F7B6
:10BBB0007BFB674890F8D90C401E654981F8D90C89
:10BBC000084690F8D90C401CC1B20123062202910C
:10BBD00000210298F9F768FB5D4890F8D8015C49AC
:10BBE00091F8D91C401AC0EBC0005A4908440246DB
:10BBF000002102900120F9F709FC554890F8D8017E
:10BC0000534991F8D91C401A00EB40015048DE30EE
:10BC100030F821100A4602910421012008F08DFF1E
:10BC20004B4890F8D81190F8D90C081A00EB400155
:10BC30004748DE3000EB810041880A460291062128
:10BC4000012008F07AFF424890F8D801404991F865
:10BC5000D91C401A00EB40013D48DE3000EB81006A
:10BC600081880A46029100E0EEE00821012008F0F8
:10BC700064FF374890F8D801354991F8D91C401A2B
:10BC800000EB40013248DE3000EB8100C1880A46FB
:10BC900002910A21012008F050FF2D4890F8D801A8
:10BCA0002B4991F8D91C401A401CC0EBC00029490F
:10BCB00001440A46029100210220F9F7A7FB24481B
:10BCC00090F8D801224991F8D91C401A401C00EB89
:10BCD00040011F48DE3030F821100A46029104214D
:10BCE000022008F02AFF1A4890F8D801184991F864
:10BCF000D91C401A401C00EB40011548DE3000EB17
:10BD0000810041880A4602910621022008F015FFB1
:10BD10000F4890F8D8010E4991F8D91C401A401CE0
:10BD200000EB40010A48DE3000EB810081880A46C2
:10BD300002910821022008F000FF054890F8D80180
:10BD4000034991F8D91C401A401C00EB400105E062
:10BD50001C0200202901002014000020FB4800EBF9
:10BD60008100C1880A4602910A21022008F0E5FEFE
:10BD7000F648DE3890F8D801F449DE3991F8D91C3C
:10BD8000401A801CC0EBC000F14901440A460291F0
:10BD900000210320F9F73AFBEC48DE3890F8D8018F
:10BDA000EA49DE3991F8D91C401A801C00EB4001A9
:10BDB000E64830F821100A4602910421032008F0D9
:10BDC000BCFEE248DE3890F8D801E049DE3991F84F
:10BDD000D91C401A801C00EB4001DC4800EB8100BC
:10BDE00041880A4602910621032008F0A6FED748A2
:10BDF000DE3890F8D801D549DE3991F8D91C401ABF
:10BE0000801C00EB4001D14800EB810081880A468C
:10BE100002910821032008F090FECC48DE3890F80B
:10BE2000D801CA49DE3991F8D91C401A801C00EBB0
:10BE30004001C64800EB8100C1880A4602910A21F0
:10BE4000032008F07AFE8AE2C248007804287CD1F8
:10BE5000012211461046F4F77DFDFF20BD49087010
:10BE60000120BA49DE3981F8D001002081F8DA0CCE
:10BE7000084690F8D80100EB4001B44830F82100A2
:10BE800042F20F7188420EDD2D20B049DE39A1F853
:10BE9000DC0C2D21AD48DE38A0F8DE1CA0F8E01C3B
:10BEA000A0F8E21C6AE0A948DE3890F8D80100EB5F
:10BEB0004001A64830F821002B904FF47A712B985E
:10BEC00090FBF1F0A149DE39A1F8DC0C0846B0F88E
:10BED000DC0C00EB4001C1EBC0112B98A0EBC100C2
:10BEE00081B22B9164212B9890FBF1F081B297489D
:10BEF000DE38A0F8DE1CB0F8DE0C00EBC00101EB70
:10BF000000112B98A0EB810081B22B910A212B9874
:10BF100090FBF1F081B28D48DE38A0F8E01CB0F85B
:10BF2000E00C00EB80012B98A0EB410081B22B913B
:10BF30008649DE392B98A1F8E20C0846B0F8DC0CF3
:10BF40003030A1F8DC0C084600E0EBE1B0F8DE0C84
:10BF5000303081B27D48DE38A0F8DE1CB0F8E00C4D
:10BF6000303081B27948DE38A0F8E01CB0F8E20C3D
:10BF7000303081B27548DE38A0F8E21C7348DE38F4
:10BF800090F8D80100EB4001704800EB8100408838
:10BF9000B0F57A7F09DB2D216C48DE38A0F8E41C6F
:10BFA000A0F8E61CA0F8E81C50E06848DE3890F8DD
:10BFB000D80100EB4001654800EB810040882B90E0
:10BFC00064212B9890FBF1F081B26048DE38A0F834
:10BFD000E41CB0F8E40C00EBC00101EB00112B985D
:10BFE000A0EB810081B22B910A212B9890FBF1F0FC
:10BFF00081B25648DE38A0F8E61CB0F8E60C00EB3B
:10C0000080012B98A0EB410081B22B914F49DE3982
:10C010002B98A1F8E80C0846B0F8E40C303081B257
:10C020004A48DE38A0F8E41CB0F8E60C303081B2A3
:10C030004648DE38A0F8E61C00E0F6E3B0F8E80C6D
:10C04000303081B24148DE38A0F8E81C3F48DE3885
:10C0500090F8D80100EB40013C4800EB810080885B
:10C06000B0F57A7F09DB2D213848DE38A0F8EA1CCC
:10C07000A0F8EC1CA0F8EE1C50E03448DE3890F834
:10C08000D80100EB4001314800EB810080882B9003
:10C0900064212B9890FBF1F081B22C48DE38A0F897
:10C0A000EA1CB0F8EA0C00EBC00101EB00112B9880
:10C0B000A0EB810081B22B910A212B9890FBF1F02B
:10C0C00081B22248DE38A0F8EC1CB0F8EC0C00EB92
:10C0D00080012B98A0EB410081B22B911B49DE39E6
:10C0E0002B98A1F8EE0C0846B0F8EA0C303000E0CE
:10C0F00036E181B21548DE38A0F8EA1CB0F8EC0C45
:10C10000303081B21148DE38A0F8EC1CB0F8EE0CEB
:10C11000303081B20D48DE38A0F8EE1C0B48DE3816
:10C1200090F8D80100EB4001084800EB8100C0887E
:10C13000B0F57A7F10DB2D210448DE38A0F8F01C22
:10C14000A0F8F21CA0F8F41C4FE00000FA02002056
:10C150002901002014000020FB4890F8D80100EBD2
:10C160004001F948DE3000EB8100C0882B9064214B
:10C170002B9890FBF1F081B2F348A0F8F01CB0F8D6
:10C18000F00C00EBC00101EB00112B98A0EB81003B
:10C1900081B22B910A212B9890FBF1F081B2EA48F1
:10C1A000A0F8F21CB0F8F20C00EB80012B98A0EB89
:10C1B000410081B22B91E4492B98A1F8F40C084678
:10C1C000B0F8F00C303081B2DF48A0F8F01CB0F8C5
:10C1D000F20C303081B2DC48A0F8F21CB0F8F40C5C
:10C1E000303081B2D848A0F8F41CD74890F8D90C68
:10C1F000401CC0B204210290F9F7ACFBD248B0F861
:10C20000DC1C08460291F9F739F8CF48B0F8DE1C7B
:10C2100008460291F9F732F8CB48B0F8E01C08461E
:10C220000291F9F72BF8C848B0F8E21C08460291D1
:10C23000F9F724F8C44890F8D90C401CC1B2029117
:10C2400006210298F9F786FB2020F9F717F8BE4877
:10C25000B0F8E41C08460291F9F710F8BA48B0F8B3
:10C26000E61C08460291F9F709F8B748B0F8E81C4F
:10C2700008460291F9F702F8B34890F8D90C401C2F
:10C28000C1B2029108210298F9F764FB2020F8F767
:10C29000F5FFAD48B0F8EA1C08460291F8F7EEFF4A
:10C2A000A948B0F8EC1C08460291F8F7E7FFA64849
:10C2B000B0F8EE1C08460291F8F7E0FFA24890F8AB
:10C2C000D90C401CC1B202910A210298F9F742FB35
:10C2D0002020F8F7D3FF9C48B0F8F01C08460291E4
:10C2E000F8F7CCFF9848B0F8F21C08460291F8F72E
:10C2F000C5FF9548B0F8F41C08460291F8F7BEFF58
:10C30000914890F8DA0C0830C1B28F48029190F849
:10C31000D90C401CC1B201220191DDE90101F9F7FC
:10C320000FF81CE089480078052818D10122114631
:10C330001046F4F70FFBFF20844908700220824961
:10C3400081F8D001084690F8D90C401CC0B20023F7
:10C35000062219460290F8F7A7FF07F097FCFDE3C5
:10C360007A48007803287CD1012211461046F4F760
:10C37000F1FAFF2075490870734890F8DA1C00F64E
:10C38000DC4030F81100202808D130216E4890F8A8
:10C39000DA2C00F6DC4020F812102AE06A4890F807
:10C3A000DA1C00F6DC4030F81100392810DA664853
:10C3B00090F8DA1C00F6DC4030F81100401C81B225
:10C3C000614890F8DA2C00F6DC4020F8121010E0FA
:10C3D0005D4890F8DA1C00F6DC4030F8110039288E
:10C3E00007D13021584890F8DA2C00F6DC4020F8CC
:10C3F0001210554890F8D90C401CC0B2042102908C
:10C40000F9F7A8FA5048B0F8DC1C08460291F8F792
:10C4100035FF4D48B0F8DE1C08460291F8F72EFFB4
:10C420004948B0F8E01C08460291F8F727FF464853
:10C43000B0F8E21C08460291F8F720FF424890F855
:10C44000D90C401CC1B2029106210298F9F782FA78
:10C450002020F8F713FF3C48B0F8E41C084602918E
:10C4600000E054E0F8F70AFF3748B0F8E61C084649
:10C470000291F8F703FF3448B0F8E81C084602912F
:10C48000F8F7FCFE304890F8D90C401CC1B202917C
:10C4900008210298F9F75EFA2020F8F7EFFE2A4803
:10C4A000B0F8EA1C08460291F8F7E8FE2648B0F812
:10C4B000EC1C08460291F8F7E1FE2348B0F8EE1CA8
:10C4C00008460291F8F7DAFE1F4890F8D90C401C94
:10C4D000C1B202910A210298F9F73CFA2020F8F73C
:10C4E000CDFE1948B0F8F01C08460291F8F7C6FED8
:10C4F0001548B0F8F21C08460291F8F7BFFE124842
:10C50000B0F8F41C08460291F8F7B8FE23E20F4891
:10C510000078B8BB012211461046F4F71BFAFF2041
:10C520000A490870084890F8DA1C00F6DC4030F838
:10C53000110020280CD13921034890F8DA2C00F69C
:10C54000DC4020F812102FE01C0200201400002014
:10C55000FE4890F8DA1C00F6DC4030F81100302874
:10C5600011DDFA4890F8DA1C00F6DC4030F81100D2
:10C57000401E81B2F54890F8DA2C00F6DC4020F835
:10C58000121011E09CE0F14890F8DA1C00F6DC4053
:10C5900030F81100302807D13921EC4890F8DA2C16
:10C5A00000F6DC4020F81210E84890F8D90C401C46
:10C5B000C0B204210290F9F7CDF9E448B0F8DC1CD0
:10C5C00008460291F8F75AFEE048B0F8DE1C08462B
:10C5D0000291F8F753FEDD48B0F8E01C08460291DE
:10C5E000F8F74CFED948B0F8E21C08460291F8F77B
:10C5F00045FED64890F8D90C401CC1B202910621E4
:10C600000298F9F7A7F92020F8F738FECF48B0F8DC
:10C61000E41C08460291F8F731FECC48B0F8E61C5D
:10C6200008460291F8F72AFEC848B0F8E81C084608
:10C630000291F8F723FEC54890F8D90C401CC1B20E
:10C64000029108210298F9F785F92020F8F716FEE3
:10C65000BE48B0F8EA1C08460291F8F70FFEBB4846
:10C66000B0F8EC1C08460291F8F708FEB748B0F89D
:10C67000EE1C08460291F8F701FEB44890F8D90C78
:10C68000401CC1B202910A210298F9F763F92020F7
:10C69000F8F7F4FDAD48B0F8F01C08460291F8F741
:10C6A000EDFDAA48B0F8F21C08460291F8F7E6FD45
:10C6B000A648B0F8F41C08460291F8F7DFFDA4E3A1
:10C6C000A348007802287CD1012211461046F4F7D5
:10C6D00041F9FF209E4908709C4890F8DA0C002828
:10C6E000EDDD9A4890F8DA0C042811DA974890F8B2
:10C6F000DA0C0830C0B20290944890F8D90C401C73
:10C70000C1B200220191DDE90101F8F719FE3EE016
:10C710008E4890F8DA0C072811DA8C4890F8DA0C79
:10C720000930C0B20290894890F8D90C401CC1B2BF
:10C7300000220191DDE90101F8F702FE27E08348BC
:10C7400090F8DA0C0A2811DA804890F8DA0C0A30EE
:10C75000C0B202907D4890F8D90C401CC1B20022B2
:10C760000191DDE90101F8F7EBFD10E0774890F861
:10C77000DA0C0B30C0B20290744890F8D90C401C0F
:10C78000C1B200220191DDE90101F8F7D9FD6F483E
:10C7900090F8DA0C401E6D4981F8DA0C084690F8E2
:10C7A000DA0C042813DA084690F8DA0C0830C0B224
:10C7B0000290084690F8D90C401CC1B201220191A8
:10C7C00000E045E0DDE90101F8F7BAFD1DE35F484F
:10C7D00090F8DA0C072811DA5C4890F8DA0C093086
:10C7E000C0B20290594890F8D90C401CC1B2012245
:10C7F0000191DDE90101F8F7A3FD06E3534890F844
:10C80000DA0C0A2812DA514890F8DA0C0A30C0B271
:10C8100002904E4890F8D90C401CC1B201220191FF
:10C82000DDE90101F8F78CFDEFE2EFE2474890F80F
:10C83000DA0C0B30C0B20290444890F8D90C401C7E
:10C84000C1B201220191DDE90101F8F779FDDCE2D5
:10C850003F48007807287DD1012211461046F4F7A1
:10C8600079F8FF203A490870384890F8DA0C0C281B
:10C8700071DA364890F8DA0C042811DA334890F867
:10C88000DA0C0830C0B20290304890F8D90C401C45
:10C89000C1B200220191DDE90101F8F751FD3EE04E
:10C8A0002A4890F8DA0C072811DA284890F8DA0CB0
:10C8B0000930C0B20290254890F8D90C401CC1B292
:10C8C00000220191DDE90101F8F73AFD27E01F4858
:10C8D00090F8DA0C0A2811DA1C4890F8DA0C0A30C1
:10C8E000C0B20290194890F8D90C401CC1B2002285
:10C8F0000191DDE90101F8F723FD10E0134890F8FC
:10C90000DA0C0B30C0B20290104890F8D90C401CE1
:10C91000C1B200220191DDE90101F8F711FD0B48D8
:10C9200090F8DA0C401C094981F8DA0C084690F8B6
:10C93000DA0C042818DA084690F8DA0C0830C0B28D
:10C940000290084690F8D90C401C05E01C0200201B
:10C950001400002048E08BE1C1B201220191DDE921
:10C960000101F8F7EDFC50E2FE4890F8DA0C0728D8
:10C9700011DAFC4890F8DA0C0930C0B20290F9489C
:10C9800090F8D90C401CC1B201220191DDE90101EE
:10C99000F8F7D6FC39E2F34890F8DA0C0A2811DAF5
:10C9A000F04890F8DA0C0A30C0B20290ED4890F8E6
:10C9B000D90C401CC1B201220191DDE90101F8F757
:10C9C000BFFC22E2E74890F8DA0C0B30C0B20290CC
:10C9D000E44890F8D90C401CC1B201220191DDE974
:10C9E0000101F8F7ADFC10E2DF48007805287DD1A1
:10C9F000012211461046F3F7ADFFFF20DA49087017
:10CA00000020D84981F8D001084690F8DA0C0428B3
:10CA100011DA084690F8DA0C0830C0B202900846E5
:10CA200090F8D90C401CC1B200220191DDE901014E
:10CA3000F8F786FC3EE0CB4890F8DA0C072811DACC
:10CA4000C84890F8DA0C0930C0B20290C54890F896
:10CA5000D90C401CC1B200220191DDE90101F8F7B7
:10CA60006FFC27E0BF4890F8DA0C0A2811DABD48BD
:10CA700090F8DA0C0A30C0B20290BA4890F8D90C9B
:10CA8000401CC1B200220191DDE90101F8F758FC18
:10CA900010E0B44890F8DA0C0B30C0B20290B14804
:10CAA00090F8D90C401CC1B200220191DDE90101CE
:10CAB000F8F746FCAB4890F8D80100EB4001A948D4
:10CAC000DE3030F821000290A64890F8D90C401CC6
:10CAD000C1B201910421DDE9010208F02EF8A1485C
:10CAE00090F8D80100EB40019E4800E03EE0DE30C7
:10CAF00000EB810041889B48029190F8D90C401CC2
:10CB0000C1B201910621DDE9010208F016F895484D
:10CB100090F8D80100EB40019248DE3000EB810034
:10CB200081889048029190F8D90C401CC1B20191C3
:10CB30000821DDE9010208F000F88A4890F8D801E0
:10CB400000EB40018748DE3000EB8100C18885485A
:10CB5000029190F8D90C401CC1B200E07CE3019135
:10CB60000A21DDE9010207F0E8FF4EE17E48007886
:10CB700004287DD1012211461046F3F7EBFEFF2079
:10CB8000794908700020774981F8D001084690F86B
:10CB9000DA0C042811DA084690F8DA0C0830C0B232
:10CBA0000290084690F8D90C401CC1B200220191B5
:10CBB000DDE90101F8F7C4FB3EE06A4890F8DA0CC1
:10CBC000072811DA674890F8DA0C0930C0B20290F1
:10CBD000644890F8D90C401CC1B200220191DDE9F3
:10CBE0000101F8F7ADFB27E05E4890F8DA0C0A285F
:10CBF00011DA5C4890F8DA0C0A30C0B20290594859
:10CC000090F8D90C401CC1B200220191DDE901016C
:10CC1000F8F796FB10E0534890F8DA0C0B30C0B2EE
:10CC20000290504890F8D90C401CC1B200220191EA
:10CC3000DDE90101F8F784FB00202B900DE04B4863
:10CC40002B9930F81100303882B248492B9821F8DE
:10CC500010202B98401C81B22B912B980D28EEDBD5
:10CC60004048B0F8DC0C4FF47A7148433D4900E08D
:10CC7000CBE0B1F8DE1C01EBC10202EB011100EBCD
:10CC800081013848B0F8E00C00EB800001EB400176
:10CC90003448B0F8E20C084481B2324890F8D80128
:10CCA00000EB40022F48DE3020F82210DE38B0F8CA
:10CCB000E40C642148432B49B1F8E61C01EB8101E7
:10CCC00000EB41012748B0F8E80C084481B2254840
:10CCD00090F8D80100EB40022248DE3000EB8200E1
:10CCE00041802048B0F8EA0C642148431D49B1F85E
:10CCF000EC1C01EB810100EB41011A48B0F8EE0C8D
:10CD0000084481B2174890F8D80100EB400215485A
:10CD1000DE3000EB820081801248B0F8F00C642114
:10CD200048431049B1F8F21C01EB810100EB4101CD
:10CD30000C48B0F8F40C084481B20A4890F8D801C5
:10CD400000EB40020748DE3000EB8200C18005485E
:10CD500090F8D80100EB40010248DE3030F82100A5
:10CD6000029005E01C02002014000020F80E0020B4
:10CD7000FE4890F8D90C401CC1B201910421DDE9B4
:10CD8000010207F0DAFEF94890F8D80100EB400103
:10CD9000F648DE3000EB81004188F448029190F8BB
:10CDA000D90C401CC1B201910621DDE9010207F056
:10CDB000C4FEEE4890F8D80100EB4001EB48DE30AD
:10CDC00000EB81008188E948029190F8D90C401C61
:10CDD000C1B201910821DDE9010207F0AEFEE3488E
:10CDE00090F8D80100EB4001E048DE3000EB810014
:10CDF000C188DE48029190F8D90C401CC1B2019163
:10CE00000A21DDE9010207F098FE27E2D848007800
:10CE100005287DD1012211461046F3F79BFDFF2125
:10CE2000D348017000212A914FF6FF712A9801EA38
:10CE300040112A9118AA20212A98F7F733FE0021E1
:10CE40002A9108E018A92A98095C08AA11542A987E
:10CE5000401C81B22A912A982028F3DB00212A91D4
:10CE60002A98411C2A914FF6FF712A9801EA401135
:10CE70002A9118AA20212A98F7F714FE00212A9156
:10CE800009E018A92A98095C08AA203011542A98A8
:10CE9000401C81B22A912A982028F2DB9DF85F007D
:10CEA00055287CD1002120912A91D5E02099481C59
:10CEB00082B208A82092415C2A9800EB4002AB485D
:10CEC000DE3020F822102A9800EB4001A748DE301F
:10CED00030F821004FF6FF7101EA00212A9800EB9B
:10CEE0004002A248DE3020F822102A9800EB4001D0
:10CEF0009E48DE3030F821202099481C83B208A8D3
:10CF00002093405C104481B22A9800EB400200E07C
:10CF1000ADE09648DE3020F822102099481C82B2FD
:10CF200008A82092415C2A9800EB40028F48DE302E
:10CF300000EB820041802A9800EB40018B48DE30F4
:10CF400000EB810040884FF6FF7101EA00212A982A
:10CF500000EB40028548DE3000EB820041802A98D9
:10CF600000EB40018148DE3000EB810042882099CF
:10CF7000481C83B208A82093405C104481B22A98D0
:10CF800000EB40027948DE3000EB820041802099BE
:10CF9000481C82B208A82092415C2B9100E05FE01F
:10CFA0004FF6FF712B9801EA00212B912099481C24
:10CFB00082B208A82092415C2B98084481B22B9140
:10CFC0004FF47A712B9890FBF1F081B22A9800EB24
:10CFD00040026648DE3000EB820081804FF47A71B7
:10CFE0002B9890FBF1F201FB120081B22A9800EB22
:10CFF00040025E48DE3000EB8200C1802A9800EBE0
:10D0000040015A48DE3000EB8100C088642190FB6B
:10D01000F1F081B22A9800EB40025448DE3000EB78
:10D02000820001812A9800EB40015048DE3000EB7D
:10D030008100C088642190FBF1F201FB120081B2F3
:10D040002A9800EB40024948DE3000EB8200418123
:10D050002A98401C81B22A912A980A28FFF626AF06
:10D06000302044490870012043490870F4E04048EA
:10D070000078042878D1012211461046F3F76AFCA3
:10D08000FF203B490870002120912A919AE02A98BC
:10D0900000EB40013548DE3030F8210003122099C2
:10D0A000481C82B208A8209243542A9800EB400101
:10D0B0002E48DE3010F821302099481C82B208A892
:10D0C000209243542A9800EB40012848DE3000EBC0
:10D0D0008100408803122099481C82B208A820923F
:10D0E00043542A9800EB40012048DE3000EB8100D9
:10D0F00083782099481C82B208A8209243542A9829
:10D1000000EB40011948DE3000EB8100808800EB25
:10D110004001C1EBC0104FF6FF7101EAC0012B9135
:10D120002A9800EB40011148DE3000EB8100C188F5
:10D130002B98084481B22B912B9803122099481CFC
:10D1400082B208A8209243542B98C3B22099481C5D
:10D1500082B208A8209243542A9800EB4001034869
:10D16000DE3000EB810009E076E000001C020020C8
:10D17000140000202C0000202E000020C088642114
:10D1800090FBF1F081B22A9800EB4002FE4800EBE0
:10D19000820001812A9800EB4001FB4800EB8100EE
:10D1A000C088642190FBF1F201FB120081B22A9841
:10D1B00000EB4002F44800EB820041812A98401CB9
:10D1C00080B22A902A980A28FFF661AF55218DF87F
:10D1D0005F1000212A9108E008A92A98095C18AA82
:10D1E00011542A98401C81B22A912A982028F3DBF6
:10D1F00000212A914FF6FF712A9801EA40112A91E5
:10D2000018AA20212A98F7F791FC00212A910AE018
:10D2100008A92A982030095C18AA2A9811542A983B
:10D22000401C81B22A912A982028F1DB00212A9102
:10D230002A98411C2A914FF6FF712A9801EA401161
:10D240002A9118AA20212A98F7F770FC3020CF499C
:10D2500008700120CE49087000E000BF05F08EBFC5
:10D26000CA480078322841F09B85C9480078E8B365
:10D270000020C749087006F0DFFB0020C249DE39F4
:10D2800081F8D001012081F8D101002081F8D80176
:10D2900081F8D90C084690F8D80100EB4001BA4853
:10D2A000783030F82100024604210290012007F076
:10D2B00044FCB548DE3890F8D80100EB4001B24894
:10D2C000783000EB810041880A4602910621012056
:10D2D00007F033FCAC48DE3890F8D80100EB400191
:10D2E000A948783000EB8100818800E0AAE00A4676
:10D2F00002910821012007F020FCA348DE3890F8B5
:10D30000D80100EB4001A048783000EB8100C188D3
:10D310000A4602910A21012007F00FFC9A48DE38E4
:10D3200090F8D801401C00EB40019748783030F865
:10D3300021100A4602910421022007F0FEFB9248C8
:10D34000DE3890F8D801401C00EB40018E48783060
:10D3500000EB810041880A4602910621022007F075
:10D36000ECFB8948DE3890F8D801401C00EB400106
:10D370008548783000EB810081880A4602910821B7
:10D38000022007F0DAFB8048DE3890F8D801401C14
:10D3900000EB40017C48783000EB8100C1880A46F0
:10D3A00002910A21022007F0C8FB7748DE3890F886
:10D3B000D801801C00EB40017348783030F8211010
:10D3C0000A4602910421032007F0B7FB6E48DE38BD
:10D3D00090F8D801801C00EB40016B48783000EBDE
:10D3E000810041880A4602910621032007F0A5FB2F
:10D3F0006548DE3890F8D801801C00EB4001624897
:10D40000783000EB810081880A46029108210320D0
:10D4100007F093FB5C48DE3890F8D801801C00EBE5
:10D4200040015948783000EB8100C1880A460291DA
:10D430000A21032007F081FB012306220021184660
:10D44000F7F732FF5048DE3890F8D00128B10128B4
:10D450007ED0022841F0A184FEE34B48DE3890F8EC
:10D46000D80109283FDA4B480078E0BB0122114679
:10D470001046F3F76FFAFF20464908704248DE383D
:10D4800090F8D801401C4049DE3981F8D80108469F
:10D4900090F8D90C02281FDA084690F8D90C401CE5
:10D4A000C0B20023062219460290F7F7FDFE364867
:10D4B000DE3890F8D90C401C3349DE3981F8D90C9C
:10D4C000084690F8D90C401CC1B2012306220291F3
:10D4D00000210298F7F7E8FE2B48DE3890F8D801D3
:10D4E0002949DE3900E031E191F8D91C401AC0EB3E
:10D4F000C000294908440246002102900120F7F7A4
:10D5000085FF2148DE3890F8D8011F49DE3991F8AF
:10D51000D91C401A00EB40011B48783030F821102C
:10D520000A4602910421012007F007FB1648DE3865
:10D5300090F8D8011449DE3991F8D91C401A00EB53
:10D5400040011148783000EB810041880A4600E034
:10D55000FEE302910621012007F0EFFA0A48DE38C7
:10D5600090F8D8010849DE3991F8D91C401A00EB2F
:10D5700040010548783000EB810081880A4602911D
:10D58000082101200AE00000FA0200202C000020FF
:10D590002E000020140000202901002007F0CDFA01
:10D5A000FE4890F8D801FD4991F8D91C401A00EBCB
:10D5B0004001FB4800EB8100C1880A4602910A2124
:10D5C000012007F0BAFAF54890F8D801F34991F82C
:10D5D000D91C401A401CC0EBC000F24901440A4665
:10D5E000029100210220F7F711FFEC4890F8D801D2
:10D5F000EA4991F8D91C401A401C00EB4001E84868
:10D6000030F821100A4602910421022007F095FA11
:10D61000E24890F8D801E14991F8D91C401A401C21
:10D6200000EB4001DE4800EB810041880A46029190
:10D630000621022007F081FAD84890F8D801D7498E
:10D6400091F8D91C401A401C00EB4001D44800EB73
:10D65000810081880A4602910821022007F06DFAB4
:10D66000CE4890F8D801CD4991F8D91C401A401CF9
:10D6700000EB4001CA4800EB8100C1880A460291D4
:10D680000A21022007F059FAC44890F8D801C3498A
:10D6900091F8D91C401A801CC0EBC000C14901445C
:10D6A0000A46029100210320F7F7B0FEBB4890F82C
:10D6B000D801BA4991F8D91C401A801C00EB4001EE
:10D6C000B74830F821100A4602910421032007F0E0
:10D6D00034FAB24890F8D801B04991F8D91C401AF0
:10D6E000801C00EB4001AE4800EB810041880A46F7
:10D6F00002910621032007F020FAA84890F8D801EB
:10D70000A64991F8D91C401A801C00EB4001A4489E
:10D7100000EB810081880A4602910821032007F06E
:10D720000CFA9E4890F8D8019C4991F8D91C401AEF
:10D73000801C00EB40019A4800EB8100C1880A463A
:10D7400002910A21032007F0F8F9D0E3934890F8FA
:10D75000D80100287DDD94480078032879D1012282
:10D7600011461046F3F7F6F8FF208F4908708B48F2
:10D7700090F8D801401E894981F8D801084690F8F0
:10D78000D90C00281DDD084690F8D90C401CC0B209
:10D790000023062219460290F7F786FD7F4890F88D
:10D7A000D90C401E7D4981F8D90C084690F8D90C57
:10D7B000401CC1B201230622029100210298F7F712
:10D7C00073FD764890F8D801744991F8D91C401A35
:10D7D000C0EBC000734908440246002102900120BA
:10D7E000F7F714FE6D4890F8D8016C4991F8D91CF0
:10D7F000401A00EB40016A4830F821100A460291B5
:10D800000421012007F099F9644890F8D801634990
:10D8100091F8D91C401A00EB4001614800EB8100EF
:10D8200041880A4602910621012007F086F95B48EB
:10D8300090F8D801594991F8D91C401A00EB4001E1
:10D84000574800EB810081880A4602910821012097
:10D8500000E0E0E007F071F9504890F8D8014F4936
:10D8600091F8D91C401A00EB40014D4800EB8100B3
:10D87000C1880A4602910A21012007F05EF9474853
:10D8800090F8D801454991F8D91C401A401CC0EBCA
:10D89000C000444901440A46029100210220F7F7E2
:10D8A000B5FD3E4890F8D8013C4991F8D91C401A82
:10D8B000401C00EB40013A4830F821100A46029122
:10D8C0000421022007F039F9344890F8D80133498F
:10D8D00091F8D91C401A401C00EB4001304800EB85
:10D8E000810041880A4602910621022007F025F9AD
:10D8F0002A4890F8D801294991F8D91C401A401CAF
:10D9000000EB4001264800EB810081880A46029125
:10D910000821022007F011F9204890F8D8011F498A
:10D9200091F8D91C401A401C00EB40011C4800EB48
:10D930008100C1880A4602910A21022007F0FDF801
:10D94000164890F8D801154991F8D91C401A801C46
:10D95000C0EBC000134901440A4602910021032094
:10D96000F7F754FD0D4890F8D8010C4991F8D91CEF
:10D97000401A801C00EB4001094830F821100A468B
:10D9800002910421032007F0D8F8044890F8D80148
:10D99000024991F8D91C401A801C07E01C020020A3
:10D9A00072030020290100201400002000EB400138
:10D9B000FE4800EB810041880A46029106210320BF
:10D9C00007F0BBF8FA4890F8D801F94991F8D91C4A
:10D9D000401A801C00EB4001F44800EB8100818874
:10D9E0000A4602910821032007F0A7F8F04890F8B2
:10D9F000D801EF4991F8D91C401A801C00EB400176
:10DA0000EA4800EB8100C1880A4602910A210320FE
:10DA100007F093F86BE2E748007804287ED10122F2
:10DA200011461046F2F796FFFF20E24908700120E8
:10DA3000DF4981F8D001002081F8DA0C084690F81F
:10DA4000D80100EB4001D94830F8210042F20F71B3
:10DA500088420CDD2D20D649A1F8DC0C2D21D448BC
:10DA6000A0F8DE1CA0F8E01CA0F8E21C62E0D048A0
:10DA700090F8D80100EB4001CC4830F821002B9001
:10DA80004FF47A712B9890FBF1F0C949A1F8DC0CA6
:10DA90000846B0F8DC1C01EB4100C0EBC1112B982B
:10DAA000A0EBC10081B22B9164212B9890FBF1F087
:10DAB00081B2BF48A0F8DE1CB0F8DE1C01EBC1004B
:10DAC00000EB01112B98A0EB810081B22B910A2170
:10DAD0002B9890FBF1F081B2B548A0F8E01CB0F8AB
:10DAE000E00C00EB80012B98A0EB410081B22B9160
:10DAF000AF492B98A1F8E20C0846B0F8DC0C3030A6
:10DB0000A1F8DC0C0846B0F8DE0C303081B2A84831
:10DB1000A0F8DE1CB0F8E00C303000E0CAE181B2C1
:10DB2000A348A0F8E01CB0F8E20C303081B2A04865
:10DB3000A0F8E21C9E4890F8D80100EB40019B48F9
:10DB400000EB81004088B0F57A7F08DB2D219848F2
:10DB5000A0F8E41CA0F8E61CA0F8E81C47E09448F4
:10DB600090F8D80100EB4001904800EB810041881B
:10DB70002B9164212B9890FBF1F081B28C48A0F896
:10DB8000E41CB0F8E41C01EBC10000EB01112B9880
:10DB9000A0EB810081B22B910A212B9890FBF1F030
:10DBA00081B28348A0F8E61CB0F8E60C00EB8001D7
:10DBB0002B98A0EB410081B22B917D492B98A1F8C5
:10DBC000E80C0846B0F8E40C303081B27848A0F890
:10DBD000E41CB0F8E60C303081B27548A0F8E61CC1
:10DBE000B0F8E80C303081B27148A0F8E81C7048F9
:10DBF00090F8D80100EB40016C4800EB8100808870
:10DC0000B0F57A7F08DB2D216948A0F8EA1CA0F85E
:10DC1000EC1CA0F8EE1C49E0654890F8D80100EB38
:10DC20004001624800EB810080882B9064212B9892
:10DC300090FBF1F081B25E48A0F8EA1CB0F8EA1C53
:10DC400001EBC10000EB01112B98A0EB810081B228
:10DC50002B910A212B9800E0FEE390FBF1F081B2BA
:10DC60005348A0F8EC1CB0F8EC0C00EB80012B98AA
:10DC7000A0EB410081B22B914D492B98A1F8EE0CFD
:10DC80000846B0F8EA0C303081B24948A0F8EA1CE6
:10DC9000B0F8EC0C303081B24548A0F8EC1CB0F87C
:10DCA000EE0C303081B24248A0F8EE1C404890F8AB
:10DCB000D80100EB40013D4800EB8100C088B0F581
:10DCC0007A7F08DB2D213A48A0F8F01CA0F8F21C5E
:10DCD000A0F8F41C49E0364890F8D80100EB400168
:10DCE000324800EB8100C0882B9064212B9890FB78
:10DCF000F1F081B22E48A0F8F01CB0F8F01C01EB56
:10DD0000C10000EB01112B98A0EB810081B22B9197
:10DD10000A212B9890FBF1F081B22548A0F8F21C63
:10DD2000B0F8F20C00EB80012B98A0EB410081B21F
:10DD30002B911F492B98A1F8F40C0846B0F8F00C71
:10DD4000303081B21A48A0F8F01CB0F8F20C00E0B4
:10DD5000CEE0303081B21648A0F8F21CB0F8F40CD6
:10DD6000303081B21248A0F8F41C114890F8D90C58
:10DD7000401CC0B204210290F7F7ECFD0C48B0F84B
:10DD8000DC1C08460291F7F779FA0948B0F8DE1C66
:10DD900008460291F7F772FA0548B0F8E01C084609
:10DDA0000291F7F76BFA024806E0000072030020C8
:10DDB0001C02002014000020B0F8E21C084602916A
:10DDC000F7F75CFAFE4890F8D90C401CC1B20291FA
:10DDD00006210298F7F7BEFD2020F7F74FFAF84822
:10DDE000B0F8E41C08460291F7F748FAF448B0F896
:10DDF000E61C08460291F7F741FAF148B0F8E81C32
:10DE000008460291F7F73AFAED4890F8D90C401C11
:10DE1000C1B2029108210298F7F79CFD2020F7F784
:10DE20002DFAE748B0F8EA1C08460291F7F726FAFF
:10DE3000E348B0F8EC1C08460291F7F71FFAE048F7
:10DE4000B0F8EE1C08460291F7F718FADC4890F893
:10DE5000D90C401CC1B202910A210298F7F77AFD51
:10DE60002020F7F70BFAD648B0F8F01C08460291CC
:10DE7000F7F704FAD248B0F8F21C08460291F7F717
:10DE8000FDF9CF48B0F8F41C08460291F7F7F6F90F
:10DE9000CB4890F8DA0C0830C1B2C948029190F82A
:10DEA000D90C401CC1B201220191DDE90101F7F753
:10DEB00047FA1CE0C3480078052818D10122114612
:10DEC0001046F2F747FDFF20BE4908700220BC490A
:10DED00081F8D001084690F8D90C401CC0B200234C
:10DEE000062219460290F7F7DFF905F0CFFEFDE3B1
:10DEF000B448007803287CD1012211461046F2F77D
:10DF000029FDFF20AF490870AD4890F8DA1C00F6F3
:10DF1000DC4030F81100202808D13021A84890F8C2
:10DF2000DA2C00F6DC4020F812102AE0A44890F821
:10DF3000DA1C00F6DC4030F81100392810DAA0486D
:10DF400090F8DA1C00F6DC4030F81100401C81B279
:10DF50009B4890F8DA2C00F6DC4020F8121010E014
:10DF6000974890F8DA1C00F6DC4030F811003928A8
:10DF700007D13021924890F8DA2C00F6DC4020F8E6
:10DF800012108F4890F8D90C401CC0B204210290A6
:10DF9000F7F7E0FC8A48B0F8DC1C08460291F7F776
:10DFA0006DF98748B0F8DE1C08460291F7F766F96C
:10DFB0008348B0F8E01C08460291F7F75FF9804803
:10DFC000B0F8E21C08460291F7F758F97C4890F83F
:10DFD000D90C401CC1B2029106210298F7F7BAFC95
:10DFE0002020F7F74BF97648B0F8E41C0846029178
:10DFF00000E054E0F7F742F97148B0F8E61C084633
:10E000000291F7F73BF96E48B0F8E81C0846029118
:10E01000F7F734F96A4890F8D90C401CC1B2029164
:10E0200008210298F7F796FC2020F7F727F96448B3
:10E03000B0F8EA1C08460291F7F720F96048B0F8FA
:10E04000EC1C08460291F7F719F95D48B0F8EE1C90
:10E0500008460291F7F712F9594890F8D90C401C7C
:10E06000C1B202910A210298F7F774FC2020F7F759
:10E0700005F95348B0F8F01C08460291F7F7FEF88E
:10E080004F48B0F8F21C08460291F7F7F7F84C48F1
:10E09000B0F8F41C08460291F7F7F0F85DE1494842
:10E0A000007898BB012211461046F2F753FCFF207E
:10E0B00044490870424890F8DA1C00F6DC4030F819
:10E0C0001100202808D139213D4890F8DA2C00F6BB
:10E0D000DC4020F812102BE0394890F8DA1C00F6EA
:10E0E000DC4030F81100302811DD354890F8DA1C9A
:10E0F00000F6DC4030F81100401E81B2304890F844
:10E10000DA2C00F6DC4020F8121011E0A1E02C48D7
:10E1100090F8DA1C00F6DC4030F81100302807D106
:10E120003921274890F8DA2C00F6DC4020F812104C
:10E13000234890F8D90C401CC0B204210290F7F794
:10E1400009FC1F48B0F8DC1C08460291F7F796F866
:10E150001B48B0F8DE1C08460291F7F78FF8184804
:10E16000B0F8E01C08460291F7F788F81448B0F8B8
:10E17000E21C08460291F7F781F8114890F8D90C93
:10E18000401CC1B2029106210298F7F7E3FB202060
:10E19000F7F774F80A48B0F8E41C08460291F7F75C
:10E1A0006DF80748B0F8E61C08460291F7F766F8E4
:10E1B0000348B0F8E81C08460291F7F75FF803E05F
:10E1C0001C02002014000020FE4890F8D90C401CCE
:10E1D000C1B2029108210298F7F7BCFB2020F7F7A3
:10E1E0004DF8F848B0F8EA1C08460291F7F746F8EF
:10E1F000F448B0F8EC1C08460291F7F73FF8F148F4
:10E20000B0F8EE1C08460291F7F738F8ED4890F8A0
:10E21000D90C401CC1B202910A210298F7F79AFB6F
:10E220002020F7F72BF8E748B0F8F01C08460291D9
:10E23000F7F724F8E348B0F8F21C08460291F7F724
:10E240001DF8E048B0F8F41C08460291F7F716F8FC
:10E2500093E3DD48007802287ED101221146104662
:10E26000F2F778FBFF20D8490870D64890F8DA0C0E
:10E27000002872DDD34890F8DA0C042811DAD1486E
:10E2800090F8DA0C0830C0B20290CE4890F8D90C61
:10E29000401CC1B200220191DDE90101F7F750F8FD
:10E2A0003EE0C84890F8DA0C072811DAC54890F823
:10E2B000DA0C0930C0B20290C24890F8D90C401C68
:10E2C000C1B200220191DDE90101F7F739F827E039
:10E2D000BC4890F8DA0C0A2811DABA4890F8DA0C3F
:10E2E0000A30C0B20290B74890F8D90C401CC1B2B5
:10E2F00000220191DDE90101F7F722F810E0B148B1
:10E3000090F8DA0C0B30C0B20290AE4890F8D90CFD
:10E31000401CC1B200220191DDE90101F7F710F8BC
:10E32000A84890F8DA0C401EA64981F8DA0C084695
:10E3300090F8DA0C042814DA084690F8DA0C083061
:10E34000C0B20290084690F8D90C401CC1B201221C
:10E350000191DDE9010101E043E0C6E0F6F7F0FFDD
:10E360000BE3984890F8DA0C072811DA954890F8F2
:10E37000DA0C0930C0B20290924890F8D90C401CD7
:10E38000C1B201220191DDE90101F6F7D9FFF4E202
:10E390008C4890F8DA0C0A2811DA8A4890F8DA0CDE
:10E3A0000A30C0B20290874890F8D90C401CC1B224
:10E3B00001220191DDE90101F6F7C2FFDDE28148AA
:10E3C00090F8DA0C0B30C0B202907E4890F8D90C6D
:10E3D000401CC1B201220191DDE90101F6F7B0FF55
:10E3E000CBE27948007807287ED1012211461046F9
:10E3F000F2F7B0FAFF2074490870724890F8DA0C0E
:10E400000C2872DA6F4890F8DA0C042811DA6D489B
:10E4100090F8DA0C0830C0B202906A4890F8D90C33
:10E42000401CC1B200220191DDE90101F6F788FF2D
:10E4300040E0644890F8DA0C072813DA614890F855
:10E44000DA0C0930C0B202905E4890F8D90C401C3A
:10E45000C1B20022019100E090E2DDE90101F6F78E
:10E460006FFF27E0574890F8DA0C0A2811DA554870
:10E4700090F8DA0C0A30C0B20290524890F8D90CE9
:10E48000401CC1B200220191DDE90101F6F758FFFD
:10E4900010E04C4890F8DA0C0B30C0B202904948BA
:10E4A00090F8D90C401CC1B200220191DDE90101B4
:10E4B000F6F746FF434890F8DA0C401C414981F8D2
:10E4C000DA0C084690F8DA0C042814DA084690F8BA
:10E4D000DA0C0830C0B20290084690F8D90C401C03
:10E4E000C1B20122019101E045E088E1DDE90101CD
:10E4F000F6F726FF41E2334890F8DA0C072811DAE4
:10E50000304890F8DA0C0930C0B202902D4890F8EB
:10E51000D90C401CC1B201220191DDE90101F6F7DD
:10E520000FFF2AE2274890F8DA0C0A2811DA25486A
:10E5300090F8DA0C0A30C0B20290224890F8D90C58
:10E54000401CC1B201220191DDE90101F6F7F8FE9C
:10E5500013E21C4890F8DA0C0B30C0B20290194854
:10E5600090F8D90C401CC1B201220191DDE90101F2
:10E57000F6F7E6FE01E21448007805287DD1012275
:10E5800011461046F2F7E6F9FF200F490870002007
:10E590000C4981F8D001084690F8DA0C042815DA05
:10E5A000084690F8DA0C0830C0B20290084690F89D
:10E5B000D90C401CC1B200220191DDE90101F6F73E
:10E5C000BFFE42E01C02002014000020F94890F831
:10E5D000DA0C072811DAF74890F8DA0C0930C0B2E3
:10E5E0000290F44890F8D90C401CC1B2002201916D
:10E5F000DDE90101F6F7A4FE27E0EE4890F8DA0C19
:10E600000A2811DAEB4890F8DA0C0A30C0B202900E
:10E61000E84890F8D90C401CC1B200220191DDE914
:10E620000101F6F78DFE10E0E24890F8DA0C0B30AD
:10E63000C0B20290DF4890F8D90C401CC1B2002251
:10E640000191DDE90101F6F77BFEDA4890F8D80187
:10E6500000EB4001D84830F821000290D54890F8EE
:10E66000D90C401CC1B201910421DDE9010206F080
:10E6700064FAD04890F8D80100E03EE000EB400199
:10E68000CD4800EB81004188CA48029190F8D90C2E
:10E69000401CC1B201910621DDE9010206F04DFAEC
:10E6A000C44890F8D80100EB4001C34800EB81005A
:10E6B0008188C048029190F8D90C401CC1B20191E8
:10E6C0000821DDE9010206F038FABA4890F8D801CD
:10E6D00000EB4001B84800EB8100C188B5480291C9
:10E6E00090F8D90C401CC1B2019100E054E30A211A
:10E6F000DDE9010206F021FA3FE1B0480078042884
:10E700007DD1012211461046F2F724F9FF20AB49D2
:10E7100008700020A74981F8D001084690F8DA0C6B
:10E72000042811DA084690F8DA0C0830C0B20290DA
:10E73000084690F8D90C401CC1B200220191DDE9D5
:10E740000101F6F7FDFD3EE09A4890F8DA0C072843
:10E7500011DA984890F8DA0C0930C0B20290954866
:10E7600090F8D90C401CC1B200220191DDE90101F1
:10E77000F6F7E6FD27E08F4890F8DA0C0A2811DA60
:10E780008C4890F8DA0C0A30C0B20290894890F8B0
:10E79000D90C401CC1B200220191DDE90101F6F75C
:10E7A000CFFD10E0834890F8DA0C0B30C0B2029035
:10E7B000804890F8D90C401CC1B200220191DDE9DB
:10E7C0000101F6F7BDFD00212B910DE07C482B994E
:10E7D00030F81100303882B279492B9821F8102096
:10E7E0002B98401C81B22B912B980D28EEDB7148A1
:10E7F000B0F8DC0C4FF47A7148436E4900E0BCE09D
:10E80000B1F8DE1C01EBC10202EB011100EB81014A
:10E810006848B0F8E00C00EB800001EB400165486F
:10E82000B0F8E20C084481B2624890F8D80100EBDD
:10E830004002614820F822105E48B0F8E40C6421E0
:10E8400048435C49B1F8E61C01EB810100EB410152
:10E850005848B0F8E80C084481B2564890F8D801FE
:10E8600000EB4002544800EB820041805148B0F870
:10E87000EA0C642148434F49B1F8EC1C01EB8101DB
:10E8800000EB41014B48B0F8EE0C084481B2494816
:10E8900090F8D80100EB4002474800EB82008180ED
:10E8A0004448B0F8F00C642148434249B1F8F21CE6
:10E8B00001EB810100EB41013E48B0F8F40C084443
:10E8C00081B23C4890F8D80100EB40023A4800EB96
:10E8D0008200C180374890F8D80100EB40013648EB
:10E8E00030F821000290334890F8D90C401CC1B296
:10E8F00001910421DDE9010206F01FF92D4890F88D
:10E90000D80100EB40012C4800EB810041882948E8
:10E91000029190F8D90C401CC1B201910621DDE9A9
:10E92000010206F00AF9234890F8D80100EB4001F3
:10E93000214800EB810081881E48029190F8D90C93
:10E94000401CC1B201910821DDE9010206F0F5F891
:10E95000184890F8D80100EB4001174800EB8100FF
:10E96000C1881448029190F8D90C401CC1B20191A1
:10E970000A21DDE9010206F0E0F80FE20F48007815
:10E9800005287DD1012211461046F1F7E3FFFF2053
:10E990000A49087002212A914FF6FF712A9801EA6C
:10E9A00040112A9118AA20212A98F6F77BF8002115
:10E9B0002A9110E01C0200207203002014000020A5
:10E9C000F80E002018A92A98095C08AA11542A9860
:10E9D000401C81B22A912A982028F3DB02212A9137
:10E9E0002A98411C2A914FF6FF712A9801EA40119A
:10E9F0002A9118AA20212A98F6F754F800212A9182
:10EA000009E018A92A98095C08AA203011542A980C
:10EA1000401C81B22A912A982028F2DB9DF85F00E1
:10EA200055287DD1002120912A91C5E02099481CCC
:10EA300082B208A82092415C2A9800EB4002FC4870
:10EA400020F822102A9800EB4001F94830F8210004
:10EA50004FF6FF7101EA00212A9800EB4002F448CA
:10EA600020F822102A9800EB4001F14830F82120CC
:10EA70002099481C83B208A82093405C104400E011
:10EA8000A5E081B22A9800EB4002E94820F8221064
:10EA90002099481C82B208A82092415C2A9800EB79
:10EAA0004002E34800EB820041802A9800EB4001DD
:10EAB000DF4800EB810040884FF6FF7101EA00213A
:10EAC0002A9800EB4002DA4800EB820041802A9845
:10EAD00000EB4001D64800EB810042882099481C99
:10EAE00083B208A82093405C104481B22A9800EBBE
:10EAF0004002CF4800EB820041802099481C82B23E
:10EB000008A82092415C2B914FF6FF712B9801EAE7
:10EB100000212B912099481C82B208A8209200E085
:10EB20004EE0415C2B98084481B22B914FF47A71EE
:10EB30002B9890FBF1F081B22A9800EB4002BC4880
:10EB400000EB820081804FF47A712B9890FBF1F2F8
:10EB500001FB120081B22A9800EB4002B44800EB9E
:10EB60008200C1802A9800EB4001B14800EB81008F
:10EB7000C088642190FBF1F081B22A9800EB40023A
:10EB8000AB4800EB820001812A9800EB4001A848C5
:10EB900000EB8100C088642190FBF1F201FB1200C0
:10EBA00081B22A9800EB4002A14800EB820041812B
:10EBB0002A98401C81B22A912A980A28FFF636AF7B
:10EBC00030209C49087001209B490870E4E09B4874
:10EBD000007804287ED1012211461046F1F7BAFED2
:10EBE000FF2096490870002120912A918AE02A98F6
:10EBF00000EB40018E4830F8210003122099481C98
:10EC000082B208A8209243542A9800EB4001884819
:10EC100010F821302099481C82B208A82092435451
:10EC20002A9800EB4001824800EB810040880312E3
:10EC30002099481C82B208A8209243542A9800EBDD
:10EC400040017B4800EB810083782099481C82B208
:10EC500008A8209243542A9800EB4001744800EB26
:10EC60008100818801EB4100C0EBC1104FF6FF71BC
:10EC700001EAC0012B912A9800EB40016C4800EB9F
:10EC80008100C1882B98084481B22B912B980312E4
:10EC90002099481C82B208A8209243542B98C3B2F2
:10ECA0002099481C82B208A8209243542A9800EB6D
:10ECB00040015F4800EB8100C088642190FBF1F0C7
:10ECC00081B22A9800EB4002594800EB8200018192
:10ECD0002A9800E060E000EB4001554800EB81001D
:10ECE000C088642190FBF1F201FB120081B22A98E6
:10ECF00000EB40024E4800EB820041812A98401C04
:10ED000080B22A902A980A28FFF671AF55218DF813
:10ED10005F1000212A9108E008A92A98095C18AA26
:10ED200011542A98401C81B22A912A982028F3DB9A
:10ED300002212A914FF6FF712A9801EA40112A9187
:10ED400018AA20212A98F5F7F1FE00212A910AE05D
:10ED500008A92A982030095C18AA2A9811542A98E0
:10ED6000401C81B22A912A982028F1DB02212A91A5
:10ED70002A98411C2A914FF6FF712A9801EA401106
:10ED80002A9118AA20212A98F5F7D0FE3020294987
:10ED9000087001202849087000E000BF04F0EEB9B7
:10EDA0002448007834287DD123480078F0B300202F
:10EDB0002149087004F08EFE0020214981F8D0011D
:10EDC000012081F8D101002081F8D80181F8D90C07
:10EDD000084690F8D80101F5EE7131F8200002469E
:10EDE00004210290012005F00DFE154890F8D8018D
:10EDF0000F49863101EB800041880A4602910821C3
:10EE0000012005F0FFFD0E4890F8D801401C08498C
:10EE1000863131F820100A4602910421022005F0C3
:10EE2000F1FD074890F8D801401C0BE035E00000E8
:10EE3000720300202C0000202E000020140000206F
:10EE40001C020020FE4901EB800041880A46029125
:10EE50000821022005F0D6FDFA4890F8D801801C60
:10EE6000F74931F820100A4602910421032005F0E9
:10EE7000C9FDF44890F8D801801CF14901EB8000ED
:10EE800041880A4602910821032005F0BBFD0123B9
:10EE9000062200211846F6F707FAEA4890F8D00152
:10EEA00030B100E0FEE301287ED002287DD1FAE3F4
:10EEB000E44890F8D8010E2840DAE3480078E8BB2F
:10EEC000012211461046F1F745FDFF20DE4908708A
:10EED000DC4890F8D801401CDA4981F8D80108468E
:10EEE00090F8D90C02281DDA084690F8D90C401C7D
:10EEF000C0B20023062219460290F6F7D5F9D14890
:10EF000090F8D90C401CCF4981F8D90C084690F8EC
:10EF1000D90C401CC1B201230622029100210298A3
:10EF2000F6F7C2F901210846F6F714FDC54890F836
:10EF3000D801C44991F8D91C401A00E0D6E0401C21
:10EF40000A2190FBF1F0303080B20290F6F796F98A
:10EF5000BC4890F8D801BB4991F8D91C401A401C14
:10EF60000A2190FBF1F201FB1200303081B2084619
:10EF70000291F6F783F9B34890F8D801B14991F8B6
:10EF8000D91C401AAE4931F820100A4602910421DA
:10EF9000012005F037FDAB4890F8D801A94991F858
:10EFA000D91C401AA64901E0EAE2FDE301EB80002A
:10EFB00041880A4602910821012005F023FD012124
:10EFC0000220F6F7C7FC9F4890F8D8019D4991F8B8
:10EFD000D91C401A801C0A2190FBF1F0303081B21C
:10EFE00008460291F6F74AF9964890F8D8019549F3
:10EFF00091F8D91C401A801C0A2190FBF1F201FB08
:10F000001200303081B208460291F6F737F98D4888
:10F0100090F8D8018B4991F8D91C401A401C8849B6
:10F0200031F820100A4602910421022005F0EAFC82
:10F03000844890F8D801834991F8D91C401A401CA3
:10F040007F4901EB800041880A4602910821022095
:10F0500005F0D8FC01210320F6F77CFC794890F8F4
:10F06000D801784991F8D91C401AC01C0A2190FB9C
:10F07000F1F0303081B208460291F6F7FFF871489E
:10F0800090F8D8016F4991F8D91C401AC01C0A2188
:10F0900090FBF1F201FB1200303081B20846029180
:10F0A000F6F7ECF8674890F8D801664991F8D91C52
:10F0B000401A801C624931F820100A46029104214E
:10F0C000032005F09FFC5F4890F8D8015D4991F856
:10F0D000D91C401A801C5A4901EB800041880A461D
:10F0E00002910821032005F08DFC48E2554890F874
:10F0F000D80100287EDD5448007803287AD1012207
:10F1000011461046F1F726FCFF204F4908704D4884
:10F1100090F8D801401E4B4981F8D801084690F874
:10F12000D90C00281DDD084690F8D90C401CC0B24F
:10F130000023062219460290F6F7B6F8414890F8E7
:10F14000D90C401E3F4981F8D90C084690F8D90CDB
:10F15000401CC1B201230622029100210298F6F759
:10F16000A3F801210846F6F7F5FB364890F8D801D8
:10F17000344991F8D91C401A401C0A2190FBF1F047
:10F18000303080B20290F6F779F82E4890F8D80126
:10F190002C4991F8D91C401A401C0A2190FBF1F22D
:10F1A00001FB1200303081B208460291F6F766F892
:10F1B000244890F8D801234991F8D91C401A2049D5
:10F1C00031F820100A4602910421012005F01AFCB2
:10F1D0001C4890F8D8011B4991F8D91C401A1849CD
:10F1E00001EB800041880A4602910821012005F0C8
:10F1F00009FC00E09DE001210220F6F7ABFB11487D
:10F2000090F8D8010F4991F8D91C401A801C0A21A6
:10F2100090FBF1F0303081B208460291F6F72EF8FB
:10F22000084890F8D801074991F8D91C401A801C69
:10F230000A2190FBF1F201FB1200303081B205E0AF
:10F24000F80300201C020020140000200846029150
:10F25000F6F714F8FE4890F8D801FD4991F8D91C4A
:10F26000401A401CFB4931F820100A460291042143
:10F27000022005F0C7FBF64890F8D801F44991F850
:10F28000D91C401A401CF34901EB800041880A4612
:10F2900002910821022005F0B5FB01210320F6F7B9
:10F2A00059FBEB4890F8D801E94991F8D91C401A6C
:10F2B000C01C0A2190FBF1F0303081B20846029167
:10F2C000F5F7DCFFE24890F8D801E14991F8D91C44
:10F2D000401AC01C0A2190FBF1F201FB12003030F1
:10F2E00081B208460291F5F7C9FFD94890F8D801D4
:10F2F000D74991F8D91C401A801CD64931F8201002
:10F300000A4602910421032005F07CFBD04890F8C6
:10F31000D801CF4991F8D91C401A801CCD4901EB86
:10F32000800041880A4602910821032005F06AFB0B
:10F3300025E1C948007804287ED1012211461046F3
:10F34000F1F708FBFF20C44908700120C04981F88B
:10F35000D001002081F8DA0C084690F8D811BD4899
:10F3600030F8210007904FF47A71079890FBF1F084
:10F370000690069800EB4001C1EBC0120798A0EB85
:10F38000C20080B207906421079890FBF1F00590CD
:10F39000059800EBC00101EB00120798A0EB82007A
:10F3A00080B207900A21079890FBF1F0049004982E
:10F3B00000EB80020798A0EB4200079007980390AB
:10F3C00006983030A249A1F8DC0C0598303081B2A3
:10F3D0009F48A0F8DE1C0498303081B29C48A0F809
:10F3E000E01C0398303081B29948A0F8E21C90F8F4
:10F3F000D811984800EB8100408807904FF47A714B
:10F40000079890FBF1F00690069800EB4001C1EBE5
:10F41000C0120798A0EBC20080B207906421079841
:10F4200090FBF1F00590059800EBC00101EB001294
:10F430000798A0EB820000E084E080B207900A21E8
:10F44000079890FBF1F00490049800EB8002079875
:10F45000A0EB42000790079803900698303081B2E5
:10F460007B48A0F8E41C0598303081B27848A0F8B9
:10F47000E61C0498303081B27548A0F8E81C039867
:10F48000303081B27248A0F8EA1C90F8D90C401CC8
:10F49000C1B2029104210298F6F75CFA6C48B0F808
:10F4A000DC1C08460291F5F7E9FE6948B0F8DE1C5D
:10F4B00008460291F5F7E2FE6548B0F8E01C084600
:10F4C0000291F5F7DBFE6248B0F8E21C08460291B3
:10F4D000F5F7D4FE5E4890F8D90C401CC1B20291F9
:10F4E00008210298F6F736FA5948B0F8E41C0846A5
:10F4F0000291F5F7C3FE5648B0F8E61C08460291A3
:10F50000F5F7BCFE5248B0F8E81C08460291F5F742
:10F51000B5FE4F48B0F8EA1C08460291F5F7AEFE7A
:10F520004B4890F8DA0C0830C1B24948029190F883
:10F53000D90C401CC1B201220191DDE90101F5F7AE
:10F54000FFFE1CE044480078052818D1012211462E
:10F550001046F1F7FFF9FF203F49087002203C49AF
:10F5600081F8D001084690F8D90C401CC0B20023A5
:10F57000062219460290F5F797FE04F087FB33E365
:10F5800035480078032869D1012211461046F1F769
:10F59000E1F9FF20304908702D4890F8DA1C00F698
:10F5A000DC4030F81100202808D13021284890F89C
:10F5B000DA2C00F6DC4020F812102AE0244890F8FB
:10F5C000DA1C00F6DC4030F81100392810DA204847
:10F5D00090F8DA1C00F6DC4030F81100401C81B2D3
:10F5E0001B4890F8DA2C00F6DC4020F8121010E0EE
:10F5F000174890F8DA1C00F6DC4030F81100392882
:10F6000007D13021124890F8DA2C00F6DC4020F8BF
:10F6100012100F4890F8D90C401CC0B2042102907F
:10F62000F6F798F90A48B0F8DC1C08460291F5F79D
:10F6300025FE0748B0F8DE1C08460291F5F71EFECD
:10F640000348B0F8E01C08460291F5F717FE06E003
:10F650001C020020F80300201400002030E0FD48C8
:10F66000B0F8E21C08460291F5F708FEF94890F858
:10F67000D90C401CC1B2029108210298F6F76AF930
:10F68000F448B0F8E41C08460291F5F7F7FDF1489C
:10F69000B0F8E61C08460291F5F7F0FDED48B0F829
:10F6A000E81C01E0EAE3A0E208460291F5F7E6FD76
:10F6B000E848B0F8EA1C08460291F5F7DFFD93E24E
:10F6C000E548007898BB012211461046F1F742F94F
:10F6D000FF20E1490870DF4890F8DA1C00F6DC40B2
:10F6E00030F81100202808D13921DA4890F8DA2CB6
:10F6F00000F6DC4020F812102BE0D64890F8DA1C17
:10F7000000F6DC4030F81100302811DDD14890F8C7
:10F71000DA1C00F6DC4030F81100401E81B2CD4802
:10F7200090F8DA2C00F6DC4020F8121011E05EE0D0
:10F73000C84890F8DA1C00F6DC4030F81100302898
:10F7400007D13921C34890F8DA2C00F6DC4020F8C4
:10F750001210C04890F8D90C401CC0B2042102908D
:10F76000F6F7F8F8BB48B0F8DC1C08460291F5F74C
:10F7700085FDB848B0F8DE1C08460291F5F77EFD1D
:10F78000B448B0F8E01C08460291F5F777FDB1489F
:10F79000B0F8E21C08460291F5F770FDAD4890F80C
:10F7A000D90C401CC1B200E065E302910821029827
:10F7B000F6F7D0F8A748B0F8E41C08460291F5F730
:10F7C0005DFDA448B0F8E61C08460291F5F756FD29
:10F7D000A048B0F8E81C08460291F5F74FFD9D4897
:10F7E000B0F8EA1C08460291F5F748FDFCE19A489A
:10F7F0000078022864D1012211461046F1F7AAF8D8
:10F80000FF2095490870934890F8DA0C002844DDF1
:10F81000904890F8DA0C042811DA8E4890F8DA0C47
:10F820000830C0B202908B4890F8D90C401CC1B28D
:10F8300000220191DDE90101F5F782FD10E0854824
:10F8400090F8DA0C0C30C0B20290824890F8D90CD3
:10F85000401CC1B200220191DDE90101F5F770FD04
:10F860007C4890F8DA0C401E7A4981F8DA0C084698
:10F8700090F8DA0C042811DA084690F8DA0C08300F
:10F88000C0B20290084690F8D90C401CC1B20122C7
:10F890000191DDE90101F5F753FDA5E16D4890F80F
:10F8A000DA0C0C30C0B202906A4890F8D90C401CB7
:10F8B000C1B201220191DDE90101F5F741FD93E1BA
:10F8C00065480078072864D1012211461046F1F7F7
:10F8D00041F8FF20604908705E4890F8DA0C07286C
:10F8E00044DA5C4890F8DA0C042811DA594890F8A8
:10F8F000DA0C0830C0B20290564890F8D90C401C7F
:10F90000C1B200220191DDE90101F5F719FD10E016
:10F91000504890F8DA0C0C30C0B202904D4890F884
:10F92000D90C401CC1B200220191DDE90101F5F7BB
:10F9300007FD484890F8DA0C401C464981F8DA0C7B
:10F94000084690F8DA0C042811DA084690F8DA0C28
:10F950000830C0B20290084690F8D90C401CC1B2E1
:10F9600001220191DDE90101F5F7EAFC3CE13948AA
:10F9700090F8DA0C0C30C0B20290364890F8D90CEE
:10F98000401CC1B201220191DDE90101F5F7D8FC6B
:10F990002AE131480078052860D10122114610463D
:10F9A000F0F7D8FFFF202C4908700020294981F882
:10F9B000D001084690F8DA0C042811DA084690F8CD
:10F9C000DA0C0830C0B20290084690F8D90C401CFE
:10F9D000C1B200220191DDE90101F5F7B1FC10E0AF
:10F9E0001C4890F8DA0C0C30C0B20290194890F81C
:10F9F000D90C401CC1B200220191DDE90101F5F7EB
:10FA00009FFC144890F8D81100F5EE7030F82100F2
:10FA10000290104890F8D90C401CC1B20191042109
:10FA2000DDE9010204F0EEFF0A4890F8D81100F574
:10FA3000EE7000EB810041880648029190F8D90CE5
:10FA4000401CC1B201910821DDE9010204F0DAFF96
:10FA5000CAE003E01C02002014000020FE480078E9
:10FA600004287DD1012211461046F0F773FFFF20D4
:10FA7000F94908700020F94981F8D001084690F84A
:10FA8000DA0C042811DA084690F8DA0C0830C0B213
:10FA90000290084690F8D90C401CC1B20022019196
:10FAA000DDE90101F5F74CFC10E0EC4890F8DA0CC8
:10FAB0000C30C0B20290E94890F8D90C401CC1B299
:10FAC00000220191DDE90101F5F73AFC00212B91BB
:10FAD0000DE0E3482B9930F81100303882B2E0494C
:10FAE0002B9821F810202B98401C81B22B912B9839
:10FAF0000828EEDBD948B0F8DC0C4FF47A714843A3
:10FB0000D649B1F8DE1C01EBC10202EB011100EB9A
:10FB10008101D248B0F8E00C00EB800001EB40011D
:10FB2000CE48B0F8E20C084480B22B902B98B0F588
:10FB30007A7F07DAC94991F8D82101F5EE712B983F
:10FB400021F82200C548B0F8E40C4FF47A7148431C
:10FB5000C249B1F8E61C01EBC10202EB011100E061
:10FB600042E000EB8101BD48B0F8E80C00EB8000FA
:10FB700001EB4001B948B0F8EA0C084480B22B9080
:10FB80002B98B0F57A7F08DAB44991F8D82101F5BD
:10FB9000EE7101EB82012B984880B04890F8D811A3
:10FBA00000F5EE7030F821000290AC4890F8D90CC6
:10FBB000401CC1B201910421DDE9010204F022FFE1
:10FBC000A64890F8D81100F5EE7000EB810041884E
:10FBD000A248029190F8D90C401CC1B201910821B1
:10FBE000DDE9010204F00EFF46E19B48007805289C
:10FBF0007ED1012211461046F0F7ACFEFF20964957
:10FC0000087004212A914FF6FF712A9801EA4011E9
:10FC10002A9118AA20212A98F4F744FF00212A915A
:10FC200008E018A92A98095C08AA11542A98401CCF
:10FC300081B22A912A982028F3DB04212A912A985C
:10FC4000411C2A914FF6FF712A9801EA40112A912E
:10FC500018AA20212A98F4F725FF00212A9109E00B
:10FC600018A92A98095C08AA203011542A98401C27
:10FC700081B22A912A982028F2DB9DF85F0055284E
:10FC800059D1002120912A9152E02099481C82B23A
:10FC900008A82092425C73492A9821F820202A98CB
:10FCA00031F820004FF6FF7101EA00226D492A98D1
:10FCB00021F820202A9831F820202099481C83B26E
:10FCC00008A82093405C104482B266492A9821F823
:10FCD00020202099481C82B208A82092425C6149E9
:10FCE0002A9801EB800042802A9801EB800000E016
:10FCF00028E040884FF6FF7101EA002259492A980E
:10FD000001EB800042802A9801EB80004288209914
:10FD1000481C83B208A82093405C104482B2514929
:10FD20002A9801EB800042802A98401C81B22A91D7
:10FD30002A980F28A9DB30204B49087001204B4935
:10FD4000087097E04448007804287DD101221146CC
:10FD50001046F0F7FFFDFF203F4908700021209179
:10FD60002A912FE03F482A9930F821000212209969
:10FD7000481C83B208A8209342543A492A9811F8A3
:10FD800020202099481C83B208A82093425435496A
:10FD90002A9801EB8000408802122099481C83B207
:10FDA00008A8209342542F492A9801EB80008278BA
:10FDB0002099481C83B208A8209342542A98401CDA
:10FDC00081B22A912A980F28CCDB55218DF85F103B
:10FDD00000212A9108E008A92A98095C18AA115460
:10FDE0002A98401C81B22A912A982028F3DB04210A
:10FDF0002A914FF6FF712A9801EA40112A9118AA18
:10FE000020212A98F4F792FE00212A910AE008A9FD
:10FE10002A982030095C18AA2A9811542A98401C64
:10FE200081B22A912A982028F1DB04212A912A986C
:10FE3000411C2A914FF6FF712A9801EA40112A913C
:10FE400018AA20212A9800E014E0F4F76FFE302071
:10FE50000549087001200BE0140000201C0200205E
:10FE6000F80E0020F80300202C0000202E000020B7
:10FE7000FA49087000E000BF03F080B9F848007844
:10FE800035287DD1F5480078F0B30020F34908709B
:10FE900003F0AEFE0020F34981F8D001012081F883
:10FEA000D101002081F8D80181F8D90C084690F8DA
:10FEB000D80100EB4001EB48663030F811000246F3
:10FEC00006210290012004F0F9FDE64890F8D801DF
:10FED00000EB4001E348663000EB410041880A46F0
:10FEE00002910821012004F0E9FDDE4890F8D801D4
:10FEF00000EB4001DB48663000EB410081880A4698
:10FF000002910A21012000E06DE004F0D7FDD54800
:10FF100090F8D801401C00EB4001D248663030F820
:10FF200011100A4602910621022004F0C7FDCD48B7
:10FF300090F8D801401C00EB4001CA48663000EB45
:10FF4000410041880A4602910821022004F0B6FDD2
:10FF5000C44890F8D801401C00EB4001C14866300D
:10FF600000EB410081880A4602910A21022004F038
:10FF7000A5FDBC4890F8D801801C00EB400100E0D2
:10FF8000FEE3B848663030F811100A4602910621A7
:10FF9000032004F093FDB34890F8D801801C00EBD7
:10FFA0004001B048663000EB410041880A460291AA
:10FFB0000821032004F082FDAA4890F8D801801C93
:10FFC00000EB4001A748663000EB410081880A46FB
:10FFD00002910A21032004F071FD01230A2200216D
:10FFE0001846F5F761F99F4890F8D00120B1012833
:10FFF0007DD002287CD1FCE39A4890F8D8010928EA
:020000040801F1
:1000000040DA99480078E8BB012211461046F0F723
:10001000A1FCFF2094490870924890F8D801401C38
:10002000904981F8D801084690F8D90C02281DDAC9
:10003000084690F8D90C401CC0B200230A22194689
:100040000290F5F731F9874890F8D90C401C8549A2
:1000500081F8D90C084690F8D90C401CC1B2012394
:100060000A22029100210298F5F71EF97D4890F8C6
:10007000D8017C4991F8D91C411A01EB410000EBF1
:10008000C10000E0F4E079490844024600210290F2
:100090000120F5F7BBF9734890F8D801714991F840
:1000A000D91C401A00EB40016E48663030F8111040
:1000B0000A4602910621012004F000FD694890F8EB
:1000C000D801684991F8D91C401A00EB40016548F5
:1000D000663000EB410041880A4602910821012068
:1000E00004F0ECFC5F4890F8D8015E4901E0B7E30A
:1000F000FEE391F8D91C401A00EB400159486630E4
:1001000000EB410081880A4602910A21012004F097
:10011000D5FC544890F8D801524991F8D91C401A9E
:10012000401C00EB400101EBC000504901440A466D
:10013000029100210220F5F769F94A4890F8D801A8
:10014000484991F8D91C401A401C00EB4001454831
:10015000663030F811100A4602910621022004F0A0
:10016000ADFC404890F8D8013E4991F8D91C401A9E
:10017000401C00EB40013B48663000EB41004188E9
:100180000A4602910821022004F098FC354890F8B4
:10019000D801344991F8D91C401A401C00EB4001A9
:1001A0003048663000EB410081880A4602910A21FE
:1001B000022004F083FC2B4890F8D801294991F8DB
:1001C000D91C401A801C00EB400101EBC0002749FC
:1001D00001440A46029100210320F5F717F921484E
:1001E00090F8D8011F4991F8D91C401A801C00EBE7
:1001F00040011C48663030F811100A460291062171
:10020000032004F05BFC174890F8D801154991F8D9
:10021000D91C401A801C00EB40011248663000EBEC
:10022000410041880A4602910821032004F046FC5F
:100230000C4890F8D8010B4991F8D91C401A801C41
:1002400000EB40010748663000EB410081880A4618
:1002500002910A21032004F031FC00E32E0000206B
:100260002C0000201C020020140000204D00002063
:10027000FE4890F8D80100287EDDFD48007803286C
:100280007AD1012211461046F0F764FBFF20F849AD
:100290000870F64890F8D801401EF44981F8D8015A
:1002A000084690F8D90C00281DDD084690F8D90CB6
:1002B000401CC0B200230A2219460290F4F7F4FF52
:1002C000EA4890F8D90C401EE84981F8D90C084654
:1002D00090F8D90C401CC1B201230A2202910021DE
:1002E0000298F4F7E1FFE14890F8D801DF4991F86E
:1002F000D91C411A01EB410000EBC100DD49084463
:100300000246002102900120F5F780F8D74890F8C6
:10031000D801D64991F8D91C401A00EB4001D348C6
:10032000663030F811100A4602910621012004F0CF
:10033000C5FBCE4890F8D801CC4991F8D91C401A99
:1003400000EB4001C948663000EB410041880A4695
:1003500002910821012004F0B1FBC44890F8D801B3
:10036000C24991F8D91C401A00EB4001BF486630E1
:1003700000EB4100818800E0AAE00A4602910A21D0
:10038000012004F09BFBB94890F8D801B74991F8D7
:10039000D91C401A401C00EB400101EBC000B549DC
:1003A00001440A46029100210220F5F72FF8AF48D8
:1003B00090F8D801AD4991F8D91C401A401C00EBC7
:1003C0004001AA48663030F811100A460291062111
:1003D000022004F073FBA54890F8D801A34991F8D6
:1003E000D91C401A401C00EB4001A048663000EBCD
:1003F000410041880A4602910821022004F05EFB78
:100400009A4890F8D801994991F8D91C401A401C93
:1004100000EB40019548663000EB410081880A46B8
:1004200002910A21022004F049FB904890F8D8017B
:100430008E4991F8D91C401A801C00EB400101EB59
:10044000C0008C4901440A46029100210320F4F7C0
:10045000DDFF864890F8D801844991F8D91C401AEC
:10046000801C00EB40018148663030F811100A46CC
:1004700002910621032004F021FB7C4890F8D8016A
:100480007A4991F8D91C401A801C00EB400177484A
:10049000663000EB410041880A46029108210320A2
:1004A00004F00CFB714890F8D801704991F8D91C00
:1004B000401A801C00EB40016C48663000EB4100A4
:1004C00081880A4602910A21032004F0F7FAC6E166
:1004D0006748007804287CD1012211461046F0F7C5
:1004E00039FAFF20624908700120604981F8D00183
:1004F000002081F8DA0C084690F8D80100EB4001A2
:100500005A48663030F81100B0F57A7F0ADB2D20AA
:100510005649A1F8DC0C2D215448A0F8DE1CA0F8A7
:10052000E01C46E0514890F8D80100EB40014F48EC
:10053000663030F811002B9064212B9890FBF1F07D
:100540004A49A1F8DC0C0846B0F8DC1C01EBC100FC
:1005500000EB01112B98A0EB810081B22B910A21B5
:100560002B9890FBF1F081B24048A0F8DE1CB0F867
:10057000DE0C00EB80012B98A0EB410081B22B91A7
:100580003A492B98A1F8E00C0846B0F8DC0C303062
:10059000A1F8DC0C0846B0F8DE0C303081B23348EC
:1005A000A0F8DE1CB0F8E00C303081B22F48A0F883
:1005B000E01C2E4890F8D80100EB40012B48663033
:1005C00000EB41004088B0F57A7F0ADB2D212748F7
:1005D00000E027E1A0F8E21CA0F8E41CA0F8E61C6B
:1005E0004FE0224890F8D80100EB40011F486630E8
:1005F00000EB410040882B9064212B9890FBF1F098
:1006000081B21A48A0F8E21CB0F8E20C00EBC0017D
:1006100001EB00112B98A0EB810081B22B910A21F4
:100620002B9890FBF1F081B21048A0F8E41CB0F8D0
:10063000E40C00EB80012B98A0EB410081B22B91E0
:100640000A492B98A1F8E60C0846B0F8E20C3030C5
:1006500081B20648A0F8E21CB0F8E40C303081B258
:100660000248A0F8E41CB0F8E60C05E01C020020EB
:10067000140000204D000020303081B2FE48A0F868
:10068000E61CFD4890F8D80100EB4001FA486630BE
:1006900000EB41008088B0F57A7F08DB2D21F64819
:1006A000A0F8E81CA0F8EA1CA0F8EC1C48E0F2480E
:1006B00090F8D80100EB4001EF48663000EB4100B4
:1006C00080882B9064212B9890FBF1F081B2EA484E
:1006D000A0F8E81CB0F8E80C00EBC00101EB001139
:1006E0002B98A0EB810081B22B910A212B9890FBD3
:1006F000F1F081B2E048A0F8EA1CB0F8EA0C00EB97
:1007000080012B98A0EB410081B22B91DA492B9804
:10071000A1F8EC0C0846B0F8E80C303081B2D648AD
:10072000A0F8E81CB0F8EA0C303081B2D248A0F84A
:10073000EA1CB0F8EC0C303081B2CF48A0F8EC1CC9
:10074000CD4890F8D90C401CC0B206210290F5F7B4
:1007500001F9C948B0F8DC1C08460291F4F78EFD97
:10076000C548B0F8DE1C08460291F4F787FDC24880
:10077000B0F8E01C08460291F4F780FDBE4800E0A6
:10078000FEE390F8D90C401CC1B2029108210298F6
:10079000F5F7E0F8B848B0F8E21C08460291F4F723
:1007A0006DFDB548B0F8E41C08460291F4F766FD0B
:1007B000B148B0F8E61C08460291F4F75FFDAE4878
:1007C00090F8D90C401CC1B202910A210298F5F7A9
:1007D000C1F8A948B0F8E81C08460291F4F74EFDAC
:1007E000A548B0F8EA1C08460291F4F747FDA24874
:1007F00000E0FDE3B0F8EC1C08460291F4F73EFD82
:100800009D4890F8DA0C0C30C1B29B48029190F8E8
:10081000D90C401CC1B201220191DDE90101F4F7BC
:100820008FFD1CE095480078052818D1012211465B
:100830001046F0F78FF8FF209049087002208E498B
:1008400081F8D001084690F8D90C401CC0B20023B2
:100850000A2219460290F4F727FD03F017FAFDE388
:100860008648007803287DD1012211461046F0F712
:1008700071F8FF20814908707F4890F8DA1C00F673
:10088000DC4030F81100202808D130217A4890F857
:10089000DA2C00F6DC4020F812102CE0764890F8B4
:1008A000DA1C00F6DC4030F81100392810DA724802
:1008B00090F8DA1C00F6DC4030F81100401C81B2E0
:1008C0006D4890F8DA2C00F6DC4020F8121012E0A7
:1008D000694890F8DA1C00F6DC4030F8110039283D
:1008E00009D13021644890F8DA2C00F6DC4000E0B1
:1008F000FEE320F81210604890F8D90C401CC0B2FA
:1009000006210290F5F726F85B48B0F8DC1C084693
:100910000291F4F7B3FC5848B0F8DE1C0846029187
:10092000F4F7ACFC5448B0F8E01C08460291F4F728
:10093000A5FC514890F8D90C401CC1B20291082185
:100940000298F5F707F84C48B0F8E21C0846029107
:10095000F4F794FC4848B0F8E41C08460291F4F718
:100960008DFC00E026E04448B0F8E61C0846029101
:10097000F4F784FC404890F8D90C401CC1B20291B5
:100980000A210298F4F7E6FF3B48B0F8E81C084655
:100990000291F4F773FC3848B0F8EA1C084602915B
:1009A000F4F76CFC3448B0F8EC1C08460291F4F7FC
:1009B00065FC6FE33148007898BB01221146104670
:1009C000EFF7C8FFFF202D4908702B4890F8DA1C7C
:1009D00000F6DC4030F81100202808D139212648E3
:1009E00090F8DA2C00F6DC4020F812102BE02248B8
:1009F00090F8DA1C00F6DC4030F81100302811DDE8
:100A00001D4890F8DA1C00F6DC4030F81100401E5A
:100A100081B2194890F8DA2C00F6DC4020F8121068
:100A200011E072E0144890F8DA1C00F6DC4030F86F
:100A30001100302807D139210F4890F8DA2C00F640
:100A4000DC4020F812100C4890F8D90C401CC0B2C1
:100A500006210290F4F77EFF0748B0F8DC1C084638
:100A60000291F4F70BFC0448B0F8DE1C0846029132
:100A7000F4F704FC004803E01C02002014000020EE
:100A8000B0F8E01C08460291F4F7F8FBFE4890F835
:100A9000D90C401CC1B2029108210298F4F75AFF08
:100AA000F948B0F8E21C08460291F4F7E7FBF64873
:100AB000B0F8E41C08460291F4F7E0FBF248B0F805
:100AC000E61C08460291F4F7D9FBEF4890F8D90CE0
:100AD000401CC1B202910A210298F4F73BFFEA4898
:100AE000B0F8E81C08460291F4F7C8FBE648B0F8F5
:100AF000EA1C08460291F4F7C1FBE348B0F8EC1C8D
:100B000008460291F4F7BAFBC4E2E04800780228F4
:100B10007ED1012211461046EFF71CFFFF20DB4972
:100B20000870D94890F8DA0C00285BDDD64890F8B8
:100B3000DA0C032811DAD44890F8DA0C0C30C0B281
:100B40000290D14890F8D90C401CC1B2002201910A
:100B5000DDE90101F4F7F4FB27E0CB4890F8DA0C6B
:100B6000062811DAC84890F8DA0C0D30C0B20290AD
:100B7000C54890F8D90C401CC1B200220191DDE9B2
:100B80000101F4F7DDFB10E0BF4890F8DA0C0E30FD
:100B9000C0B20290BC4890F8D90C401CC1B20022EF
:100BA0000191DDE90101F4F7CBFBB74890F8DA0CCD
:100BB000401EB54981F8DA0C084690F8DA0C032893
:100BC00011DA084690F8DA0C0C30C0B202900846F0
:100BD00090F8D90C401CC1B201220191DDE901015C
:100BE000F4F7AEFB56E2A84890F8DA0C062813DAC0
:100BF000A54890F8DA0C0D30C0B20290A24890F8E7
:100C0000D90C401CC1B201220191DDE9010100E0D3
:100C100014E0F4F795FB3DE29B4890F8DA0C0E30B7
:100C2000C0B20290984890F8D90C401CC1B2012281
:100C30000191DDE90101F4F783FB2BE29348007891
:100C400007287CD1012211461046EFF783FEFF20D2
:100C50008E4908708C4890F8DA0C08285BDA8A48CC
:100C600090F8DA0C032811DA874890F8DA0C0C3087
:100C7000C0B20290844890F8D90C401CC1B2002246
:100C80000191DDE90101F4F75BFB27E07E4890F874
:100C9000DA0C062811DA7C4890F8DA0C0D30C0B274
:100CA0000290794890F8D90C401CC1B20022019101
:100CB000DDE90101F4F744FB10E0734890F8DA0C29
:100CC0000E30C0B20290704890F8D90C401CC1B2EE
:100CD00000220191DDE90101F4F732FB6A4890F846
:100CE000DA0C401C684981F8DA0C084690F8DA0CF6
:100CF000032811DA084690F8DA0C0C30C0B20290E2
:100D0000084690F8D90C401CC1B201220191DDE9DE
:100D10000101F4F715FBBDE15B4890F8DA0C0628F9
:100D200013DA594890F8DA0C0D30C0B202905648E8
:100D300090F8D90C401CC1B20122019100E016E0EC
:100D4000DDE90101F4F7FCFAA4E14F4890F8DA0C70
:100D50000E30C0B202904C4890F8D90C401CC1B281
:100D600001220191DDE90101F4F7EAFA92E1474835
:100D7000007805287DD1012211461046EFF7EAFDE3
:100D8000FF204249087000203F4981F8D001084601
:100D900090F8DA0C032811DA084690F8DA0C0C30D7
:100DA000C0B20290084690F8D90C401CC1B2002293
:100DB0000191DDE90101F4F7C3FA27E0324890F828
:100DC000DA0C062811DA304890F8DA0C0D30C0B28F
:100DD00002902D4890F8D90C401CC1B2002201911C
:100DE000DDE90101F4F7ACFA10E0274890F8DA0CDD
:100DF0000E30C0B20290244890F8D90C401CC1B209
:100E000000220191DDE90101F4F79AFA1E4890F8F9
:100E1000D80100EB40011C48663030F81100029008
:100E2000194890F8D90C401CC1B201910621DDE9A6
:100E3000010203F043FE144890F8D80100EB400192
:100E40001148663000EB410041880F48029190F84C
:100E5000D90C401CC1B201910821DDE9010203F067
:100E60002DFE094890F8D80100EB40010648663095
:100E700000E014E000EB410081880348029190F803
:100E8000D90C401CC1B203E01C0200201400002059
:100E900001910A21DDE9010203F010FEFAE0FE48AB
:100EA000007804286DD1012211461046EFF752FD5B
:100EB000FF20F94908700020F84981F8D001084660
:100EC00090F8DA0C032811DA084690F8DA0C0C30A6
:100ED000C0B20290084690F8D90C401CC1B2002262
:100EE0000191DDE90101F4F72BFA27E0EB4890F8D6
:100EF000DA0C062811DAE94890F8DA0C0D30C0B2A5
:100F00000290E64890F8D90C401CC1B20022019131
:100F1000DDE90101F4F714FA10E0E04890F8DA0C8A
:100F20000E30C0B20290DD4890F8D90C401CC1B21E
:100F300000220191DDE90101F4F702FA00202B9073
:100F40000DE0D7482B9930F81100303882B2D449DF
:100F50002B9821F810202B98401C81B22B912B98B4
:100F60000928EEDBCD48B0F8DC0C64214843CB49BE
:100F7000B1F8DE1C01EB810100EB4101C74801E043
:100F800050E287E0B0F8E00C084481B2C34890F822
:100F9000D80100EB4002C148663020F812106638D4
:100FA000B0F8E20C64214843BC49B1F8E41C01EB01
:100FB000810100EB4101B948B0F8E60C084481B268
:100FC000B64890F8D80100EB4002B448663000EB18
:100FD00042004180B148B0F8E80C64214843AF4971
:100FE000B1F8EA1C01EB810100EB4101AB4800E0E4
:100FF00051E0B0F8EC0C084481B2A84890F8D80150
:1010000000EB4002A548663000EB42008180A34817
:1010100090F8D80100EB4001A048663030F811008C
:1010200002909E4890F8D90C401CC1B20191062153
:10103000DDE9010203F042FD984890F8D80100EB89
:1010400040019648663000EB410041889348029188
:1010500090F8D90C401CC1B2019100E0E0E10821F8
:10106000DDE9010203F02AFD8C4890F8D80100EB7D
:1010700040018A48663000EB410081888748029130
:1010800090F8D90C401CC1B201910A21DDE901029E
:1010900003F014FDC4E18048007805287DD10122C9
:1010A00011461046EFF756FCFF207B4908700621D9
:1010B0002A914FF6FF712A9801EA40112A9118AA45
:1010C00020212A98F3F7EEFC00212A9108E018A9C4
:1010D0002A98095C08AA11542A98401C81B22A91C6
:1010E0002A982028F3DB06212A912A98411C00E047
:1010F00095E12A914FF6FF712A9801EA40112A9151
:1011000018AA20212A98F3F7CDFC00212A9109E0A2
:1011100018A92A98095C08AA203011542A98401C62
:1011200081B22A912A982028F2DB9DF85F00552889
:101130007ED1002120912A91B7E02099481C82B2EB
:1011400008A82092415C2A9800EB40025348663080
:1011500020F812102A9800EB40015048663030F811
:1011600011004FF6FF7101EA00212A9800EB4002BE
:101170004A48663020F812102A9800EB4001474890
:10118000663030F811202099481C83B208A82093BB
:10119000405C104481B22A9800E091E000EB4002EC
:1011A0003E48663020F812102099481C82B208A8E8
:1011B0002092415C2A9800EB40023848663000EBF0
:1011C000420041802A9800EB40013448663000EB31
:1011D000410040884FF6FF7101EA00212A9800EB98
:1011E00040022E48663000EB420041802A9800EB16
:1011F00040012A48663000EB410042882099481C93
:1012000083B208A82093405C104481B22A9800EB76
:1012100040022248663000EB420041802099481C81
:1012200082B208A82092415C2A9800EB400200E0BC
:101230003FE01A48663000EB420081802A9800EBBC
:1012400040011648663000EB410080884FF6FF7180
:1012500001EA00212A9800EB40021048663000EBBA
:10126000420081802A9800EB40010C48663000EB78
:10127000410082882099481C83B208A82093405CD2
:10128000104481B22A9800EB40020448663000EB1B
:10129000420081802A9805E0140000201C020020F2
:1012A000F80E0020401C81B22A912A980A28FFF6E5
:1012B00044AF3020F94908700120F9490870ADE0C9
:1012C000F848007804287DD1012211461046EFF736
:1012D00041FBFF20F3490870002120912A9152E040
:1012E0002A9800EB4001F04830F8110002122099D2
:1012F000481C83B208A8209342542A9800EB40016E
:10130000E94810F811202099481C83B208A82093BE
:1013100042542A9800EB4001E34800EB410040882A
:1013200002122099481C83B208A8209342542A989C
:1013300000EB4001DC4800EB410082782099481C1A
:1013400083B208A8209342542A9800EB4001D64863
:1013500000EB4100808802122099481C83B208A843
:10136000209342542A9800EB4001CF4800EB410003
:1013700002792099481C83B208A8209342542A98E5
:10138000401C81B22A912A980A28A9DB55218DF8A0
:101390005F1000212A9108E008A92A98095C18AA80
:1013A00011542A98401C81B22A912A982028F3DBF4
:1013B00006212A914FF6FF712A9801EA40112A91DD
:1013C00018AA00E02AE020212A98F3F7AFFB0021B9
:1013D0002A910AE008A92A982030095C18AA2A98BC
:1013E00011542A98401C81B22A912A982028F1DBB6
:1013F00006212A912A98411C2A914FF6FF712A98BA
:1014000001EA40112A9118AA20212A98F3F78EFBAD
:101410003020A24908700120A149087000E000BFF7
:1014200001F0ACBE9D480078332872D19C4800780A
:10143000F0B300209A49087002F0B6FC00209A49E7
:10144000663981F8D001012081F8D101002081F8AE
:10145000D80181F8D90C954A0721022002F082FEBA
:10146000924880790009924908709048807900F08C
:101470000F0048708D484079C0F3001088708B4889
:10148000407900F00F00C8708848C078C0F30110A0
:1014900008718648C07800F00F0048718348807852
:1014A000C0F3011088718148807800F00F0000E0DF
:1014B00027E0C8717D484078C0F3021008727B486D
:1014C000407800F00F00487278480078C0F30210AE
:1014D00088727648007800F00F00C8720A46022130
:1014E000012003F0FAFB7048663890F8D801714982
:1014F000085C001DC0B20122014602901046F3F7BD
:101500001FFF6948663890F8D00118B102287DD1D4
:1015100004E160E16348007840BB012211461046B7
:10152000EFF718FAFF205F4908705F48663890F8B7
:10153000D8015F49085C60B15B48663890F8D80113
:10154000085C401E5849663991F8D811584A5054E1
:1015500006E009205449663991F8D811544A50548C
:10156000534A0221012003F0B8FBD6E04D48007831
:10157000032829D1012211461046EFF7EBF9FF208D
:10158000484908704848663890F8D8014849085CCE
:1015900009280CDA4448663890F8D801085C401CE9
:1015A0004149663991F8D811414A505406E000206B
:1015B0003D49663991F8D8113D4A50543C4A0221C0
:1015C000012003F08AFBA8E03648007802283AD1CF
:1015D000012211461046EFF7BDF9FF20314908708E
:1015E0003148663890F8D8013249085C001DC0B215
:1015F0000022014602900120F3F7A2FE2A48663835
:1016000090F8D80158B12848663800E0E1E090F839
:10161000D801401E2449663981F8D80104E00B2026
:101620002149663981F8D8011F48663890F8D801F9
:101630002049085C001DC0B20122014602901046FC
:10164000F3F77EFE69E017480078072846D10122AB
:1016500011461046EFF77EF9FF2012490870124834
:10166000663890F8D8011349085C001DC0B200220A
:10167000014602900120F3F763FE0B48663890F8AC
:10168000D8010B2818DA0848663890F8D801401CB1
:101690000549663981F8D80112E000002C000020CD
:1016A0002E000020140000208202002046000020AE
:1016B000EA440020386401080020FE4981F8D8017E
:1016C000FC4890F8D801FC49085C001DC0B201221A
:1016D000014602901046F3F733FE1EE0F74800780B
:1016E00005281AD1012211461046EFF733F9FF20E1
:1016F000F24908700220EF4981F8D001084690F8BD
:10170000D801ED49085C001DC0B2002201460290DC
:101710000120F3F715FE02F0B9FA5BE0E748007824
:1017200005280ED1012211461046EFF713F9FF20CC
:10173000E24908703020E24908700120E149087050
:1017400046E0DE480078042842D1012211461046C6
:10175000EFF700F9FF20D9490870DB484078DA49F3
:10176000097800EB0110D9498871D748C078D6496B
:10177000897800EB0110D5494871D3484079D249A6
:10178000097900EB0110D149C870CF48C079CE4922
:10179000897900EB0110CD498870CB48407ACA495D
:1017A000097A00EB0110C9494870C748C07AC64998
:1017B000897A00EB0110C54908700A46072102200A
:1017C00002F0F6FC3020BE4908700120BD490870C7
:1017D00000E000BF24E6BA48007836287ED1B94838
:1017E0000078E8B30020B749087002F08FFA0020B3
:1017F000B04981F8D001012081F8D101002081F8A1
:10180000D80181F8D90C084690F8D80100EB4001C6
:10181000A848A23030F811000246062102900120AB
:1018200003F04CF9A34890F8D80100EB4001A1481F
:10183000A23000EB410041880A46029108210120B4
:1018400003F03CF99B4890F8D80100EB400199481F
:10185000A23000EB410081880A4602910A2100E093
:101860006EE0012003F02AF9924890F8D801401C5C
:1018700000EB40018F48A23030F811100A46029167
:101880000621022003F01AF98A4890F8D801401C7A
:1018900000EB40018748A23000EB410041880A4636
:1018A00002910821022003F009F9824890F8D8013A
:1018B000401C00EB40017F48A23000EB41008188D2
:1018C0000A4602910A21022003F0F8F8794890F8BC
:1018D000D801801C00EB4001764800E0FDE3A23017
:1018E00030F811100A4602910621032003F0E6F8B1
:1018F000704890F8D801801C00EB40016D48A23080
:1019000000EB410041880A4602910821032003F0C0
:10191000D5F8684890F8D801801C00EB4001654874
:10192000A23000EB410081880A4602910A2103207F
:1019300003F0C4F801230A2200211846F3F7B4FC8F
:101940005C4890F8D00120B101287DD002287CD1DC
:10195000FEE3584890F8D801092841DA5748007842
:10196000F0BB012211461046EEF7F4FFFF20534969
:101970000870504890F8D801401C4E4981F8D801B1
:10198000084690F8D90C02281DDA084690F8D90CC0
:10199000401CC0B200230A2219460290F3F784FCCF
:1019A000444890F8D90C401C424981F8D90C0846AB
:1019B00090F8D90C401CC1B201230A2202910021E7
:1019C0000298F3F771FC3B4890F8D801394991F837
:1019D000D91C401A00EB400101EBC0003C4900E07B
:1019E000FAE008440246002102900120F3F70EFDC0
:1019F000304890F8D8012F4991F8D91C401A00EBD3
:101A000040012C48A23030F811100A4602910621FC
:101A1000012003F053F8274890F8D801254991F8A0
:101A2000D91C401A00EB40012248A23000EB4100D3
:101A300041880A4602910821012003F03FF81D4821
:101A400090F8D8011B4901E0BEE3F5E391F8D91CF9
:101A5000401A00EB40011748A23000EB410081889A
:101A60000A4602910A21012003F028F8114890F853
:101A7000D801104991F8D91C401A401C00EB4001D4
:101A800001EBC000124901440A46029100210220E4
:101A9000F3F7BCFC074890F8D801064991F8D91C27
:101AA000401A401C00EB40010248A23030F81110EF
:101AB0000A460FE01C0200203864010814000020D0
:101AC0002C0000202E000020EA44002046000020C8
:101AD000BB00002002910621022002F0EFFFFE4829
:101AE00090F8D801FC4991F8D91C401A401C00EB31
:101AF0004001F948A23000EB410041880A460291BA
:101B00000821022002F0DAFFF34890F8D801F249E8
:101B100091F8D91C401A401C00EB4001EE48A2305D
:101B200000EB410081880A4602910A21022002F05E
:101B3000C5FFE94890F8D801E74991F8D91C401A47
:101B4000801C00EB400101EBC000E44901440A465F
:101B5000029100210320F3F759FCDF4890F8D801E7
:101B6000DD4991F8D91C401A801C00EB4001DA488D
:101B7000A23030F811100A4602910621032002F02B
:101B80009DFFD54890F8D801D34991F8D91C401A47
:101B9000801C00EB4001D048A23000EB410041889E
:101BA0000A4602910821032002F088FFCA4890F8F3
:101BB000D801C94991F8D91C401A801C00EB40019A
:101BC000C548A23000EB410081880A4602910A21F3
:101BD000032002F073FFF6E2BF4890F8D801002816
:101BE0007EDDBF48007803287AD1012211461046D5
:101BF000EEF7B0FEFF20BA490870B74890F8D80158
